:020000040800F2
:203000008029002001310008C31A0108B9C50008C1190108354B0008C55C010800000000AC
:2030200000000000000000000000000023360108016E000800000000251E01088545010898
:203040001B3100081B3100081B3100081B3100081B3100081B3100081B3100081B310008D0
:20306000097400081B3100081B310008855B00081B3100081B3100081B3100081B310008EB
:203080001B3100081B310008C54200081B31000849550108394B00081B3100081B3100084A
:2030A0001B310008B14601081B3100081B3100081B3100081B3100081B3100081B310008C4
:2030C0001B3100081B3100081B3100081B3100081B3100081B3100081B3100085D540108EA
:2030E000FD7300081B3100081B310008DFF80CD001F098F800480047A14200088029002039
:203100000648804706480047FEE7FEE7FEE7FEE7FEE7FEE7FEE7FEE7FEE7FEE7594601086B
:20312000ED3000082DE9FF1F002000210022002300240025002600275FF000085FF000096B
:203140005FF0000A5FF0000B5FF0000C002001210222032304240525062607275FF00808CA
:203160005FF009095FF00A0A5FF00B0B5FF00C0C00281DD101291BD1022A19D1032B17D167
:20318000042C15D1052D13D1062E11D1072F0FD1B8F1080F0CD1B9F1090F09D1BAF10A0FDA
:2031A00006D1BBF10B0F03D1BCF10C0F00D101E004F002BCBDE8FF1F7047000073B40020B1
:2031C00000210124002501262046A04226D1A94224D12846A84221D1A9421FD14FEA440498
:2031E00006F10106202EEFDD5FF0FF305FF0FF317FF000445FF0FF3501262046A0420DD137
:20320000A9420BD12846A84208D1A94206D14FEA740406F10106202EEFDD01E004F0CCBBCF
:2032200073BC7047E7B40021002000220125002601272946A94230D1B0422ED1B2422CD1F9
:203240003146B14229D1B04227D1B24225D14FEA450507F10107202FEBDD5FF0FF315FF0CE
:20326000FF305FF0FF327FF000455FF0FF3601272946A94211D1B0420FD1B2420DD13146E8
:20328000B1420AD1B04208D1B24206D14FEA750507F10107202FEBDD01E004F08DBBE7BC40
:2032A00070472DE9CE01002200210023012600275FF001083246B24233D1B94231D1BB42FC
:2032C0002FD13A46BA422CD1B9422AD1BB4228D14FEA460608F10108B8F1200FEADD5FF014
:2032E000FF325FF0FF315FF0FF337FF000465FF0FF375FF001083246B24212D1B94210D1E0
:20330000BB420ED13A46BA420BD1B94209D1BB4207D14FEA760608F10108B8F1200FEADD79
:2033200001E004F049BBBDE8CE0170472DE99C0300230022002401275FF000085FF0010993
:203340003B46BB4233D1424531D144452FD1434643452CD142452AD1444528D14FEA470740
:2033600009F10109B9F1200FEADD5FF0FF335FF0FF325FF0FF347FF000475FF0FF385FF09B
:2033800001093B46BB4212D1424510D144450ED1434643450BD1424509D1444507D14FEA0A
:2033A000770709F10109B9F1200FEADD01E004F003BBBDE89C0370472DE9381C00240023AC
:2033C00000255FF0010A5FF0000B5FF0010C5446544533D15B4531D15D452FD15C465C45FA
:2033E0002CD15B452AD15D4528D14FEA4A0A0CF1010CBCF1200FEADD5FF0FF345FF0FF335D
:203400005FF0FF357FF0004A5FF0FF3B5FF0010C5446544512D15B4510D15D450ED15C46D1
:203420005C450BD15B4509D15D4507D14FEA7A0A0CF1010CBCF1200FEADD01E004F0BCBA66
:20344000BDE8381C70472DE9701C0025002400265FF0010A5FF0000B5FF0010C5546554566
:2034600033D15C4531D15E452FD15D465D452CD15C452AD15E4528D14FEA4A0A0CF1010CF1
:20348000BCF1200FEADD5FF0FF355FF0FF345FF0FF367FF0004A5FF0FF3B5FF0010C5546C7
:2034A000554512D15C4510D15E450ED15D465D450BD15C4509D15E4507D14FEA7A0A0CF1BA
:2034C000010CBCF1200FEADD01E004F075BABDE8701C70472DE9E01C0026002500275FF07D
:2034E000010A5FF0000B5FF0010C5646564533D15D4531D15F452FD15E465E452CD15D45A2
:203500002AD15F4528D14FEA4A0A0CF1010CBCF1200FEADD5FF0FF365FF0FF355FF0FF374D
:203520007FF0004A5FF0FF3B5FF0010C5646564512D15D4510D15F450ED15E465E450BD1AA
:203540005D4509D15F4507D14FEA7A0A0CF1010CBCF1200FEADD01E004F02EBABDE8E01CAB
:2035600070472DE9C01D002700265FF000085FF0010A5FF0000B5FF0010C5746574533D1B0
:203580005E4531D1D8452FD15F465F452CD15E452AD1D84528D14FEA4A0A0CF1010CBCF12B
:2035A000200FEADD5FF0FF375FF0FF365FF0FF387FF0004A5FF0FF3B5FF0010C57465745AF
:2035C00012D15E4510D1D8450ED15F465F450BD15E4509D1D84507D14FEA7A0A0CF1010C2A
:2035E000BCF1200FEADD01E004F0E6B9BDE8C01D70472DE9801F5FF0000800275FF00009F0
:203600005FF0010A5FF0000B5FF0010CD046D04533D15F4531D1D9452FD1D846D8452CD16F
:203620005F452AD1D94528D14FEA4A0A0CF1010CBCF1200FEADD5FF0FF385FF0FF375FF040
:20364000FF397FF0004A5FF0FF3B5FF0010CD046D04512D15F4510D1D9450ED1D846D845C9
:203660000BD15F4509D1D94507D14FEA7A0A0CF1010CBCF1200FEADD01E004F09DB9BDE8C0
:20368000801F70472DE970075FF000095FF000085FF0000A012400250126A146A14530D100
:2036A000A8452ED1AA452CD1A946A94529D1A84527D1AA4525D14FEA440406F10106202EC4
:2036C000EBDD5FF0FF395FF0FF385FF0FF3A7FF000445FF0FF350126A146A14511D1A84594
:2036E0000FD1AA450DD1A946A9450AD1A84508D1AA4506D14FEA740406F10106202EEBDD14
:2037000001E004F059B9BDE8700770472DE9700E5FF0000A5FF000095FF0000B0124002506
:203720000126A246A24530D1A9452ED1AB452CD1AA46AA4529D1A94527D1AB4525D14FEADA
:20374000440406F10106202EEBDD5FF0FF3A5FF0FF395FF0FF3B7FF000445FF0FF35012618
:20376000A246A24511D1A9450FD1AB450DD1AA46AA450AD1A94508D1AB4506D14FEA740403
:2037800006F10106202EEBDD01E004F015B9BDE8700E70472DE9701C5FF0000B5FF0000A43
:2037A0005FF0000C012400250126A346A34530D1AA452ED1AC452CD1AB46AB4529D1AA45C5
:2037C00027D1AC4525D14FEA440406F10106202EEBDD5FF0FF3B5FF0FF3A5FF0FF3C7FF06B
:2037E00000445FF0FF350126A346A34511D1AA450FD1AC450DD1AB46AB450AD1AA4508D106
:20380000AC4506D14FEA740406F10106202EEBDD01E004F0D1B8BDE8701C70472DE9701837
:203820005FF0000C5FF0000B012400250126A446A44526D1AB4524D1AC46AC4521D1AB45EE
:203840001FD14FEA440406F10106202EEFDD5FF0FF3C5FF0FF3B7FF000445FF0FF3501266F
:20386000A446A4450DD1AB450BD1AC46AC4508D1AB4506D14FEA740406F10106202EEFDD7F
:2038800001E004F099B8BDE8701870472DE9F0030024002546594E51445105F10405182DB5
:2038A000F8DB04255FF0000801245FF0010944514659B4425FD105F10407C659B0455AD19D
:2038C0002F1FC659B04556D140F805804659B04551D105F10407C659B0454CD12F1FC6594D
:2038E000B04548D14FEA440409F10109B9F1200FDDDD05F10405142DD6DB5FF0FF3400250A
:20390000445105F10405182DFADB04255FF0FF387FF000445FF0010944514659B4422AD119
:2039200005F10407C659B04525D12F1FC659B04521D140F805804659B0451CD105F10407E9
:20394000C659B04517D12F1FC659B04513D14FEA740409F10109B9F1200FDDDD05F10405DE
:20396000142DD5DB00254E59465105F10405182DF9DB012000E00020BDE8F00370472DE955
:20398000F00300240025445105F104058D42FADB00255FF0000801245FF001094451465985
:2039A000B44268D1002D03D02F1FC659B04562D105F104078F4202DAC659B0455BD140F81D
:2039C00005804659B04556D1002D03D02F1FC659B04550D105F104078F4202DAC659B04562
:2039E00049D14FEA440409F10109B9F1200FD5DD05F104058D42CEDB5FF0FF3400254451EA
:203A000005F104058D42FADB00255FF0FF387FF000445FF0010944514659B4422BD1002DF9
:203A200003D02F1FC659B04525D105F104078F4202DAC659B0451ED140F805804659B04559
:203A400019D1002D03D02F1FC659B04513D105F104078F4202DAC659B0450CD14FEA7404E6
:203A600009F10109B9F1200FD5DD05F104058D42CDDB012000E00020BDE8F0037047202A87
:203A800004DB203A21FA02F00021704721FA02F3D040C2F12002914008431946704740EAB7
:203AA00001039B0703D009E008C9121F08C0042AFAD203E011F8013B00F8013B521EF9D249
:203AC0007047D2B201E000F8012B491EFBD270470022F6E710B513460A4604461946FFF7AF
:203AE000F0FF204610BD10B5044604E00B7800F8013B03B1491C521EF8D2204610BD421C16
:203B000010F8011B0029FBD1801A704730B505460020034600E05B1C934205D2EC5CC85C33
:203B2000201A01D1002CF6D130BD2DE9F0410546002090460E46044600E0641C44450BD2AD
:203B4000285D00F083FA0746305D00F07FFA381A02D1295D0029F0D1BDE8F081F0B480EA77
:203B60000102D40F4200B2EB410F02D20246084611464A0042D0C30DDDB2C1F3C752AD1A20
:203B8000202D35DAC1F3160141F4000204B15242C5F1200602FA06F12A411044B3EBD05F23
:203BA00023D0C4B1012DA0EBC35009DCF0BC4FF0004202EAC352DBB200F5000000F055BA3D
:203BC000400000F1807000EBC350A0F1807040EAD170490009E0490841EAC071A0EBC3505D
:203BE00000F50000400800EBC350F0BC00F034BA6142012202EB4101001BF6E7F0BC7047B0
:203C000081F00041AAE780F00040A7E780EA010210B502F00043400022D04A001FD0010E42
:203C200001EB1261C0F35600C2F3560240F4000042F40002A0FB022000047F39140400D042
:203C4000401C50EA124001D44000491EC2B20C0604EBD010401C4008802A02D003E0002088
:203C600010BD20F00100002900DA0020184310BD2DE9FE4F804681EA0300C00F0C460090D3
:203C800021F0004123F00045B8EB0200A94105D24046214690461C460B46024623F0004003
:203CA000104347D0270DC7F30A00C3F30A510290401A019040286BDAC3F3130040F4801BCF
:203CC0000098924620B10023D2EB030A63EB0B0B01985946C0F14002504600F096F90646C6
:203CE0000D4650465946019A00F09EF910EB08006141002487EA115284EAE7731A4340D048
:203D0000009A62B3019A012A4FEA075215DC001B61EB02014FF0004202EA0752CDE9004283
:203D2000001C41F5801132462B4600F0DBF903B0BDE8F08F40462146F9E7001B61EB0201E5
:203D4000001C41F5801300185B412018A2F5001747EB030140EAD570B6196D4111E06D085C
:203D60004FEA360645EAC0754FEA0752001B61EB0201001C41F5801149084FEA30000019B8
:203D8000514132462B4603B0BDE8F04F00F09BB90098012240000023D0EB020263EBE0734F
:203DA000009821464FEAE074B8EB000061EB0401E9E783F000435BE781F0004158E72DE9B4
:203DC000F04D81EA030404F0004B21F0004514464FF0000A23F0004150EA050220D054EA39
:203DE00001021DD0C5F30A570246C5F31303C1F31300C1F30A5640F4801543F48013A7EBA4
:203E00000608101BD64608F2FD3873EB050002D308F1010801E092185B41B8F1000F03DA28
:203E200000200146BDE8F08D00204FF48011064684460EE0171B73EB050705D3121B63EB12
:203E4000050306434CEA010C49084FEA300092185B4150EA0107EDD152EA030012D082EA41
:203E6000040083EA0501084305D0101BAB4106D20122002306E000224FF0004302E06FF0AB
:203E8000010253101AEB06004CEB085110EB0A0041EB0B01BDE8F04D00F015B99623002269
:203EA000114600F0E2B80EB5C10F80EAE0700844CA07002140F233438DE80E000A460B46CA
:203EC00000F010F903B000BD0EB540F2334102910021CDE900110A460B4600F003F903B055
:203EE00000BD00F0004220F00040C10DC0F3160040F400007F2901DA00207047962903DCC0
:203F0000C1F19601C84001E096398840002AF4D04042704720F00040C10DC0F3160040F496
:203F200000007F2901DA00207047962903DCC1F19601C840704796398840704770B5C1F35A
:203F40000A5201F000450024C1F3130140F2FF3341F480119A4201DA002070BD40F233430D
:203F60009A42A2F2334203DC5242FFF788FD00E090402C43F1D0404270BDC1F30A5210B50A
:203F8000C1F3130140F2FF3341F480119A4201DA002010BD40F233439A42A2F2334203DC1F
:203FA0005242FFF76CFD10BD904010BD00F0004230F000400AD0C10D01F56071C0F31600DA
:203FC00042EA0151C20840071143704700200146704701F0004330B421F0004150EA010282
:203FE00006D00A0DA2F56072C1F31301002A02DC30BC00207047440F44EAC104C100E018D9
:2040000030BC00EBC25000F027B8202A04DB203A00FA02F1002070479140C2F1200320FAE0
:2040200003F3194390407047202A06DBCB17203A41FA02F043EAE07306E041FA02F3D0406D
:20404000C2F120029140084319467047A0F14101192900D8203070470029A8BF7047401CC2
:20406000490008BF20F00100704710B4B0FA80FC00FA0CF050EA010404BF10BC704749B109
:20408000CCF1200421FA04F411FA0CF118BF012121430843A3EB0C01CB1D4FEA00614FEA26
:2040A000102042BF002010BC704700EBC35010440029A4BF10BC7047401C490008BF20F04F
:2040C000010010BC704710B5141E73F1000408DA401C41F1000192185B411A4301D120F007
:2040E000010010BD2DE9F04D92469B4611B1B1FA81F202E0B0FA80F220329046FFF785FF66
:2041000004460F4640EA0A0041EA0B0153465A46084313D0114653EA010019D0C8F14002B5
:204120005046FFF7ACFC05460E46504659464246FFF76BFF084305D0012004E02046394685
:20414000BDE8F08D0020054346EAE0762C4337430A986305E40AA0EB08000022FD0A44EA84
:2041600047540A3002D500200146E9E7010510196941DDE9084500196941BDE8F04DA2E742
:204180002DE9F04D00231A461B1A8A4103DB00200146BDE8F08DC1F30A52C1F3130141F4D5
:2041A00080154FF0000BD10702D100186D41521E0027044640F2FF11384601EB620A3E4632
:2041C0008046024600204FF48011FFF758FCC2197141BB1846EB0100B4EB030C75EB000CE7
:2041E00004D3E41A65EB000517460E46241908F101006D4180463428E3DDF91946EB0600D4
:20420000091BA84103D24FF0FF32134601E0002213461BEB070046EB0A51BDE8F04DFFF726
:2042200052BF0000064C074D06E0E06840F0010394E8070098471034AC42F6D3FEF75AFFBA
:20424000AC7F0108CC7F010870B58C1810F8015B15F0070301D110F8013B2A1106D110F86A
:20426000012B03E010F8016B01F8016B5B1EF9D12B0705D40023521E0DD401F8013BFAE77E
:2042800010F8013BCB1A921C03E013F8015B01F8015B521EF9D5A142D8D3002070BD00008F
:2042A00010B572B606480079AA2801D00FF0BAF800200349087162B612F00AFA10BD000026
:2042C0000030024010B5024804F002FE10BD0000B01D002070B5044600252068806800F0BB
:2042E0000100F0B12068806820F001002168886006F0A8FA05460EE006F0A4FA401B022840
:2043000009D9A06A40F01000A062E06A40F00100E062012070BD2068806800F001000028DB
:20432000EAD10020F6E770B505466C6AA06A00F05000E0B9A06A40F40070A062206880687C
:2043400000F46020B0F5602F0DD1E06858B9A06A20F48070A062A06A00F4805018B9A06AC5
:2043600040F00100A062204604F0DEFB03E0206A016B2846884770BD70B505466C6AA06A44
:2043800040F04000A062E06A40F00400E062204604F09DFD70BD70B50446656A284604F02A
:2043A00095FD70BD38B504460025002000902068806800F0010080BB2068806840F00100F5
:2043C00021688860164800681649B0FBF1F0009002E00098401E009000980028F9D106F043
:2043E00031FA054613E006F02DFA401B02280ED9A06A40F01000A062E06A40F00100E062C2
:2044000000BF002084F8240000BF012038BD2068806800F001000028E5D00020F6E700000D
:204420000000002040420F0070B505460E4606F009FA22490968401A02283DD3002418E082
:204440001F4850F824001F4931F81410C0EB81201B4951F8241001EBE010194941F824000C
:20446000084650F82400C0F38F2025F81400601CC4B2092CE4DB002418E0134850F8240026
:20448000124931F81410C0EB81200F4951F8241001EBE0100C4941F82400084650F824000B
:2044A000C0F38F2026F81400601CC4B2032CE4DB06F0C8F90149086070BD0000700500205D
:2044C000241E00205C1D0020481E00201C05002010B5154803F0ECFF144803F0E9FF124889
:2044E00004F0ACFE114804F0A9FE104804F0F0F909220F490C4804F039FF0B48006A0068CD
:20450000006820F004000849096A09680860094807F0DBF90C21074807F04EFC0C2105482F
:2045200007F0F4F810BD0000801D0020B01D00205C1D00209C1C00200146002266488142D6
:204540000DD1664848604A68824201D000207047634848604A68824201D00020F7E76148C8
:2045600081420DD1604848604A68824201D00020EDE75E4848604A68824201D00020E6E78D
:2045800040F2555048614A69824201D00020DEE740F6AA2048614A69824201D00020D6E7A0
:2045A00040F2555088618A69824201D00020CEE740F6AA2088618A69824201D00020C6E7A0
:2045C00040F25550C861CA69824201D00020BEE740F6AA20C861CA69824201D00020B6E7A0
:2045E00040F2555008620A6A824201D00020AEE740F6AA2008620A6A824201D00020A6E79C
:2046000040F2555048624A6A824201D000209EE740F6AA2048624A6A824201D0002096E79B
:2046200040F2555088628A6A824201D000208EE740F6AA2088628A6A824201D0002086E79B
:204640002B48C862CA6A824201D000207FE72948C862CA6A824201D0002078E726480863B2
:204660000A6B824201D0002071E7244808630A6B824201D000206AE71F4848634A6B8242DB
:2046800001D0002063E71D4848634A6B824201D000205CE71A4888638A6B824201D000202B
:2046A00055E7184888638A6B824201D000204EE700204860C860086148618861C861086216
:2046C00040F6FF70486200208862C86208634863886301203BE700000024014055554500BF
:2046E000AAAA8A000028014055554000AAAA800055555500AAAAAA0055555515AAAAAA2A7C
:2047000055551500AAAA2A0088B001460022086800904868019088680290CB6803930B69BB
:2047200004934B690593552008600A68552A02D0002008B07047AA2008600A68AA2A01D01E
:204740000020F6E745F2555048604A68824201D00020EEE74AF6AA20486048684AF6AA232D
:2047600000EA03021846824201D00020E1E745F2555088608A68824201D00020D9E742F60C
:20478000AA2088608A68824201D00020D1E745F25553CB60CA681846824201D00020C8E70A
:2047A00042F6AA23CB60CA681846824201D00020BFE745F255530B610A691846824201D02D
:2047C0000020B6E742F6AA230B610A691846824201D00020ADE745F255534B614A691846F5
:2047E000824201D00020A4E742F6AA234B614A691846824201D000209BE7009808600198E7
:20480000486002988860039BCB60049B0B61059B4B6101208DE70246002004E0002322F830
:204820001030431C98B28842F8DB70472DE9F04704460E46924699466527844800780128A0
:204840007AD105F0FFFF40F6C411884202D20020BDE8F0877E480088401C7D490880608A53
:204860007C49096808447B49086079480088012801DC1920ECE776480088032801DC32208F
:20488000E6E773480088052801DC4B20E0E770480088072801DC6420DAE700206B490870EF
:2048A000B9F1180F0AD16B480068C0F3CF0000EB80004000072190FBF1F011E0B9F1300F96
:2048C0000AD164480068C0F3CF0000EB800040000D2190FBF1F003E05E480068C0F3CF00AF
:2048E00080B25D490880002523E0781EA84205DC4FF00008C4F804800020A9E7B01C30F8A4
:2049000015005549098888420EDC30886843642190FBF1F03188A1EB0008C4F80480781B2B
:20492000401EC0B294E707E04FF00008681C80B20546BD42D9DB86E0484880F800A00078C4
:2049400047490870607C00287AD143F698216069B0FBF1F081B2434802780078401C414B21
:20496000187004F11C0020F81210184600780C2827DBB9F1180F0BD10C2104F11C0003F07A
:20498000E1FC00EB80004000072190FBF1F013E0B9F1300F0BD10C2104F11C0003F0D2FC44
:2049A00000EB800040000D2190FBF1F004E00C2104F11C0003F0C6FC274908800020294951
:2049C0000870002524E0781EA84207DC4FF00008C4F804800020224908701BE0B01C30F85A
:2049E00015001D49098888420EDC30886843642190FBF1F03188A1EB0008C4F80480781B83
:204A0000401E1749087005E04FF00008681C85B2BD42D8DB00BF1248007810490978884292
:204A20000ADD0F4801780D4800781430814203DA0A4800780A4908700020606101206074A3
:204A40000748007804E700BF02E70000920300208E03002098030020940300209103002070
:204A6000900300209303002030B51E2A04DB0CDB64280ADA0A2908DA9C891C809C89DC8112
:204A80009C895C8000245C6030BD40F6EB244C43B4EB002F01D2040202E040F6EB244C4317
:204AA000950405EB85056D00B5FBF4F41C801C88B4F5FA7F02DA4FF4FA7407E01C88B4F5BB
:204AC000FA5F02DD4FF4FA5400E01C881C801D885C68C4EB85245D6805EB64145C605C687F
:204AE000C4F38F245C805C88DC8100BFCCE7000038B504460B48012300220A2100900A48E0
:204B000007F054FF0948012300220A210090084807F04CFF034800780449097808402070FE
:204B200038BD000046040020FC1B002047040020101C002000BFFEE710B5024804F076FD0E
:204B400010BD0000B422002000B58BB0002006900790012008904CF22000019000200290FB
:204B60004DF2E01003904FF6FF700490002005900120099001A9244804F0B8FC20B14FF4EA
:204B8000A77122A011F03AFB0120069000200790012008904FF460400190002002904CF27A
:204BA000E01003904FF6FF700490002005900120099001A9144804F099FC20B140F26311B5
:204BC00012A011F01BFB0220069000200790012008904FF240500190002002904FF6C0705B
:204BE00003904FF6FF70049001200590099001A9054804F07BFC20B14FF4BC7103A011F044
:204C0000FDFA0BB000BD0000B42200202E2E5C436F72655C5372635C63616E2E630000004B
:204C20002DE9F04104460D46002700260DB9666B00E0A66B206800F5D87000EB051000688E
:204C400000F00400B060B06858B9206800F5D87000EB0510006840F2FF7101EA505030603D
:204C60000AE0206800F5D87000EB051000686FF0604101EAD0007060206800F5D87000EBE2
:204C80000510006800F00200F060206800F5D87000EB0510406800F00F0030613562206839
:204CA00000F5D87000EB05104068C0F30720F061206800F5D87000EB05108068307520680A
:204CC00000F5D87000EB05108068010A7175206800F5D87000EB05108068010CB175206856
:204CE00000F5D87000EB05108068000EF075206800F5D87000EB0510C0683076206800F50C
:204D0000D87000EB0510C068010A7176206800F5D87000EB0510C068010CB176206800F593
:204D2000D87000EB0510C068000EF0764DB920202168C8602068406920F00A00216848611B
:204D400008E02020216808612068406920F050002168486194F83C70222F01D0322F05D1E5
:204D60002068406920F40F4021684861EDB994F83C00422804D0622806D072280CD107E003
:204D8000122084F83C000BE0322084F83C0007E0522084F83C0003E0012084F83C0000BFA8
:204DA00000BF204604F0CAFE1CE094F83C00522804D0622806D072280CD107E0122084F894
:204DC0003C000BE0222084F83C0007E0422084F83C0003E0012084F83C0000BF00BF204611
:204DE00004F074FE0020BDE8F08100002DE9F34F83B0044660790B287EDB0021204611F055
:204E000047FB00906449009808700121204611F03FFB8246604981F801A0009855286CD163
:204E2000BAF1AA0FFBD12088000A88702078C8700221204611F02CFB064657490E71112E6D
:204E400003D0162E01D00C2E7ED10321204611F01FFB8046504880F805800521204611F054
:204E600017FB83460421204611F012FB0BEB00201FFA80F94FEA19204749887181F807900B
:204E80000521204611F004FB0546A8EB0500022872D1617908F10900814217DA207C0128E1
:204EA00004D105F0CFFCE0600020207405F0CAFCE168411A0498814205D96179204611F08C
:204EC000A3FA0120207405B0BDE8F08F0120207400270EE0B81DC1B2204611F0D9FA2F49E3
:204EE000C8550846C15D07F108002B4A1154781C87B2AF42EEDB01E04CE047E0A81DC1B25C
:204F0000204611F0C5FA4FEA006BE81DC1B2204611F0BEFA0BEB004B05F10800C1B2204618
:204F200011F0B6FA0BEB002B05F10900C1B2204611F0AEFA0BEB0001019105F10801164838
:204F400000F038F9029000E01BE0DDE90110081A0CD12088114B4A46314600F09BFE08F160
:204F60000900C1B2204611F04FFAACE70121204611F04AFA0EE0FFE70121204611F044FA0A
:204F800008E00121204611F03FFA03E00121204611F03AFA00BF96E74B0D00204C0C00209B
:204FA00030B50A4600211CE00F4B5B6B14335B5CC57884686355C3785B1CDBB2C370847832
:204FC000A34201DB0023C37043795B1CDBB243718478A34203DD83784371012383714B1C57
:204FE000D9B29142E0DB30BDB42200202DE9F047824688461446002C5FDD2046E11704EBC3
:205000005171C910A4EBC1018FB237B90827E11704EB5171C1F3CF0907E02046E11704EBDB
:205020005171C910491C1FFA81F92548006BC0F800A000202249096BC8602149096B8860C0
:2050400000261CE008201E49096B086100250AE0082000FB065018F800101948006B14300A
:205060004155681C85B2082DF2DB0A21144804F0D5FD012801D10CF093FA701C86B2A9F1AE
:205080000100B042DEDC0E48006B076100250AE0082000FB065018F800100948006B143092
:2050A0004155681C85B2BD42F2DB0A21044804F0B5FD012801D10CF073FABDE8F087000036
:2050C000B422002010B504462068406920F001002168486194F83C00122805D1206840694E
:2050E00020F40F402168486194F83C00422804D0522806D072280CD107E0222084F83C006D
:205100000BE0322084F83C0007E0622084F83C0003E0012084F83C0000BF00BF204604F0E5
:20512000D5FE002010BD000010B5014600224C69CB69552008600A68552A01D0002010BD0C
:20514000A82008600A6802F0A802A82A01D00020F5E70A4848614A69824201D00020EEE73A
:20516000074848614A69824201D00020E7E74C61CB614FF4004008600120E0E755050100FA
:205180002A8A020030B503460C460021002200BF09E0985C80EA1120C0B2054D35F810005E
:2051A00080EA0121521CA242F3D388B230BD0000B0750108F0B502460B460025681E0021EC
:2051C0000FE0565C7040002407E0060E064F57F8265000026840661CB4B2042CF5DB4E1C49
:2051E000B1B29942EDDBF0BDB077010800B585B000BF1848806940F0040016498861084610
:20520000806900F00400009000BF00BF00BF0846806940F0080088610846806900F008005D
:20522000009000BF00BF08200190002002900120039001A9084805F065F94FF400400190E0
:20524000002002900120039001A9044805F05AF905B000BD00100240000C01400008014050
:205260002DE9F84F04460D4616461F4600F0FAF8009000F0F7F8804600F0F4F88146009821
:20528000404504D1C84502D16A4880F800906A48007830B9674800786649487001206649A9
:2052A00008706448007863494978884238D0614840786049097801F00301604A515C884272
:2052C00009D1002060705E4908805E4908806068401C606024E0574840785649097801F056
:2052E0000301594A515C88420DD155480088401C5349088008460088042811DB012060702E
:20530000002008800CE04F480088401C4D490880084600880A2803DD0120607000200880DF
:205320004FF0020A4348007800F001004149497801F0010188422DD005F084FA43490968B9
:20534000401A4FF47A71B1FBF0F04149088005F079FA3E49086017B94FF0010A00E0B246DE
:20536000607858B93B480078401C3A49087008460078504504DB0120A07001E00020A07076
:2053800035490888012111F0F5FB208105F05AFA32490860324800682D490988C0EB8120EA
:2053A0002F49096801EB20202D49086008460068C0F3872020704FF0640B2548008814287B
:2053C00002DA4FF496700DE021480088282801DD642007E01E48008800EB80004FF4FA712A
:2053E000A1EB40001FFA80FB0BFB05F0642190FBF1F085B205F026FA18490968401AA842FF
:2054000011D90020A070022060700020207010490880134908600F4908700F490888002152
:2054200011F0A8FB20810348007802494870BDE8F88F0000D0030020D2030020807F010845
:20544000D4030020D6030020847F0108D8030020E0030020E20300202A050020E4030020F7
:20546000DC03002070B54FF40041084805F0D8F905462C460821064805F0D2F9064644EA00
:205480004600C4B204F0030070BD000000080140000C014000BF084A1268526A91B201EB20
:2054A000810292004FF47A7392FBF3F202800022014B1B685A627047DC1C002010B54FF42F
:2054C000FA710948FFF792FC4FF4FA710748FFF78DFC4FF4FA710648FFF788FC4FF4FA71EC
:2054E0000448FFF783FC10BD98050020AC050020C0050020D4050020F0B58DB007460E462F
:20550000154618A103C9CDE90B0118A103C9CDE9070109AB002231460BA811F023F805ABDA
:205520000022314607A811F01DF8002405E009A8005D01A90855601CC4B2082CF7DB0024D3
:2055400007E005A8015D01AA04F108001154601CC4B2082CF5DB294601A801F058FC0DB03C
:20556000F0BD000039FF6C063454333029270957FFFFFFFF30B502460B460021002400BFBB
:205580000EE0481C84B207E0505C155DA84201D1002030BD601C84B29C42F5DB481C81B2BE
:2055A0009942EEDB0120F4E731B581B0BDF80400ADF80000BDF9040044F6E61500FB05F1F6
:2055C000C913BDF9060000FB05F2D2130C4613466042C01AC01A00B2ADF8020000983CBD71
:2055E00070B504460AB9084670BD081B800290FBF2F086B2934202DD0D462846F4E706FB63
:2056000003F004EBA02085B22846EDE710B510223A493B480DF042F8044624B91022374962
:205620003848FEF73CFA10223449354814300DF035F804462CB91022304932481030FEF79C
:205640002EFA20222D492E4828300DF027F8044624B9202229492C48FEF721FA102227497F
:2056600027484C300DF01AF8044624B9102223492648FEF714FA10222049214860300DF069
:205680000DF8044624B910221C492148FEF707FA10221A491A4874300DF000F8044624B931
:2056A000102216491B48FEF7FAF908221349144888300CF0F3FF04462CB917480F490A682E
:2056C000026049684160CC220C490D4894300CF0E5FF044624B9CC2208491048FEF7DFF94F
:2056E000202206490E480CF0D9FF044624B9202202490C48FEF7D3F910BD0000FC15002028
:2057000008FC01081C090020400B0020600B0020700B0020800B0020B8040020B409002042
:205720006CFD01089801002010B50446594B0C220421204602F04EFE401C28B9554B0C2289
:205740000421204602F046FE534B20221221204602F040FE401C28B94F4B2022122120462D
:2057600002F038FE4C4800784C4908704C4B04223421204602F02EFE401C28B9484B04225C
:205780003421204602F026FE464B10223A21204602F020FE401C28B9424B10223A212046E7
:2057A00002F018FE404B30224C21204602F012FE401C28B93C4B30224C21204602F00AFE4C
:2057C00039480068401C384908600B4630224C2120460EF0E4FA401C28B9334B30224C21CF
:2057E00020460EF0DCFA314B1022EC21204602F0F1FD401C28B92D4B1022EC21204602F022
:20580000E9FD2B4B18227E21204602F0E3FD401C28B9274B18227E21204602F0DBFD254BF3
:2058200008229821204602F0D5FD401C28B9214B08229821204602F0CDFD1F4B1022A2214E
:20584000204602F0C7FD401C28B91B4B1022A221204602F0BFFD194B1022D621204602F09B
:20586000B9FD401C28B9154B1022D621204602F0B1FD134B2022B421204602F0ABFD401CD5
:2058800028B90F4B2022B421204602F0A3FD002010BD0000C40B0020B00A0020C101002026
:2058A000C2010020F00A0020000B0020300B00206E150020C70100203C0C00202C0C00201A
:2058C000D00A00201CB52A492A4801F04BFD10222949284808300EF0FFF9102226491031BB
:2058E00024481C300EF0F8F920222449214830300EF0F2F9102222491E4854300EF0ECF936
:20590000102220491B4868300EF0E6F910221E4918487C300EF0E0F908221C4915489030EC
:205920000EF0DAF9CC221A4912489C300EF0D4F92022184918480EF0CFF9184800780006AD
:205940001649497800EB01401449897800EB01201249C9780844009004211048FFF72AFC80
:20596000019002226946034801F0CEFE1CBD0000FFFF010800FC01081C090020400B002026
:20598000600B0020700B0020800B0020B8040020B4090020980100206CFD0108887F010842
:2059A00038B50546002410F0DBFB10F0B3FB284601F084FB284601F03DFB1F480088009013
:2059C0009DF800200021284601F042FC401C28B99DF800200021284601F03AFC9DF80120F6
:2059E0000121284601F034FC401C28B99DF801200121284601F02CFC02216846FFF7C2FBD6
:205A0000044622120221284601F022FC401C20B922120221284601F01BFCE2B20321284640
:205A200001F016FC401C20B9E2B20321284601F00FFC002038BD00008C7F010810B5094ACB
:205A40000949A2F10C00FFF757FD064B0C22042106480EF0A4F90648006820F40010044957
:205A6000086010BDC40B0020C7010020340400209401002070B50546002639480078C8B9FD
:205A8000002404E03748C0880644601C84B20A2CF8DB0A20B6FBF0F03349088004F0D2FEAF
:205AA0003249086004F0CEFE3149086001202C4908704FE004F0C6FE2D490968401AB0F586
:205AC000FA7F03D904F0BEFE284908602868C0F3804000283ED104F0B5FE24490968401ACF
:205AE000B0F5FA6F36D9002404E01E48C0880644601C84B20A2CF8DB0A20B6FBF0F01A49B0
:205B0000088008460088B0F57A7F05DB0846008840F6B831884219DD286820F4802000F5BB
:205B2000802028600720134948800F4800888880084601F0EBFC00200F4908700F484089D5
:205B4000401C0E49488102200D49087004F07AFE0649086004F076FE0549086070BD00006B
:205B6000400000205C1D002040050020440000204800002090070020A5030020300B002021
:205B8000C601002010B5024804F022FA10BD0000E01D00203FB504460025206800906068D2
:205BA0000190A0680290E06803900020206045F2555020602568854202D0002004B030BDFC
:205BC0000020206042F6AA2020602568854201D00020F3E70020206045F255506060052023
:205BE0000DF010FD656845F25550854201D00020E4E74AF6AA20606005200DF003FD6568B6
:205C00004AF6AA20854201D00020D7E74FF05530A060A568B5F1553F01D00020CEE74FF014
:205C2000AA30A060A568B5F1AA3F01D00020C5E74FF05530E060E568B5F1553F01D00020D5
:205C4000BCE74FF0AA30E060E568B5F1AA3F01D00020B3E7019860600298A0600398E06013
:205C6000009820600120A9E730B590F840500124AC40C56B6C60046863604468102C04D165
:205C80000468A2600468E16003E00468A1600468E26030BD2DE9F84F0746884615461C46C9
:205CA00005F0FF0A40F23171781A8F4273D00CDCA7F25160002801F05D80CF280ED0D02877
:205CC0000DD0DF2841F06F8064E00F287ED010287DD01F287CD02028F4D1C0E300BF41F23D
:205CE0000C61681A8D4236D00BDCA5F58050A0F1100070B1B0F53E7F23D0B0F5806F45D1CE
:205D000023E0B0F5807F2CD0A0F5C850F93878BB2FE052462146F948FDF7C1FEF748407AD4
:205D2000F749C8730020F749887604F08BFDF549C8610020F449087004F084FDF24948607A
:205D400025E001200CF08EF921E052462146EF48FDF7A5FE1BE052462146ED48FDF79FFE0C
:205D600015E052462146EA480C30FDF798FE0EE00CE052462146E7A0FDF7C8FE28B9E7480D
:205D8000007820F00100E549087000E000BF00BF63E300E000BFB5F5545F76D025DC43F2B8
:205DA0000511A5EB01008D4270D014DCA5F58050A0F10800B0B3B0F5017F38D0B0F5417F45
:205DC0003BD0A0F5F850FA38002802E049E249E244E37DD138E0A0F20310002879D0F82886
:205DE00078D0B0F5007FF4D1D1E0B5F5824F72D00DDCA5F55850A0F1050000286CD0A0F24D
:205E0000FB20002869D0B0F5E16FE2D167E1A5F584400838002873D0F82872D0B0F5067F81
:205E2000D7D1F3E1FFE701200CF01CF917E252462146BB48FDF733FE11E252462146B848BC
:205E40000C30FDF72CFE0AE2B648007801280DD052462146B448FDF722FEB3480078C043FB
:205E6000B2490870B0484078C0434870B048007868B9AD480078052824D104F0E3FCAD495B
:205E800008600120AA4908701CE0C3E03AE0A848007801280BD1A4480078052812D004F081
:205EA000D1FCA44908600020A14908700AE0A0480078022806D19C480078052802D1332044
:205EC00099490870984800788D494873964805E0C4E124E031E057E1A5E0D8E040788873DA
:205EE0000B464FF481520C214FF4E2600DF0F6FF00209149087004F0A5FC8F494860AEE181
:205F000049E15CE15246214682A0FDF7FFFD28B98248007820F00200804908709FE152467B
:205F200021468648FDF7BBFD85A345F203320C2140F213700DF0D2FF91E1824B2022122188
:205F4000814802F047FA7F48007B20707D48407860707C480079A0707A48C07EE0707B4BC3
:205F60002022B421784802F035FA012020710F2060717648007CA0710020E071234645F21B
:205F800008420C2140F213700DF0A8FF67E1207840B26C49C876084690F91B000A2801DD6A
:205FA0000A20C876674890F91B0010F10A0F02DAF6206449C8766078624948700B46202261
:205FC000122161480DF0EBFE207940B25F490874084690F91000002802DD0020087408E0DE
:205FE0005A4890F9100010F1140F02DAEC2057490874564B2022B42153480DF0D0FE01F02F
:20600000A5FE4FA345F203320C2140F213700DF065FF24E14E4B41F210520C214FF4E26057
:206020000DF05CFF1BE1524621464AA0FDF76EFD60BB002046498860C8600922474948A047
:20604000FDF764FD80B142480068B0F57A7F03D200203F4908604860092241A13F48FDF715
:2060600042FD002041490870394B1022D62136480DF095FE32A345F203320C2140F21370E1
:206080000DF02CFF00201E4908834883E7E03848007818BB1022374937480CF0FFFA102211
:2060A00034491031344814300CF0F8FA0C213348FFF780F806462F48C66203464FF4925203
:2060C0000C214FF4E2600DF009FF2D4B4FF4B9520C214FF4E2600DF001FF00BFBFE052469E
:2060E00021462848FDF7DBFC15A345F203320C2140F213700DF0F2FEB1E000007C090020D5
:20610000DC0800201C030020F4010020A40900208C0900205245414459000000B801002057
:20612000800A0020D8000020DA000020DC0000200601002008010020E4010020B901002098
:2061400041434B00B00A002034040020D00A00202C0C0020434C454152000000600B0020FA
:20616000434C4541525F4F444F0000002D0400200A0200201C09002008FC0108B80B0020C5
:206180005C090020B0040020F54AF649F648007802F022F863E052462146F248FDF77FFC7B
:2061A0000020F249087001F0D1FDAFF26C0345F203320C2140F213700DF090FE4FE0EC4BFE
:2061C00020221221EB4802F005F9E9480E30016821604168616000892081E74B2022B421F1
:2061E000E44802F0F7F8E44812300168C4F80A104168C4F80E1000896082234645F22062D5
:206200000C2140F213700DF069FE28E0D8480E30216801606168416021890181D6481230F2
:20622000D4F80A100160D4F80E104160618A0181CF4B20221221CF480DF0B1FDCE4B202273
:20624000B421CC480DF0ABFDAFF20C1345F203320C2140F213700DF041FE00E000BF00BF08
:2062600096E500BFB5F5445F5ED010DCA5F58050A0F58670C8B1B0F5807F1CD0B0F57F7FDC
:2062800020D0A0F5F050F43800287DD122E0A5F548500838F0B3FD2877D0B0F5FC7F75D0AF
:2062A000A0F2FD200028F0D19DE052462146B348FDF7F5FBD0E052462146B0480C30FDF714
:2062C000EEFBC9E00020AE49087004F0BBFAAC494860C1E0AB48007828BB1022AA49AB4850
:2062E0000CF0DCF91022A8491031A84814300CF0D5F90C21A648FEF75DFF0646A248C662A1
:2063000003464FF492520C214FF4E2600DF0E6FDA04B00E023E04FF4B9520C214FF4E260AD
:206320000DF0DCFD00BF97E0914B20221221914802F050F88E48007B20708D4840786070AF
:206340008B480079A0708A48C07EE070234647F208320C2140F214700DF0C0FD7CE0207814
:2063600040B28349C876084690F91B000A2801DD0A20C8767E4890F91B0010F10A0F02DA57
:20638000F6207B49C87602E065E015E022E06078774948700B462022122176480DF0FFFCFB
:2063A00001F0D4FCAFF2682347F203420C2140F214700DF093FD4FE052462146AFF2AC2067
:2063C000FDF7A4FB28B97448007820F004007249087041E0714B41F210520C214FF4E260AA
:2063E0000DF07CFD38E052462146AFF29820FDF78DFB78BB002069498860C860092268494A
:20640000AFF2A420FDF782FB88B164480068B0F57A7F03D200206149086048600922AFF240
:20642000C0215F48FDF75FFB0020504908705B4B1022D6214F480DF0B2FCAFF2FC2347F24B
:2064400003420C2140F214700DF048FD002055490883488300BF00BF00BFFDE300BF42F2AE
:206460002041681A8D4273D04CDCB5F5D05F70D027DCB5F5A85F6DD015DCB5F5905F6AD031
:2064800008DCB5F5805F67D0A5F588500838002863D1C8E0B5F5985F60D0A5F5A0501038FF
:2064A0000028F5D114E1A5F5B0501038F0B3F02855D0B0F5007F77D0A0F2F1200028E7D149
:2064C0005AE1B5F5F85F70D00DDCB5F5D95F6DD0B5F5E05F6BD0A5F5E8501038002867D09B
:2064E000F028D5D1B6E1B5F5005F75D0B5F5045F73D0A5F50850103800286FD0B0F5807F64
:20650000C6D1F6E1B0F51D6F69D052DCB0F59C6F73D00EDCE52871D0A0F2E51000286ED05D
:20652000A0F2031000286BD0FA2800E0F1E0AFD1A5E2A0F2E150002872D0A0F20110002881
:206540006FD0FF286ED0A0F206200028A0D101E3E2E12DE1CEE07DE053E0F5E3A6E0EAE02B
:2065600090040020B8040020C10400202D040020B00A002034040020D00A0020980A002067
:20658000EC0100200A0200201C09002008FC0108B80B00205C090020B80100202C0C0020D7
:2065A000600B0020DC080020D4E064E10FE12DE13BE141F2E942811A904273D010DCB0F59A
:2065C0001E6F70D0B0F52E6F6ED0B0F53E6F6CD0B0F5506F85D158E35CE16DE175E1EBE23D
:2065E000A1F2C311002970D044296FD0B1F59A7F6DD0B1F5157F9AD1A7E365E29EE1B8E195
:20660000E2E1FE4B08229821FD4801F0E3FEFB4B4AF208420C2140F215700DF05FFCA7E3E2
:206620005BE273E292E252462146F448FDF737FAF24B08229821F2480DF0B1FBAFF20053FD
:206640004AF603120C214FF4E2600DF047FCFFF7F5F98DE3EB48007818BB1022EA49EB4889
:206660000CF01CF81022E8491031E84814300CF015F80C21E648FEF79DFD0646E248C66261
:2066800003464FF492520C214FF4E2600DF026FCE04B4FF4B9520C214FF4E2600DF01EFC77
:2066A00000BF65E306E3CEE2D7E2DFE21022DA49D6484C300BF0F2FFD74B4AF210620C21E8
:2066C00040F215700DF00AFC52E308E319E32DE352462146D048FDF7E2F90020CF4908703E
:2066E000AFF2A4534AF603120C214FF4E2600DF0F5FB3DE31022CA49C44860300BF0CEFF45
:20670000C74B4AF210720C2140F215700DF0E6FB2EE352462146C248FDF7C1F90020BF49F7
:206720000870AFF2E4534AF603120C214FF4E2600DF0D4FB1CE31022BA49B44874300BF067
:20674000ADFFB84B4AF610020C2140F215700DF0C5FB0DE352462146B248FDF7A0F9002001
:20676000AE490870AFF228634AF603120C214FF4E2600DF0B3FBFBE22078AB49087008469D
:206780000078C043A9490870A748007878B1A848006820F48060A64908600846006820F417
:2067A000805008600846006820F400600860DFE2A04B20221221924801F00CFE9D4B4AF2F5
:2067C00020020C2140F215700DF088FBD0E2524621469848FDF763F99648007896490870A5
:2067E000944B2022122186480DF0D9FA9149487B0EF0A8FF01F0AAFAAFF2BC634AF60312BB
:206800000C2140F215700DF069FBB1E28B4B10223A217B4801F0DEFD884B4AF210120C2150
:2068200040F215700DF05AFBA2E2524621468348FDF735F9814B10223A2171480DF0AFFA27
:20684000AFF204734AF603120C2140F215700DF045FB8DE27A4B4AF230220C2140F2157004
:206860000DF03CFB774B4AF610420C2140F215700DF034FB7CE220227349644828300BF025
:206880000DFF714B4AF220520C2140F215700DF025FB6DE2234618227E21594801F09AFDC7
:2068A0006A48C08AE082694B4AF218320C2140F215700DF013FB5BE2654B41F201420C21C1
:2068C0004FF4E2600DF00AFB52E2524621464E48FDF7E5F8002051490870AFF29C734AF675
:2068E00003120C214FF4E2600DF0F8FAFFF7A6F83EE25246214644481030FDF7D0F8002087
:2069000046490870AFF2C8734AF603120C214FF4E2600DF0E3FA2BE2524621464A48FDF721
:20692000BEF800203D490870AFF2EC734AF603120C214FF4E2600DF0D1FA19E252462146BA
:2069400044A0FDF7E3F898B9AFF60C034AF603120C2140F215700DF0C1FA00200BF082FBF6
:20696000642003F089FC01200FF020FD04F08CF8FEE152462146AFF62400FDF7C7F810BB41
:20698000FF23042200211E4800F026FBFF2350224C211B4800F020FB30491C48083800F09B
:2069A000E1FC2F492F4800F0DDFCAFF66C034AF603120C2140F215700DF090FA01200FF04E
:2069C000F5FC04F061F8D3E15246214626A0FDF79DF888B90FF0C4FB094800F06FFBFEF7D8
:2069E00071FFAFF6A4034AF603120C2140F215700DF074FA01203DE040E00000C7010020F1
:206A0000340400200A0200201C09002008FC0108B80B00205C090020600B00202D0400205C
:206A2000700B0020800B0020D8000020D900002094010020B00A0020C1010020F00A002094
:206A4000000B0020300B0020400B00206E150020B80100205245534554000000FFFF01083F
:206A6000FFF3010800F001085245434F56455259000000000FF09AFC04F006F878E152463B
:206A80002146CB48FDF70BF8C9480078C043C9490870C7484078C04348700020C649087046
:206AA00003F0D0FEC4494860C1480078C3494873BF48407888730B464FF481520C214FF487
:206AC000E2600DF00BFA53E1BD4B4AF604220C2140F215700DF002FA4AE152462146B848C9
:206AE000801CFCF7DCFFB64B04223421B5480DF056F9AFF6B4134AF603120C214FF4E260F4
:206B00000DF0ECF95520AE49C87031E1AC48C078552803D0AA48C078AA2816D1AA20A849C3
:206B2000C87052462146A648FCF7B9FFA44B04223421A4480DF033F9AFF6FC134AF60312FD
:206B40000C214FF4E2600DF0C9F911E120789E4908700DE100BF20790006617900EB014089
:206B6000A17900EB0120E179084421780906627801EB0241A27801EB0221E2781144401A66
:206B8000461C20780006627800EB0240A27800EB0220E2788118324604F10800FCF77FFFEE
:206BA0004AF60830304482B223460C2140F215700DF094F900BFDBE000BF2078000661782E
:206BC00000EB0140A17800EB0120E178461820790006617900EB0140A17900EB0120E17988
:206BE00000EB010BABEB060000F10109B6F1005F0FD94A4604F108013046FCF750FFAFF62E
:206C0000C0234AF603120C2140F215700DF066F917E06E48864214D906F2FF31304600F00C
:206C2000A1FB09F0FF0204F1080130460DF054F8AFF6F4234AF603120C2140F215700DF00F
:206C40004DF900BF00BF624B41F210520C214FF4E2600DF043F98BE0A6E05E4B41F208620C
:206C60000C214FF4E2600DF039F981E05A4B2022B421544801F0AEFB574B4AF620520C215F
:206C800040F215700DF02AF972E0524621465248FCF705FF504B2022B4214A480DF07FF883
:206CA000AFF664334AF603120C2140F215700DF015F95DE05246214648A0FCF727FF68B9F6
:206CC0000FF028FA3F4800F0B5F9AFF68C334AF603120C2140F215700DF000F948E052461B
:206CE00021464148FCF7DBFE002040490870AFF6B0334AF603120C2140F215700DF0EEF813
:206D000036E0524621463248FCF7C9FE304B1022D6212C480DF043F8AFF6DC334AF60312D1
:206D20000C2140F215700DF0D9F821E02022304930480BF0B3FC2E4B4BF620320C2140F258
:206D400015700DF0CBF813E011E0524621462848FCF7A5FE002025490870AFF61C434AF6BB
:206D600003120C214FF4E2600DF0B8F800E000BF00BF19E0A5F51450053820B1A0F5F8406F
:206D8000063828B900E000BF02201B49087000E000BF00BF2B46424640F251611748009409
:206DA0000DF0E8F800E000BF00BFBDE8F88F0000DA000020DC000020E4010020DC0800206D
:206DC000C201002034040020DB010020003000082C0C0020FC010020D00A00204C4F4720D3
:206DE000434C454152000000B40900202D040020980100206CFD01085D000020F805002039
:206E0000704700BF0100A0F10100FBD1704710B50246002016E0135C041D145D63400B54C0
:206E2000031DD35C00F10804145D6340041D0B55231DD35C0834145D634000F108040B5555
:206E4000431CD8B20428E6DB10BD000010B503F0F9FC14490968401AB0F5FA7F21D303F0B5
:206E6000F1FC104908601048007858B90FA343F20902112140F212700DF030F801200A4912
:206E800008700EE00848007801280AD107A345F20902112140F213700DF020F8002002496D
:206EA000087010BDD0000020D400002048414E445348414B450000001FB54FF460400090DB
:206EC00011200190022003906946194803F01AFB4FF4E060009011200190022003906946EA
:206EE000144803F00FFB00224FF48071114803F0A3FC00224FF400710E4803F09DFC00221E
:206F00004FF480610B4803F097FC00224FF40051074803F091FC00224FF48041044803F08A
:206F20008BFC00224FF40041014803F085FC1FBD000C01400008014010B500210D4804F0C6
:206F40005BFF04210B4804F057FF0821094804F053FF0021074804F0EFFB0421054804F0A1
:206F6000EBFB0821034804F0E7FB0C21014804F023FF10BD9C1C0020F8B504460020009009
:206F80006A460021204600F00DF90DF101020121204600F007F902216846FEF7F3F806464E
:206FA0006A460221204600F0FDF80DF101020321204600F0F7F89DF801009DF8001000EB23
:206FC000012085B2A81B03D12046FEF7ADFBF8BD2046FEF7E5FCFAE72DE9F04780460C4688
:206FE00016461F46301B00F0FF09002507E06019C1B23A46404600F02BF9681CC5B24D45EE
:20700000F5DBBDE8F08700001FB50446022000900120019003906946054803F073FA0122F0
:207020000221034803F008FC204605F0F1FA1FBD000C014010B504461C4B30224C212046E1
:207040000CF0ADFE401C28B9184B30224C2120460CF0A5FE164B1022EC2120460CF09FFE86
:20706000401C28B9124B1022EC2120460CF097FE104B1022D62120460CF091FE401C28B98E
:207080000C4B1022D62120460CF089FE0A4B1022A22120460CF083FE401C28B9064B10229A
:2070A000A22120460CF07BFE10BD0000000B0020300B00202C0C00203C0C002010B5044610
:2070C000314B0C22042120460CF069FE401C28B92D4B0C22042120460CF061FE2B4B0822AF
:2070E000982120460CF05BFE401C28B9274B0822982120460CF053FE254B2022122120468C
:207100000CF04DFE401C28B9214B2022122120460CF045FE1F4B2022B42120460CF03FFE45
:20712000401C28B91B4B2022B42120460CF037FE194B10223A2120460CF031FE401C28B93F
:20714000154B10223A2120460CF029FE134B0422342120460CF023FE401C28B90F4B0422A0
:20716000342120460CF01BFE0D4B18227E2120460CF015FE401C28B9094B18227E212046C9
:207180000CF00DFE10BD0000C40B0020C7010020B00A0020D00A0020F00A0020C201002073
:2071A0006E1500202DE9F04106460F4615460024304605F0A0FAA021304605F0E1FA00BFFA
:2071C00000BF601C84B240F6B830844203DD4FF0FF30BDE8F081304605F0FAF90028F0D1AF
:2071E0003946304605F0CCFA002400BF601C84B240F6B830844202DD4FF0FF30E9E73046D3
:2072000005F0E6F90028F1D1304605F074FAA121304605F0B5FA002400BF601C84B240F630
:20722000B830844202DD4FF0FF30D2E7304605F0CFF90028F1D12946304605F006FA30462D
:2072400005F036FA304605F076FA0020C1E700002DE9F04106460F461546002400220221BA
:20726000294803F0E9FA304605F045FAA021304605F086FA00BF00BF601C84B240F6B83023
:20728000844203DD4FF0FF30BDE8F081304605F09FF90028F0D13946304605F071FA00245F
:2072A00000BF601C84B240F6B830844202DD4FF0FF30E9E7304605F08BF90028F1D1294614
:2072C000304605F05DFA002400BF601C84B240F6B830844202DD4FF0FF30D5E7304605F0FF
:2072E00077F90028F1D1304605F025FA0A2002F0C3FF01220221044803F09EFA034803F071
:20730000CFFA0020C0E70000000C014004080020F8B50E480468001D0568200E8DF80000B8
:20732000200C8DF80100200A8DF80200E0B28DF8030004216846FDF73DFF0646701B02D123
:20734000FEF764F901E0FEF7BDFAF8BD00FC010810B50446207818B9FEF7B4FA01202070C8
:2073600010BD000038B504460D4600200C49086008468460281B401C800AC86003F04AF821
:2073800000BF34200749C86000BF6946044802F087FF02F0DDFF642002F06EFF38BD00008A
:2073A000EC1500200020024010B504220E490F480BF074F90446A4B904220B490CA0FCF789
:2073C000A5FB70B928220849084808300BF066F9044634B9282204490748FCF760FB0020DC
:2073E00010BD0120FCE70000FC15002000E80108464C414700000000900B002010B54FF4BD
:20740000805003F071F810BD10B5042003F06CF810BD00001FB54FF460400090022001906C
:2074200003906946064803F06DF84FF4E06000900220019003906946024803F063F81FBDE8
:20744000000C01400008014010B50021104804F0B3FC04210E4804F0AFFC08210C4804F02A
:20746000ABFC0C210A4804F0A7FC0021084804F04DF90421064804F049F90821044804F092
:2074800045F90C21024804F041F90AF077FE10BD9C1C00202DE9F04107460C46207860BB5C
:2074A000384600F057F846B2701C48B11448402101FB06054022394628460CF043FC1AE04A
:2074C0000F49491E0F48FFF74DFFF0220C4940310C4800F019F90C490948FFF743FFF02236
:2074E0000849074800F010F9074D3F3D4022394628460CF027FC01202070BDE8F0810000EE
:2075000000F0010800EC0108FFF3010810B504460B480068A0600B484068E06020220A49E8
:2075200004F11000FCF7BBFA0848016821634068606307480168A1634068E06310BD000082
:2075400094010020000B0020DC080020FC010020DE00002010B50246002116E00F4C04EBBE
:20756000811003884FF6FF7083420CD111B90120108006E04020C0EB8110084C035B581C76
:207580001080084610BD481C41B21029E6DB04480388581C10804FF0FF30F3E700F00108D3
:2075A000C0F301080021074AD1610749096941F00401054A11611146096941F04001116105
:2075C0007047000028070020002002400021074AD1610749096941F00201054A1161114691
:2075E0004861096941F040011161704728070020002002400022054BDA61054A126942F07B
:207600000102034B1A61018070470000280700200020024000201E49C96801F0100139B111
:207620001C49C96941F002011A4AD16140F010001749C96801F0040139B11649C96941F076
:207640000101144AD16140F004001149C96901F0010169B10F49C96941F004010D4AD16182
:2076600000BF0B49C96921F00101094AD16100BF00BF40F20111884206D10549C96921F039
:207680000101034AD16101E00149C86000BF7047002002402807002070B5044603F0D2F8C3
:2076A000054609E0601C38B124B103F0CBF8401BA04201D9032070BD1248C06800F00100CC
:2076C0000028EFD10F48C06800F0200020B100BF20200C49C86000BF0A48C06800F01000AD
:2076E00048B90848C06900F0010020B90548C06800F0040018B1FFF78DFF0120DBE700208F
:20770000D9E70000002002402DE9F04104460E461746002502F07EFE00BF0FE056F825C091
:20772000624600232146022002F01CFE08B9241D03E002F00DFEBDE8F0816D1CBD4202D295
:2077400003488442EAD902F003FE00BFF3E70000FBFF0108022005490870002004490880E9
:2077600048800449088048807047000030000020280000202C00002001200149087070476F
:20778000300000202DE9FF4705460E4617464FF0000A0CF0F3F903900398FDF705FF029058
:2077A00039B202980AF0F8FA0090714800990160B0F900006F490968C1EB80206D490968D0
:2077C00001EBA0206B49086008460068801200B2694908806648B0F9020068490968C1EB86
:2077E00080206649096801EBA0206449086008460068801200B2624908806248007C00288D
:2078000049D161480078042845D16048408840F6EC01884210DA5E4805605E48006810F18A
:20782000040F05DA5B480068001D5A49086042E00020584908603EE05448408840F6BE1151
:20784000884221DA51484088A0F6EC0000EB800040F21A41081A50490860084600688542E8
:2078600001DA284601E04C4800684949086049480068801E474908600846006810F5D27F4D
:2078800019DA4648086016E00020414908604348404908600FE03E4805603E48006810F1B2
:2078A000040F05DA3B480068001D3A49086002E00020384908603A4A2F48B0F900103448C8
:2078C000008800B20AF028FA044636480068C0EB44203449096801EBE000324908603248FC
:2078E0004088B7214843C0F3CF1947F698107043B9F57A7F02DA4FF47A7100E0494690FB7F
:20790000F1FA284800680AEB602447F69810844200DD00E02046044620B224490880244ADE
:207920001748B0F900101B48008800B20AF0F4F9804620480068C0EB48201E49096801EB3E
:20794000E0001C49086008460068401200B21749488008460AF0D8FE1448006800900AF02C
:20796000F9FE019001980BF05DFEBDE8FF870000280000200C000020200000201000002081
:2079800022000020D0070020DE0000205C1D00200400002008000020240000205CFEFFFF2F
:2079A0004C06002018000020F00A00202C000020700600201C00002004F030FF09F038FE93
:2079C00009F0D8FE62B60020124981F83C0009F0E7FD72B609F0AEFE0AF0D8FBFFF76CFABD
:2079E00000200D4908600846006820F4005000F5005008600DE0084B41F204120C214FF4E9
:207A0000E2600CF06BFAC8200BF0ECFD034802F047FFF0E7B42200209401002004080020C6
:207A200070B505460E46049CAC4208DAFF2E01D100210DE0281B7043C0F5806108E09442BB
:207A400002DA4FF4806103E0A01A5843C0F58061002901DC002000E00846014688B270BD56
:207A600087B0014600220868009048680190C86803903D4881423AD04FF0553008600A6872
:207A8000B2F1553F02D0002007B070474FF0AA3008600A68B2F1AA3F01D00020F4E74FF0C5
:207AA000553048604A68B2F1553F01D00020EBE74FF0AA3048604A68B2F1AA3F01D00020FD
:207AC000E2E745F25550C860CA6890B245F25553984201D00020D7E74AF6AA20C860CA6899
:207AE00090B24AF6AA23984235D00020CCE700986FF30B0000F2555008600A68C2F30B004F
:207B000040F25553984201D00020BDE700986FF30B0000F6AA2008600A68C2F30B0040F687
:207B2000AA23984201D00020AEE7039820F00700C01DC860CA6802F00700072801D0002016
:207B4000A2E7039820F00700C860CA6802F0070008B1002098E70098086001984860039863
:207B6000C860012090E70000001401402DE9F04104460E46154629480078012812D128484B
:207B800001780078401C264A1070264820F8116010460078322810DB002020490870114646
:207BA00008700AE032221F49304609F06FFF643087B22088B84200DD00BF2888C0F3C0306C
:207BC00050BB208840F2DC51884203DC02F03AFE1549086002F036FE13490968401A42F279
:207BE0001071884218D9286820F4004000F50040286001200D494880208888800846FFF775
:207C000085FC00200A4908700A488088401C09498880022008490870BDE8F0817F04002044
:207C200080040020381C00208404002090070020A5030020300B0020C6010020B1F5967F08
:207C400003DA0122044B1A7002E00022024B1A7001F16402028070477E04002010B5024630
:207C60000020B2F5FA7F01DC01200EE0B2F5E16F01DB084609E040F2145393FBF1F4A2F52B
:207C8000FA7393FBF4F35B1CD8B210BD10B50446207800284DD12749087002F0D3FD25492F
:207CA0004860608840F2AA71884236D120792249087060794870A0798870E079C870617A8C
:207CC000207A01EB00201C4988801C48807EEE2811D10846808820B94FF6FF70184988600B
:207CE00009E0154880884EF6602191FBF0F0144988600020C870A07A0F498871E07AC8716A
:207D000008468079C0F3401018B100200D4908700DE001200B49087009E0608840F2AB7169
:207D2000884204D1084861680160A16841600120207010BDA8040020E4070020B00A002051
:207D4000F4030020C10400208C04002010B500BF2A480078052803DA05202849087006E00B
:207D600026480078182802DD18202449087023480078401E43F2C82191FBF0F084B21821A7
:207D80001F48FCF748FD00200BE000FB04F10A2291FBF2F101F5FA71194A22F81010411C53
:207DA000C8B216490978491E8142EEDC4FF4E16112480078401E124A22F8101000BF00BFAC
:207DC0001048807900EB4000C0000A2190FBF1F00D4908700B48C07948700A48007B09499F
:207DE000C97E084464380849487104484078887002488078C87000BF10BD0000B80400206C
:207E0000C2040020B00A00209404002010B502F019FD40F6B831884206D9C1480078F028BC
:207E200002D1C049C87710BDBF48FFF72FFFBF48007858B902F006FDBC494968401A40F664
:207E4000B831884202D90120B8490870B4480078202823D040285CD080285BD0F02875D186
:207E6000AF480078AF49C87700BF02F0EBFCB0490968401AC82809D90120AE490870084650
:207E800000F086F902F0DEFCA949086000BFA748007810B92020A24908703DE1A04800783D
:207EA00000F0E0009F49C87700BFA3480078052800DB16E002F0C6FCA0490968401AC82853
:207EC0000ED99F4A9F49A048007800F085F902F0B9FC9A49086098480078401C964908701F
:207EE00000BF00BF9948007890B198480078032803D140208A4908700AE0944800780428FE
:207F000003D092480078082802D180208449087002E100BF8D480078082805D18549087019
:207F200000204880888054E088480078032829D140207B49087003207E490870834840782F
:207F4000012804DA82480088488017E0E3E07F4840787C490978884208DD7A480078401E3A
:207F60007B4931F810007349488007E077484078401E774931F810006E49488000206D4976
:207F8000888026E071480078042822D18020644908700420674908706C4840786949497893
:207FA000884204DA67484078624988800EE06748407864498978884204DD624880785D4909
:207FC000888003E0614840785A49888000205949488056480078012803D1F0205149C87724
:207FE00025E04F480078402812D1564A1178594A5278642302FB03F0FFF730FE00F01F00E2
:208000004749097801F0E00108444649C8770EE04348007880280AD14148007800F0E0001E
:208020004C49497801F01F0108443E49C87700BF02F008FC48490968401AB0F57A7F39D906
:208040004248007808280FD144480078052807DA384800F09DF841480078401C3F4908709A
:2080600000203F49087021E03D480078012808DA3C4800F07DF83A480078401C384908709F
:2080800011E03748007805280DDA2A4800F080F833480078401C32490870084600780528D5
:2080A00001DB0020087000202C49087002F0CAFB2949086000BF00BF022402F0C3FB2A49E7
:2080C0000968401AB0F57A7F23D91F480078012809D100BF1A4A1B49204600F07DF80020E7
:2080E0002249087011E01848007870B900241F480078052809DA124A1249204600F06CF827
:208100001A480078401C1949087002F09BFB1649086000BF00E000BF00BF00BF83E60000BB
:20812000C0040020DC0800209C040020A8040020F4040020EE070020FC040020F804002062
:2081400090040020B8040020C1040020B0040020C2040020E4070020000500200505002096
:208160000405002094040020080500200C0500201CB5044600200090019020680090606884
:2081800001900822694640F2AC70FCF72FFF1CBD1CB5044600200090019020788DF80000B4
:2081A000608800128DF80100A0788DF80200A08800128DF8030020798DF8040000208DF817
:2081C00005008DF806008DF807000822694640F2AD70FCF70BFF1CBD7FB506460C46154658
:2081E000002000900190029003908DF800602088ADF80100A0788DF8030028788DF804001D
:208200006B4645F210520C2140F213700BF066FE7FBD000038B5044601234FF47A720A21E2
:208220000248009404F0C2FB38BD0000241C002030B503460024002204E033F812502C4405
:20824000551CAAB28A42F8DBB4FBF1F5A8B230BD70B505462C480078012811D100202A49DC
:20826000087002F0EFFAB0F5E16F05D902F0EAFAC8302649088003E04FF4FA60234908809F
:2082800002F0E0FA2149098888423BD920480078012837D11F48007858B11F480088C82861
:2082A00007DC40F2C27085420CDD40F63E00854208DA00201949C8720A2219A11B48FBF7B3
:2082C00012FC1CE001201549C872002415E0184830F81400A8420EDB0A2216A11348FBF723
:2082E00002FC1748015D1148203880F8271000200749087070BD601CC4B2092CE7DB002045
:208300000349087000BFF5E78A040020880400200A020020DC010020D8010020D00700208B
:208320005144303037482E20343800003C0900208E7F010854544B5A303139413438000000
:20834000A07F010810B502460B460020002107E032F81140844201DD32F811004C1CA1B25A
:208360009942F5DB10BD10B502460B464FF6FF70002107E032F81140844201DA32F8110014
:208380004C1CA1B29942F5DB10BD00000246002108E0064830F81100904201DC084670471E
:2083A000481CC1B2C829F4DB0020F8E7048001080246002108E0064830F81100904201DC13
:2083C00008467047481CC1B2BF29F4DB0020F8E7948101082DE9F84F82460D4614461F46B6
:2083E00000260EE01C488219A819C1B25046FEF7D9FE401C18B94FF0FF30BDE8F88F701C81
:20840000C6B2A642EEDB21461348FCF7BBFE81462819C1B26A465046FEF7C4FE2819401CB0
:20842000C1B20DF101025046FEF7BCFE9DF801009DF8001000EB01201FFA80F8B8EB0900FF
:2084400006D1224604493846FBF729FB0020D4E74FF0FF30D1E70000FC1A00202DE9FC5F54
:20846000804689464FF0000A002549464046FFF7DFFE8346002407E038F81400ABEB00055E
:2084800005FB05AA601C84B24C45F5DB5046FBF70AFD06460F46304639460EF045FBCDE901
:2084A0000001FBF74BFD05462846BDE8FC9F0000F8B5044600260020009000BF94F824004C
:2084C000012801D10220F8BD012084F8240000BF2046FBF7FFFE0646002E62D1A06A20F42A
:2084E000885040F00200A062022002F0EFFA30490968B1FBF0F04000009002E00098401E55
:20850000009000980028F9D12046FBF74BFF2068806840F008002168886002F093F90546BD
:2085200011E002F08FF9401B0A280CD9A06A20F0020040F01000A06200BF002084F8240081
:2085400000BF0120BFE72068806800F008000028E7D12068806840F004002168886002F046
:2085600071F9054611E002F06DF9401B0A280CD9A06A20F0020040F01000A06200BF00204E
:2085800084F8240000BF01209DE72068806800F004000028E7D1A06A20F0020040F0010046
:2085A000A06200BF002084F8240000BF30468AE70000002038B50246002300200090906874
:2085C00000B100BF00BF92F82400012801D1022038BD012082F8240000BF906890B948683D
:2085E000012809D11068806B6FF315000C6840EAC4301468A06338E0906A40F02000906239
:20860000012332E00C694868A0421ED84C680869001BC0F1030000EB80041F20A04040F471
:2086200040141068806BA0434D680C69641BC4F1030404EB84050C68AC400D8A6D1E44EA13
:20864000055420431468A0630FE04C680869001BC0F1030000EB80041F20A04040F44014E6
:208660001068806BA0431468A0631068806800F0010040B91068806847F20104A043CC6935
:2086800020431468A060886901280FD1C869B0F5E04F06D11068406840F4806014686060B5
:2086A00004E0906A40F0200090620123486901280DD1886930B91068406840F48050146844
:2086C000606004E0906A40F020009062012308680A2812D31068C0680C780A3C04EB44056D
:2086E0000724AC40A0430D780A3D05EB45058C68AC4020431468E0600FE0106800690C7827
:2087000004EB44050724AC40A0430D7805EB45058C68AC402043146820610868102802D0AE
:208720000868112805D11068806840F400001468A0604868012806D002280DD0032814D0E5
:2087400004281BD11BE0106840696FF30B00CC682043146860611BE0106880696FF30B00DB
:20876000CC6820431468A06112E01068C0696FF30B00CC6820431468E06109E000BF106871
:20878000006A6FF30B00CC6820431468206200BF00BF0868102802D00868112827D1174C71
:2087A0001068A0421ED11068806800F40000F0B91068806840F400001468A06008681028BB
:2087C00015D10F4800680F4CB0FBF4F000EB80004000009002E00098401E009000980028A7
:2087E000F9D104E0906A40F020009062012300BF002082F8240000BF1846E9E6002401409D
:208800000000002040420F0010B504460121204600F044F84FF6FF7101EA00101A49488009
:208820000221204600F03AF84FF6FF7101EA0010154988800321204600F030F84FF6FF7120
:2088400001EA001010490880104800880988401A00B20F4908800D4840880B494988401A43
:2088600000B20B4948800948808807498988401A00B2074988800749054809F0D5FA012086
:208880000549087010BD00001C0500202E050020340500203A050020280500200246002044
:2088A00001290FD0022909D0032904D0042908D11368986C09E01368586C06E01368186C19
:2088C00003E000BF1368D86B00BF00BF7047000070B50446002500BF94F82400012801D105
:2088E000022070BD012084F8240000BF2046FBF759FD0546002D5BD1A06A42F2010188434C
:2089000040F48050A0622E492068884208D12D48006800F4702008B9012002E0002000E08A
:20892000012020B1A06A20F48010A06203E0A06A40F48010A062A06A00F4807008B9002013
:20894000E06200BF002084F8240000BF401F216808602068406840F08000216848602068AE
:20896000406800F4806010BB2068806800F4E040B0F5E04F15D112492068884208D1114893
:20898000006800F4702008B9012002E0002000E0012030B12068806840F4021021688860FE
:2089A0000BE02068806840F400402168886004E000BF002084F8240000BF284691E700006F
:2089C000002801400424014038B5024600230020009000BF92F82400012801D1022038BD3E
:2089E000012082F8240000BF4868072812D21068406B0C79641E04EB84051F24AC40A04382
:208A00000D796D1E05EB85050C68AC4020431468606327E048680D2812D21068006B0C7991
:208A2000E41F04EB84051F24AC40A0430D79ED1F05EB85050C68AC4020431468206311E0EA
:208A40001068C06A0C790D3C04EB84051F24AC40A0430D790D3D05EB85050C68AC4020430F
:208A60001468E06208680A2812D31068C0680C780A3C04EB44050724AC40A0430D780A3D49
:208A800005EB45058C68AC4020431468E0600FE0106800690C7804EB44050724AC40A04317
:208AA0000D7805EB45058C68AC402043146820610868102802D00868112827D1174C1068C1
:208AC000A0421ED11068806800F40000F0B91068806840F400001468A0600868102815D12A
:208AE0000F4800680F4CB0FBF4F000EB80004000009002E00098401E009000980028F9D1A0
:208B000004E0906A40F020009062012300BF002082F8240000BF184661E7000000240140CA
:208B20000000002040420F0070B50646CD480068401CCC49086008460068B0F5967F01D973
:208B400000200860C8480078012805D14120C74948758875C87599E0C548C07A012808D1DC
:208B6000C4480078012804D10020C249087008F0DDFBC1480088C14909680844BF49086038
:208B8000BD488088BE4909680844BD490860BA48C089BC4909680844BA490860BA48008894
:208BA000401CB94908800846008840F6B83188426CDBAF48C07A012822D1B0480068B0FB71
:208BC000F1F085B22846FFF7F3FBA8494875AC48006840F6B831B0FBF1F085B22846FFF7DB
:208BE000E7FBA2498875A748006840F6B831B0FBF1F085B22846FFF7DBFB9C49C8753CE0FA
:208C00009E48006840F6B831B0FBF1F085B22846FFF7BCFB954948759948006840F6B83106
:208C2000B0FBF1F085B22846FFF7B0FB8F4988759648007801280ED10846407D94490870CF
:208C40009048006840F6B831B0FBF1F09149088000208E4908708B48006840F6B831B0FB53
:208C6000F1F08C490988081A00EB400080018849097801EBA0207D49C8750020824908806B
:208C80007E4908607E4908607E4908607A48408881490968C1EB80207F49096801EB602091
:208CA0007D49086008460068801244F2CE714843C0F38F206D49C8800846C0880989C911DC
:208CC00001EBC10202EB011108446849C8807348007803280BD10846C088A0F5F850A43818
:208CE00040F27A514843C0F38F206049C8806C48407C01281FD101F0A5FDB0F5FA6F1AD382
:208D00005A48C0880A2190FBF1F06549488208464069498A08446249486108468069401C5D
:208D200088610846806943F69821884203D300205B49886148744E48C07A012815D14E48A3
:208D4000C08858490988401A49F6192148438412002C01DC002006E049F61920844201DB7C
:208D6000401E00E02046044613E04348C0884D490988401A4CF250314843C412002C01DC95
:208D8000002005E04CF25030844200DB00E02046044645480068C0EB84204349096801EBB2
:208DA00060204149086008460068C0F38F202F4908813E48C078AA2811D02F4800893C4932
:208DC000C98A401A642148433849897890FBF1F4002C01DC002000E02046044607E0344AC6
:208DE000D18A254A1089314A0CF018F8044631490C8031480078D8B91F4880892F4909883E
:208E0000441A002C01DC002000E0204604462C480068C0EB84202A49096801EB202028498F
:208E2000086008460068C0F38F202249488002E00020204948801048408922490968C1EBA3
:208E400080202049096801EB60201E49086008460068C0F38F201C4908800749488809F03F
:208E6000C3F870BD440500200A020020DC080020D00700206C0500205C1D002058050020D3
:208E8000540500205C0500205005002060050020610500206205002048050020040200203E
:208EA0003C030020400500204C050020C20100206E1500202A0500207E0400207C04002066
:208EC0006405002068050020080200207047704710B504462068406800F0200020282FD14D
:208EE0002068006800F00200022829D1A06A00F0100018B9A06A40F40070A0622068806871
:208F000000F46020B0F5602F13D1E06888B92068406820F0200021684860A06A20F480709D
:208F2000A062A06A00F4805018B9A06A40F00100A0622046FFF7F8FD6FF0120021680860A0
:208F40002068406800F0800080283BD12068006800F00400042835D1A06A00F0100018B9CC
:208F6000A06A40F40050A0622068806800F4E040B0F5E04F0DD02068406800F48060D0B99F
:208F80002068806800F46020B0F5602F13D1E06888B92068406820F0800021684860A06A51
:208FA00020F48050A062A06A00F4807018B9A06A40F00100A0622046FFF726FC6FF00C00E6
:208FC000216808602068406800F0400040280FD12068006800F0010050B1A06A40F4803028
:208FE000A062204600F0A8F86FF001002168086010BD00002DE9F041044600270025002658
:20900000A84614B90120BDE8F081A06810B1606900B100BFA06A30B90020E06284F8240067
:20902000204600F08BF82046FBF754F90746A06A00F01000002873D1002F71D1A06A20F460
:20904000885040F00200A062E16960680843E16840EA41000643A068B0F5807F02D0A06824
:20906000012802D14FF4807000E0002005436069012811D1E06838B9A069401E4FF4006161
:2090800041EA4030054307E0A06A40F02000A062E06A40F00100E0622068406820F4694000
:2090A0002843216848602068806821490840304321688860A068B0F5807F02D0A06801285F
:2090C00002D14FF4807000E00020B0F5807F03D1208A401E4FEA00582068C06A20F4700043
:2090E00040EA08002168C8622068806811490840B04208D10020E062A06A20F0020040F000
:209100000100A06211E0A06A20F0020040F01000A062E06A40F00100E062012705E0FFE74D
:20912000A06A40F01000A062012738466BE70000FDF7E1FFFE0E1FFF7047000010B586B03B
:2091400004463249206888423CD100BF3048806940F400702E4988610846806900F400702C
:20916000019000BF00BF1F2002900320039002A9284801F0C7F9A02002900320039002A9DA
:20918000254801F0BFF9254825490860002048600021234881608021C1604900016189004B
:2091A0004161202181610021C16100F0DFFF20B140F217111BA00DF021F800BF184820623C
:2091C000446221E01C49206888421DD100BF1048806940F480600E4988610846806900F4C4
:2091E0008060019000BF00BF0E2002900320039002A9094801F086F901221146122001F001
:20920000F0FB122001F0E0FB06B010BD002401400010024000100140000801400800024047
:20922000E01D00202E2E5C436F72655C5372635C6164632E630000000028014070B504465F
:20924000002500BF94F82400012801D1022070BD012084F8240000BF2046FBF7A3F8054672
:20926000002D77D1A06A40F20121884340F48070A0623C492068884208D13B48006800F49B
:20928000702008B9012002E0002000E0012078B1A06A20F48010A0622068406800F480607C
:2092A00000B3A06A20F4005040F48050A06219E0A06A40F48010A0622B49091F20688842D0
:2092C00003D028492068884204D12748006800F4806000E0002028B1A06A20F4005040F4FD
:2092E0008050A062A06A00F4805020B1E06A20F00600E06201E00020E06200BF002084F8BD
:20930000240000BFC01E216808602068806800F46020B0F5602F16D112492068884208D116
:209320001148006800F4702008B9012002E0002000E0012038B12068806840F4A00021684D
:2093400088600CE006E02068806840F480102168886004E000BF002084F8240000BF28461E
:2093600075E7000000280140042401402DE9F04104460D461646002757492068884203D093
:2093800056492068884205D15348001D006800F4702000E0002000287ED100BF94F824007C
:2093A000012802D10220BDE8F081012084F8240000BF2046FAF7F6FF0746002F6DD1A06AE9
:2093C00040F60161884340F48070A06243492068884209D14048001D006800F4702008B9FA
:2093E000012002E0002000E0012078B1A06A20F48010A0622068406800F4806000B3A06AAF
:2094000020F4005040F48050A06219E0A06A40F48010A06230492068884203D02F4920687B
:20942000884205D12C48001D006800F4806000E0002028B1A06A20F4005040F48050A06272
:20944000A06A00F4805020B1E06A20F00600E06201E00020E06200BF002084F8240000BF4A
:209460001F48216A88621F48216AC8621E48216A08636FF00200216808602068806840F4A2
:20948000807021688860226802F14C0133462A46206A00F0A3FE01E01AE014E0206880685E
:2094A00000F46020B0F5602F06D12068806840F4A000216888600CE02068806840F4801058
:2094C0002168886005E000BF002084F8240000E00127384667E70000002401400028014015
:2094E00027430008974300087943000830B5024600230C7D012000FA04F31068D0F8000227
:2095000020F47C5001254C6A45EA042420431468C4F800021068D0F81C0298431468C4F82A
:209520001C02C869E8B91068D0F80C0298431468C4F80C02888880B28C8940EA044410688B
:2095400000F510704D6940F83540088880B20C8940EA0444106800F510704D6900EBC50017
:209560004460C86901281DD11068D0F80C0218431468C4F80C02888880B20C8840EA0444C8
:20958000106800F510704D6940F83540888980B20C8940EA0444106800F510704D6900EBA3
:2095A000C5004460886938B91068D0F8040298431468C4F8040206E01068D0F8040218437A
:2095C0001468C4F80402086938B91068D0F8140298431468C4F8140206E01068D0F8140230
:2095E00018431468C4F81402086A012806D11068D0F81C0218431468C4F81C021068D0F801
:20960000000220F001001468C4F80002002030BD0168496941F0020102685161016849696A
:2096200041F0100102685161704700002DE9F0410446002500260027A8462068C068C0F3C1
:20964000001520684069C0F3C0062DB126B148F4007810202168C86020680069C0F3001548
:2096600020684069C0F380162DB126B148F480681020216808612068406900F0010000282B
:209680003BD0206880687A490840884201D1012000E00020054620688068764908408842FB
:2096A00001D1012000E0002006462068806872490840884201D1012000E0002007460DB928
:2096C00006B9D7B120688068C0F3400520688068C0F340262068806800F001070DB906B965
:2096E0001FB12046FBF7EEFC01E048F400682068806862490843216888602068C06800F05C
:20970000030520684069C0F3400625B11EB100212046FBF785FA2068006900F00305206809
:209720004069C0F3001625B11EB101212046FBF777FA206C40EA080020642068806900F084
:20974000010520684069C0F3002620684069C0F3C0372DB126B11FB1206C40F00100206458
:2097600020688069C0F3400520684069C0F3402620684069C0F3C0372DB126B11FB1206C4A
:2097800040F00200206420688069C0F3800520684069C0F3802620684069C0F3C0372DB127
:2097A00026B11FB1206C40F0040020642068806900F0700008B9012000E000200546206838
:2097C0004069C0F3C02620684069C0F3C03795BB8EB387B32068806900F07005402D1BD073
:2097E00006DC102D09D0202D0CD0302D24D10EE0502D16D0602D1FD118E0206C40F008006C
:2098000020641AE0206C40F01000206415E0206C40F02000206410E0206C40F040002064B5
:209820000BE0206C40F08000206406E0206C40F48070206401E007E000BF00BF20688069AC
:2098400020F0700021688861206C78B1042021684860012084F83C002068406948F65B71F8
:209860008843216848612046FFF7D2FEBDE8F081010000040001000800000110090501007B
:209880002DE9F041044600270026002514B90120BDE8F08194F83C0028B9002084F83D003F
:2098A000204600F0A5F8022084F83C002068006820F00200216808602068006840F00100C7
:2098C0002168086000F0BEFF06460EE000F0BAFF801B0A2809D9032084F83C0000BF00209E
:2098E00084F83D0000BF0320D2E72068406800F001000028EAD02068406800F001000028C8
:2099000067D0A069012802D145F0800501E025F08005E069012802D145F0400501E025F021
:209920004005206A012802D145F0200501E025F02005606A012802D145F0100501E025F0E1
:209940001005A06A012802D145F0080501E025F00805E06A012802D145F0040501E025F02D
:2099600004052068006820F0FC00284321680860D4E90201084321690843616908436168C8
:20998000491E08432168C8612068006820F001002168086000F056FF06460EE000F052FFB1
:2099A000801B0A2809D9032084F83C0000BF002084F83D0000BF03206AE72068406800F032
:2099C00001000028EAD12068406800F0010000B90127012F06D100202064012084F83C001D
:2099E000002055E7042084F83C00012050E7000010B586B004462D492068884254D100BFE6
:209A00002B48C06940F000702949C8610846C06900F00070019000BF00BF8815029000203A
:209A20000390049002A9234800F06CFD4FF400700290022003900320059002A91D4800F0DE
:209A400061FD00BF1C49486820F4C04040F0E06040F48040486000BF01221146142000F057
:209A6000C0FF142000F0B0FF01221146152000F0B8FF152000F0A8FF10482063104860633C
:209A80001048A063FBF760F80F480068406940F002000D49096848610B480068406940F083
:209AA000100009490968486106B010BD0064004000100240000C014000000140541E002091
:209AC000701E0020941E0020B4220020816B896811B9416B096941B916490968496941F09E
:209AE0001001144A126851617047816B0968A1F2AA7111B1012911D100E000BF816B09693E
:209B000008290AD100210C4A1170816B09885180816B4B6953608969916000E000BF00BF5F
:209B200004490968496941F01001024A1268516100BFD9E7B42200209C04002010B50446B7
:209B4000606B806810B9606B006940B92E480068406940F002002C490968486110BD606B7C
:209B6000006840F23172811A904214D009DCA0F2516080B3CF2818D0D02817D0DF2837D12F
:209B800008E00F291CD010291BD01F2924D020292ED122E000BF606B00881C490880606B45
:209BA000017C1A48FBF7FCF923E000BF606B008817490880606B017C1548FBF7F1F918E069
:209BC00000BF606B008813490880606B017C1148FBF7E6F90DE001E000BF00BF606B00887E
:209BE0000D490880606B017C0B48FBF7D9F900E000BF00BF04480068406940F002000249F0
:209C00000968486100BFA9E7B422002098050020AC050020C0050020D40500202DE9F04132
:209C200004460E46042500272068806800F08060B0F1806F0DD02068806800F00060B0F128
:209C4000006F06D02068806800F08050B0F1805F7ED100BF94F83D00012802D10220BDE875
:209C6000F081012084F83D0000BF94F83C00222804D0322806D062280CD107E0422084F898
:209C80003C000BE0522084F83C0007E0722084F83C0003E0122084F83C0000BF00BF20686F
:209CA000806800F0806008B1002507E02068806800F0006008B1012500E00225206800F504
:209CC000C07000EB0510006800F00101206800F5C07000EB05100160206B806898B92068A0
:209CE00000F5C07000EB05100068216BC968226B128841EA42510843216801F5C07101EB4E
:209D00000511086015E0206800F5C07000EB05100068216B8968226B526841EAC201226B7C
:209D2000D26811430143206800F5C07000EB05100160206B007C00F00F00216B08612068C0
:209D400000F5C07000EB0510406820F00F0100E0B1E0206800F5C07000EB051041602068CF
:209D600000F5C07000EB05104068216B09690843216801F5C07101EB05114860206BC07DAB
:209D80000106206B807D41EA0041206B407D41EA0020216B097D0843216801F5C07101EB3C
:209DA00005118860206BC07E0106206B807E41EA0041206B407E41EA0021206B007E0143FE
:209DC000206800F5C07000EB0510C160206800F5C07000EB0510006840F00101206800F5F1
:209DE000C07000EB0510016000F02CFD074620E0701CF0B126B100F025FDC01BB04218D998
:209E0000032084F83C001DB980202168886009E0012D03D1E8032168886003E04FF4000013
:209E20002168886000BF002084F83D0000BF032015E74DB92068806821490840884201D177
:209E4000012016E0002014E0012D09D1206880681C490840884201D101200AE0002008E003
:209E60002068806818490840884201D1012000E000200028BCD094F83C00422804D05228D8
:209E800006D072280CD107E0222084F83C000BE0322084F83C0007E0622084F83C0003E09B
:209EA000012084F83C0000BF00BF00BF002084F83D0000BFD3E6042084F83C000120CEE68A
:209EC000010000040001000800000110704710B504460CB9012010BD607920B90020207187
:209EE000204600F005F8012060710020F3E7000008B5094A016891420DD100BF0749496938
:209F000041F04001054A51611146496901F04001009100BF00BF08BD0030024000100240FB
:209F200070B50446002594F82100022803D00420A063012548E02068006820F00E002168D7
:209F400008602068006820F00100216808601F492068884201D1012026E01C4914312068C2
:209F6000884201D110201FE0184928312068884201D1801518E015493C312068884201D1BC
:209F8000801411E0114950312068884202D14FF4803009E00D4964312068884202D14FF40D
:209FA000801001E04FF08070084908394860012084F8210000BF002084F8200000BF606B04
:209FC00010B12046616B8847284670BD0800024070B50446E06B05682068066894F84010E1
:209FE000042088402840002846D006F00400002842D02068006800F0200028B920680068CA
:20A0000020F004002168086057492068884201D1042027E0544914312068884201D14020E6
:20A0200020E0514928312068884201D1001519E04D493C312068884202D14FF4804011E0DF
:20A04000494950312068884202D14FF4802009E0454964312068884202D14FF4800001E010
:20A060004FF08060404908394860E06A00287AD02046E16A884776E094F8401002208840F7
:20A080002840A0B306F0020088B32068006800F0200040B92068006820F00A0021680860DE
:20A0A000012084F8210030492068884201D1022028E02D4914312068884201D1202021E0FB
:20A0C000294928312068884201D140151AE026493C312068884202D14FF4005012E0224951
:20A0E00050312068884203D14FF400300AE017E01D4964312068884202D14FF4001001E011
:20A100004FF0007018490839486000BF002084F8200000BFA06A30B32046A16A884722E0DD
:20A1200094F84010082088402840E0B106F00800C8B12068006820F00E002168086094F858
:20A14000401001208840E16B48600120A06384F8210000BF002084F8200000BF206B10B18B
:20A160002046216B884770BD080002400146002209B901207047184B0868C01A1423B0FB15
:20A18000F3F08000086414480838C863022081F821000868026843F6F0708243D1E9010377
:20A1A0001843CB6818430B6918434B6918438B691843CB69184302430868026000208862D9
:20A1C000C862086348638863012081F82100002081F8200000BFCDE7080002402DE9F041DC
:20A1E00004460D4616461F464FF0000800BF94F82000012802D10220BDE8F081012084F87E
:20A20000200000BF94F8210001282CD1022084F821000020A0632068006820F00100216820
:20A2200008603B46324629462046FBF71DFDE06A30B12068006840F00E00216808600BE0A7
:20A240002068006820F00400216808602068006840F00A00216808602068006840F00100CD
:20A260002168086006E000BF002084F8200000BF4FF002084046BFE770B5044600F0E2FA1D
:20A2800006462546681C10B104480078054400BF00F0D8FA801BA842FAD370BD580000203D
:20A2A0002DE9F04104460E460127002500BF2648007E012802D10220BDE8F0810120224901
:20A2C000087600BF2068022813D14CF25030FDF7E3F990BB0120FDF765F94CF25030FDF7AD
:20A2E000DBF907461948006920F004001749086123E04CF25030FDF7CFF9F0B94FF0FF3002
:20A300003060A56812E02846FDF760F94CF25030FDF7C2F907460D48006920F002000B4915
:20A3200008610FB1356007E005F58065D4E9021001EB8020A842E6D800BF00BF00200249AD
:20A34000087600BF3846B7E728070020002002400348006940F08000014908610020704705
:20A36000002002402DE9FE4F05468B4617469846012600240020029000BF2448007E0128F2
:20A3800002D10220BDE8FE8F01202049087600BF4CF25030FDF780F9064686BB012D02D116
:20A3A0000120029006E0022D02D10220029001E00420029000241EE02201B946C2464846DD
:20A3C0005146F9F75CFB80B20190022000FB04B000900199FDF70EF94CF25030FDF75CF9DF
:20A3E00006460B48006920F001000949086106B104E0601CC4B202988442DDDB00BF00BF66
:20A4000000200249087600BF3046BBE7280700200020024000200849096901F0800151B174
:20A420000649054A5160064951601146096901F0800101B1012070470020024023016745D6
:20A44000AB89EFCD10B50446042C3BD100202149C8700846807840B900F0F4F91D494860D5
:20A46000601F88600120887011E000F0EBF919494968401A17498860084680684B2802D265
:20A4800015480068886000F0DDF91249486011488068114908600F4880684B2818D30F484F
:20A4A0000068401C0D4908600D48007E08B9012001E00B48007E09490968B1FBF0F0054916
:20A4C000C86005E0B4F5805F02D101200549087010BD0000F40300209405002090050020DB
:20A4E000B00A0020E002002010B5044604480068204020B1024804602046FFF7A3FF10BD13
:20A50000140401402DE9F84703460024002000258446002700226EE14FF0010808FA02F439
:20A52000D1F8008008EA0400A0427DD1DFF8D0A2D1F80480A8EB0A09D0453AD014DCB8F1B8
:20A54000030F50D009DCB8F1000F31D0B8F1010F1CD0B8F1020F49D120E0B8F1110F18D001
:20A56000B8F1120F42D11EE0B9F5881F25D006DCB9F5803F20D0B9F5801F37D11AE0B9F57A
:20A58000001F18D0B9F5041F30D117E0D1F80CC02DE0D1F80C8008F1040C28E0D1F80C808E
:20A5A00008F1080C23E0D1F80C8008F10C0C1EE000BF00BF00BF00BF00BF00BFD1F808805C
:20A5C000B8F1000F02D14FF0040C0BE0D1F80880B8F1010F03D14FF0080C1C6102E04FF0E7
:20A5E000080C5C6103E04FF0000C00E000BF00BFFF2801D8984601E003F104084646FF288C
:20A6000002D84FEA820803E0A2F108084FEA88084746D6F800804FF00F0909FA07F928EA07
:20A6200009080CFA07F900E088E048EA0908C6F80080D1F8048008F08058B8F1805F7DD147
:20A6400000BFDFF8C081D8F8188048F00108DFF8B491C9F81880C846D8F8188008F001088E
:20A66000CDF8008000BF00BF4FEAB9384FEA920958F829504FEA82784FEA18794FF00F08FD
:20A6800008FA09F825EA0805DFF87C81434502D14FF0000816E0DFF87481434502D14FF0C9
:20A6A00001080FE0DFF86881434502D14FF0020808E0DFF86081434502D14FF0030801E018
:20A6C0004FF004084FEA82794FEA197908FA09F848EA0505DFF840814FEA920948F82950CC
:20A6E000D1F8048008F48038B8F5803F0AD1DFF82C81D8F8008048EA0008DFF82091C9F8BB
:20A70000008009E0DFF81481D8F8008028EA0008DFF80891C9F80080D1F8048008F40038C8
:20A72000B8F5003F10D1DFF8F48008F10408D8F8008048EA0008DFF8E49000E05AE009F113
:20A740000409C9F800800DE0DFF8D08008F10408D8F8008028EA0008DFF8C09009F10409FA
:20A76000C9F80080D1F8048008F48018B8F5801F0ED1DFF8A88008F10808D8F8008048EA02
:20A780000008DFF8989009F10809C9F800800DE0DFF8888008F10808D8F8008028EA000827
:20A7A000DFF8789009F10809C9F80080D1F8048008F40018B8F5001F0ED1DFF8608008F1B2
:20A7C0000C08D8F8008048EA0008DFF8509009F10C09C9F800800DE0DFF8408008F10C0843
:20A7E000D8F8008028EA0008DFF8309009F10C09C9F80080521C102AFFF48EAEBDE8F8870D
:20A80000000011100010024000080140000C014000100140001401400800014000040140FB
:20A82000024693680B400BB1012000E000207047C2684A40C26070470AB1016101E00B045C
:20A840000361704701480068704700005000002070B504460CB9012070BD4CF6CC402168AC
:20A86000086045F2555021680860D4E9001048602168A0688860FFF7E5FF054606E0FFF7B4
:20A88000E1FF401B302801D90320E5E72068C0680028F4D14AF6AA20216808600020DBE7E2
:20A8A00001464AF6AA200A6810600020704700000348006803490978084401490860704759
:20A8C000500000205800002010B50848006840F0100006490860032000F0C2F8002000F03F
:20A8E00007F800F02BF8002010BD00000020024070B504460E4800784FF47A71B1FBF0F000
:20A900000C490968B1FBF0F5284600F06FFE08B1012070BD102C07D200222146501E00F012
:20A9200060F80548046001E00120F2E70020F0E758000020000000205400002008B500BFB4
:20A940001F48806940F001001D4988610846806900F00100009000BF00BF032000F080F866
:20A96000002211466FF00B0000F03BF8002211466FF00A0000F035F8002211466FF00900F1
:20A9800000F02FF800221146501F00F02AF800221146101F00F025F800221146901E00F0DA
:20A9A00020F800221146501E00F01BF800BF0549486820F0E06040F00070486000BF08BDBC
:20A9C000001002400000014000BF00F01F02012191404209920002F1E022C2F8001100BFC5
:20A9E00070472DE9F05F80460D461646002707F069F8074639462A46334601F00700C0F1E9
:20AA0000070ABAF1040F02D94FF0040A01E0C0F1070AD14600F1040ABAF1070F02D24FF0B2
:20AA2000000A01E0A0F1030AD4464FF0010A0AFA09FAAAF1010A0AEA020A0AFA0CFA4FF033
:20AA4000010B0BFA0CFBABF1010B0BEA030B4AEA0B042146404607F03DF8BDE8F09F0000A3
:20AA600000BF00F00702064B19684FF6FF031940044B0B4343EA0221014B196000BF704784
:20AA80000CED00E00000FA0500BF00BF00BF00BF00BFBFF34F8F00BF00BF00BF094800689D
:20AAA00000F4E06008490843001D0649086000BF00BF00BFBFF34F8F00BF00BF00BF00BF29
:20AAC00000BFFDE70CED00E00000FA052DE9F04385B006463DA30FCB01AC0FC43FA00068B0
:20AAE00000904FF00008002500270024A146012E30D0022E58D0102E61D13948446800689C
:20AB000000F0807000B301A8C4F38341475C04F4803070B132484068C0F340401DF8008028
:20AB200004F4803040B12F48B0FBF8F000FB07F502E02D4807FB00F52948406800F48000A0
:20AB4000B0F5800F01D1A94603E068000321B0FBF1F935E02248046A04F44070B0F5807FC3
:20AB600005D104F0020010B14FF400491BE004F44070B0F5007F07D11948406A00F0020020
:20AB800010B149F640490EE004F44070B0F5407F07D11348006800F4003010B14FF2244904
:20ABA00001E04FF000090BE000F0A0F90C494968C1F38131491C4900B0FBF1F900E000BFAA
:20ABC00000BF484605B0BDE8F083000002030405060708090A0B0C0D0E0F101001020000C1
:20ABE0000010024000127A0000093D00F8B5044600260025207800F0010000286BD00027DC
:20AC00004348C06900F0805070B900BF4048C06940F080503E49C8610846C06900F0805040
:20AC2000009000BF00BF01273A48006800F48070B0B93848006840F4807036490860FFF7BE
:20AC400001FE064606E0FFF7FDFD801B642801D90320F8BD2F48006800F480700028F2D04D
:20AC60002B48006A00F440752DB3A08800F44070A84220D02648006A20F440750120264997
:20AC80000860002008602248056205F0010090B1FFF7D8FD064608E0FFF7D4FD801B41F228
:20ACA0008831884201D90320D3E71948006A00F002000028F0D01648006A20F44070616860
:20ACC000084313490862012F04D10846C06920F08050C86100BF207800F00200022807D193
:20ACE0000B48406820F44040A168084308494860207800F01000102807D10548406820F4C7
:20AD00008000E1680843024948600020A1E7000000100240007000404004424270B504464B
:20AD20000D4600266248006800F00700A8420ED25F48006820F0070028435D4908600846DA
:20AD4000006800F00700A84201D0012070BD207800F00200022807D15648406820F0F000B9
:20AD6000A168084353494860207800F0010000285DD06068012806D14E48006800F4003073
:20AD800090B90120E2E76068022806D14948006800F0007040B90120D8E74648006800F09F
:20ADA000020008B90120D1E74248406820F00300616808433F494860FFF744FD0646606823
:20ADC000012810D108E0FFF73DFD801B41F28831884201D90320B9E73648406800F00C0041
:20ADE0000428F0D123E06068022810D108E0FFF729FD801B41F28831884201D90320A5E7B2
:20AE00002C48406800F00C000828F0D10FE008E0FFF718FD801B41F28831884201D90320F9
:20AE200094E72448406800F00C000028F0D12048006800F00700A8420ED91D48006820F029
:20AE4000070028431A4908600846006800F00700A84201D0012079E7207800F00400042814
:20AE600007D11448406820F4E060E168084311494860207800F00800082808D10D48406876
:20AE800020F46050216940EAC1000A49486000F03DF808494968C1F30311074A515CC84089
:20AEA000064908600020FFF723FD00204EE700000020024000100240C06C01080000002047
:20AEC00001480068704700000000002000B5FFF7F7FF04494968C1F30221034A515CC84072
:20AEE00000BD000000100240D06C010800B5FFF7E7FF04494968C1F3C221034A515CC840D6
:20AF000000BD000000100240D06C0108F0B585B00FF26C0C9CE8E01001A8A0E8E0101CA534
:20AF20002D68009500210022002300240020194D696801F00C05F5B1042D02D0082D19D13C
:20AF400001E0154819E001ADC1F38346AC5D01F4803555B10F4D6D68C5F340451DF805202E
:20AF60000D4D6543B5FBF2F302E00C4D04FB05F3184602E000BF084800BF00BF05B0F0BDD9
:20AF800002030405060708090A0B0C0D0E0F1010010200000010024000127A0000093D00F3
:20AFA000F8B504460025207800F00100002878D0F848406800F00C0004280CD0F5484068AB
:20AFC00000F00C00082811D1F248406800F48030B0F5803F0AD1EF48006800F400300028B3
:20AFE0005FD0606800285CD10120F8BD00BF6068B0F5803F06D1E748006840F48030E549C4
:20B00000086028E0606858B9E248006820F48030E04908600846006820F4802008601AE034
:20B020006068B0F5A02F0BD1DA48006840F48020D84908600846006840F4803008600AE025
:20B04000D448006820F48030D24908600846006820F48020086000BF606888B1FFF7F2FBB0
:20B06000054606E0FFF7EEFB401B642801D90320BBE7C848006800F400300028F2D010E0C4
:20B08000FFF7E0FB054606E0FFF7DCFB401B642801D90320A9E7BF48006800F400300028B2
:20B0A000F2D1207800F00200022857D1B948406800F00C0050B1B748406800F00C00082878
:20B0C00018D1B448406800F4803098B9B148006800F0020020B12069012801D0012084E7BB
:20B0E000AC48006820F0F800616940EAC100A949086033E02069E8B10120A7490860FFF739
:20B10000A1FB054606E0FFF79DFB401B022801D903206AE79F48006800F002000028F2D0D6
:20B120009C48006820F0F800616940EAC1009949086013E0002098490860FFF783FB0546A1
:20B1400006E0FFF77FFB401B022801D903204CE79048006800F002000028F2D1207800F03F
:20B16000080008282DD1A069B8B101208B490860FFF768FB054606E0FFF764FB401B022866
:20B1800001D9032031E78348406A00F002000028F2D0012007F016F813E000207F490860E0
:20B1A000FFF750FB054606E0FFF74CFB401B022801D9032019E77748406A00F002000028DB
:20B1C000F2D1207800F00400042873D100267148C06900F0805070B900BF6E48C06940F0F1
:20B1E00080506C49C8610846C06900F08050009000BF00BF01266A48006800F48070B0B9CE
:20B200006748006840F4807065490860FFF71AFB054606E0FFF716FB401B642801D90320B6
:20B22000E3E65F48006800F480700028F2D000BFE068012806D15748006A40F00100554989
:20B24000086227E0E06858B95248006A20F00100504908620846006A20F00400086219E0DD
:20B26000E06805280BD14B48006A40F00400494908620846006A40F0010008620AE0454886
:20B28000006A20F00100434908620846006A20F00400086200BFE068A0B1FFF7D3FA0546A1
:20B2A00009E0FFF7CFFA401B41F28831884202D903209AE622E03748006A00F00200002852
:20B2C000EFD012E0FFF7BEFA054608E0FFF7BAFA401B41F28831884201D9032085E62D4844
:20B2E000006A00F002000028F0D1012E05D12948C06920F080502749C86100BFE069C8B36E
:20B300002448406800F00C00082860D0E069022848D1002020490866FFF794FA054606E085
:20B32000FFF790FA401B022801D903205DE61948006800F000700028F2D1206AB0F5803FC6
:20B3400007D11448406820F40030A168084311494860D4E9080108430E49496821F47411C4
:20B3600008430C49486001200B490866FFF76AFA054607E02DE0FFF765FA401B022801D955
:20B38000032032E60348006800F000700028F2D01FE0000000100240000042428004424298
:20B3A0000070004000200C490866FFF74BFA054606E0FFF747FA401B022801D9032014E6DB
:20B3C0000648006800F000700028F2D101E001200BE6002009E60000000042420010024094
:20B3E000042808D14FF0E021096941F004014FF0E022116107E04FF0E021096921F00401FE
:20B400004FF0E022116170470EB55A480078012800D10EBD5848407E08B9022001E0564860
:20B42000407E02465448418801235448F9F718FF5348007830B9534A1188534A1088534AD6
:20B4400003F0A4FD524853490978CDE90010524802784D480068029050480378484800781D
:20B46000029903F0C5FA4A480078C0434C49087047488079C04388714548B0F90200C043A6
:20B4800048804348B0F90400C04388804548007838B945488278454801893C4B444809F001
:20B4A000EDFB4448007828B940488189374A4248FCF75CFB41494248F8F7B6FF414805F0A2
:20B4C000D5FD41480088401C3F49088008460088052801DB002008803C480088401C3B49AA
:20B4E0000880084600880A2809DB00200880254B1A88997A5B8898B2354BF9F7B5FA354842
:20B500000088401C3349088008460088322804DB002008803048F9F7BDFF30480088401C0C
:20B520002E49088008460088642809DB00200880124908780A222A4906F0A8FA11498872B8
:20B5400028480088401C2749088008460088C82801DB0020088024480088401C2249088012
:20B5600008460088B0F57A7F01DB0020088000BF4FE700005C000020B00A0020C4030020A1
:20B58000D8000020DC0800202A05002094010020DE00002045040020DA00002044040020E2
:20B5A000E600002020040020C20100205C1D0020841500207E0400207C0400202205002083
:20B5C0006E1D0020D00B00205E000020600000200C02002062000020D8010020640000209A
:20B5E000E2140020660000206800002070B504462546681EB0F1807F01D301200FE0681EBD
:20B600004FF0E02148610F214FF0FF3006F062FA00204FF0E021886107200861002070BD2B
:20B6200010B5FFF7F1FE10BD7047704710B50346002200BF93F83C00012801D1022010BD85
:20B64000012083F83C0000BF22F0FF00CC6840EA040222F440708C6840EA040222F48060FE
:20B660004C6840EA040222F400600C6840EA040222F480500C6940EA040222F400504C6926
:20B6800040EA040222F480408C6940EA040222F400408C6940EA04021868426400BF0020FF
:20B6A00083F83C0000BF00BFC9E7024600BF92F83C00012801D102207047012082F83C002D
:20B6C00000BF022082F83D001068406820F0700013685860106840680B68184313685860DE
:20B6E0001068806820F0800013689860106880684B68184313689860012082F83D0000BF6F
:20B70000002082F83C0000BF00BFD5E770B504460D4604222946206809F01AF82068406CFB
:20B7200040F40040216848642068006840F0010021680860002070BD70B504460D4600221D
:20B740002946206809F004F800BF2068006A41F21111084050B92068006A8910084028B9F2
:20B760002068406C20F400402168486400BF00BF2068006A41F21111084050B92068006A04
:20B780008910084028B92068006820F001002168086000BF002070BD10B504460CB90120F4
:20B7A00010BD94F83D0028B9002084F83C00204600F00CF8022084F83D00211D206808F047
:20B7C0007FFF012084F83D000020E9E710B586B0044632492068884233D100BF30488069EB
:20B7E00040F400602E4988610846806900F40060019000BF00BF8814029000200390049046
:20B8000002A92848FEF77EFE4FF46040029002200390059002A92348FEF774FE4FF470604D
:20B82000029002200390059002A91F48FEF76AFE012211461920FFF7D4F81920FFF7C4F85D
:20B8400029E02068B0F1804F25D100BF1448C06940F001001249C8610846C06900F0010090
:20B86000019000BF00BF00BF0846806940F0040088610846806900F00400019000BF00BF6C
:20B88000012002900020039004900220059002A90548FEF737FE06B010BD0000002C0140E5
:20B8A00000100240000C0140000801400146022081F83D000868006840F001000A68106096
:20B8C000012081F83D000020704701460868C06840F001000A68D0600868006840F00100FF
:20B8E0000A681060002070472DE9F04104460D46002600BF94F83C00012802D10220BDE83B
:20B90000F081012084F83C0000BF022084F83D002068866826F0770626F47F4620688660ED
:20B92000286850283BD00CDC202860D004DC002853D0102865D155E030285DD0402860D1A8
:20B9400041E0602835D070280DD0B0F5805F03D0B0F5005F55D115E02068806820F00700C7
:20B96000216888604EE0D5E902136A68206808F0FDFE2068866826F0770646F077062068C4
:20B9800086603FE0D5E902136A68206808F0EEFE2068806840F480402168886032E0EA6858
:20B9A0006968206808F0C0FF5021206808F0EAFE28E0EA686968206808F0CBFF6021206820
:20B9C00008F0E0FE1EE0EA686968206808F0ACFF4021206808F0D6FE14E00021206808F0FB
:20B9E000D1FE0FE01021206808F0CCFE0AE02021206808F0C7FE05E03021206808F0C2FE28
:20BA000000E000BF00BF012084F83D0000BF002084F83C0000BF00BF71E7704710B50446BB
:20BA200020680069C0F34000D8B12068C068C0F34000B0B16FF0020021680861012020778A
:20BA40002068806900F0030018B12046FFF7E5FF05E0204600F0D6F8204600F0ABF9002056
:20BA6000207720680069C0F38000D8B12068C068C0F38000B0B16FF00400216808610220C7
:20BA800020772068806900F4407018B12046FFF7C4FF05E0204600F0B5F8204600F08AF951
:20BAA0000020207720680069C0F3C000D8B12068C068C0F3C000B0B16FF008002168086105
:20BAC000042020772068C06900F0030018B12046FFF7A3FF05E0204600F094F8204600F023
:20BAE00069F90020207720680069C0F30010D8B12068C068C0F30010B0B16FF01000216824
:20BB00000861082020772068C06900F4407018B12046FFF782FF05E0204600F073F82046F6
:20BB200000F048F9002020772068006900F0010058B12068C06800F0010030B16FF0010050
:20BB400021680861204600F095F920680069C0F3C01058B12068C068C0F3C01030B16FF01F
:20BB60008000216808612046FFF75EFD20680069C0F3801058B12068C068C0F3801030B18B
:20BB80006FF0400021680861204600F077FA20680069C0F3401058B12068C068C0F340109D
:20BBA00030B16FF02000216808612046FFF73DFD10BD00001FB504460E492068884218D120
:20BBC00040200090022001900320039069460A48FEF798FC00BF0949486820F4406040F0DD
:20BBE000E06040F44060486000BF0021044800F00BF81FBD000400400010014000000140B8
:20BC00001C1D00207047000030B504460D4601222946206808F08EFD0A492068884201D17E
:20BC2000012000E0002028B12068406C40F40040216848642068006840F00100216808601B
:20BC4000002030BD002C014070B504460D46164600BF94F83C00012801D1022070BD01205A
:20BC600084F83C0000BF022084F83D0036B1042E1BD0082E31D00C2E5ED145E029462068B2
:20BC800008F08AFD2068806940F00800216888612068806920F004002168886120688069A2
:20BCA000296908432168886147E02946206808F0A5FD2068806940F400602168886120687E
:20BCC000806920F480602168886120688069296940EA0120216888612FE02946206808F057
:20BCE000C5FD2068C06940F008002168C8612068C06920F004002168C8612068C06929692D
:20BD000008432168C86118E02946206808F0E4FD2068C06940F400602168C8612068C069B6
:20BD200020F480602168C8612068C069296940EA01202168C86100E000BF00BF012084F822
:20BD40003D0000BF002084F83C0000BF00BF85E710B504460CB9012010BD94F83D0028B9B9
:20BD6000002084F83C00204600F00CF8022084F83D00211D206808F0A3FC012084F83D007F
:20BD80000020E9E708B5094A016891420DD100BF0749C96941F00201054AD1611146C9690A
:20BDA00001F00201009100BF00BF08BD00040040001002407047000030B504460D460122C9
:20BDC0002946206808F0B6FC0A492068884201D1012000E0002028B12068406C40F40040A9
:20BDE000216848642068006840F0010021680860002030BD002C014030B504460D460022DE
:20BE00002946206808F096FC19492068884201D1012000E0002090B100BF2068006A41F2D5
:20BE20001111084050B92068006A8910084028B92068406C20F400402168486400BF00BFA0
:20BE40002068006A41F21111084050B92068006A8910084028B92068006820F0010021680C
:20BE6000086000BF012084F83D00002030BD0000002C014038B5044670480088401C6F49BC
:20BE8000088008460088B0F5967F01DB002008806B4840786B4B0090DA79997958796A4B6A
:20BEA0001B7800F05BFE69480078401C674908700846007805280ADB65480068806840F0F4
:20BEC000010063490968886000206049087061480068401C5F49086000F04CFA5D48C0887B
:20BEE00042F6FF7188420CDA5A480089594989880844584908810846C08889880844554905
:20BF0000C880544A917A108905F05CFD524948805249534804F0E0FA5248007852490978B4
:20BF20004840FF281AD14F4880794F4989794840FF2813D14B4880884B498988484080B2B0
:20BF40004FF6FF71884209D14648408846494988484080B24FF6FF7188420AD0FEF772FC5C
:20BF600042490968401AC82807D902204049087003E0FEF767FC3D4908603D480078012829
:20BF800002D0022856D151E03648807901284CD138480078012804D1FBF73CFA00203549D4
:20BFA000087030480078012811D0022804D003280ED0042837D116E0264B1A89264BB3F9AD
:20BFC0000210284BB3F90200FBF7DCFB2CE000BF204B1A89204BB3F90210224BB3F9040046
:20BFE000FBF7D0FB20E02448007800F0010050B9184B1A89184BB3F902101A4BB3F904006A
:20C00000FBF7C0FB0EE01C48007800F0010048B1104B1A89104BB3F90210124BB3F902009D
:20C02000FBF7B0FB00E000BF00BF04E001201149087000E000BF00BF38BD0000180500209E
:20C04000DA000020D00A00204404002010050020801D0020D0070020DC08002094010020E2
:20C06000E0020020DE000020E6000020140500203000002011050020C101002070477047AB
:20C080002DE9F0470446206805682068C668206847694FF00008C14605F00F08B8F1000F14
:20C0A0000AD105F0200038B106F0200020B1204609F05AF8BDE8F087B8F1000F6DD007F007
:20C0C000010018B906F49070002866D005F0010030B106F4807018B1E06B40F00100E063ED
:20C0E00005F0040030B107F0010018B1E06B40F00200E06305F0020030B107F0010018B14C
:20C10000E06B40F00400E06305F0080030B107F0010018B1E06B40F00800E063E06B68B392
:20C1200005F0200028B106F0200010B1204609F01BF820684069C0F38019E06B00F0080008
:20C1400010B9B9F1000F22D0204608F09EFF2068406900F04000B0B12068406920F040002D
:20C1600021684861606B50B11748616B4863606BFDF7D6FE10B1606B416B88470CE02046FF
:20C18000FFF77DFF08E02046FFF779FF04E02046FFF775FF0020E0638CE705F0800030B191
:20C1A00006F0800018B1204609F024F982E705F0400030B106F0400018B1204608F075FF74
:20C1C00078E700BF76E70000394F010810B504460CB9012010BDA06900B100E000BF94F8AC
:20C1E000390028B9002084F83800204600F028F8242084F839002068C06820F40050216845
:20C20000C860204609F012F82068006920F49040216808612068406920F02A002168486129
:20C220002068C06840F400502168C8600020E063202084F8390084F83A000020CAE700003A
:20C2400010B586B004462B49206888424FD100BF2948C06940F480202749C8610846C06976
:20C2600000F48020019000BF00BF0815029002200390012004900320059002A91F48FEF743
:20C2800041F94FF400600290002003900120049002A91A48FEF736F900BF1949486820F0B5
:20C2A000300040F0E06040F01000486000BF012211462720FEF795FB2720FEF785FB1148DC
:20C2C0000068C06840F480700E490968C8600D480068406940F001000A4909684861094865
:20C2E0000068C06840F0200006490968C86006B010BD0000004800400010024000100140C8
:20C3000000000140F82400207047704710B500F011F9054931F8100041F25551084403497B
:20C3200008810020086010BD707F0108D007002000B585B000BF0D48806940F010000B49B5
:20C3400088610846806900F01000009000BF00BF4FF460700190002002900120039001A9FB
:20C360000348FEF7CFF805B000BD00000010024000100140F8B500F0DDF8064600F0DAF821
:20C38000044600F0D7F80546A64203D1AC4201D15E4805705E48007830B95C4800785B49EB
:20C3A000487001205A4908705848007857494978884210D0FEF746FA564908605648007814
:20C3C00028B155480078401C5349087017E001205249887213E0FEF735FA4E490968401AD9
:20C3E000C8280CD900204D4988724B4908704B498881C8814A4908700120484908744748FE
:20C40000807A10B9002047490870404800783F494978454A515C884245D14048006840B1EB
:20C420003E48006842F6AA21B1FBF0F03B49888002E00120394988803A480078401C39498E
:20C4400008700846007802280DDD3448006844F63E11B1FBF0F031498881002030490870FD
:20C4600001202E4908742F4800780F280CDA274800782E4931F8100041F255510844274970
:20C4800008810020888009E00F20264908701F480078264931F810002049088100201F49EB
:20C4A0000860C88026E019484078184909781E4A515C88421ED100201A490870174988809A
:20C4C00012480078194931F8100041F255510844124908814FF6FF70086011480078401C9D
:20C4E000C0B20F490870052804DD0620087000200A490874054800680D49009003F0F8F8E1
:20C500000248007801494870F8BD0000A8030020AA030020AC030020AB030020D007002076
:20C52000B0030020B1030020607F0108707F01089401002010B51E48C07AA8B94FF4007145
:20C540001C48FEF76DF904464FF480711948FEF767F944EA4000C4B280211648FEF760F9B7
:20C5600044EA8000C4B220E04FF400711148FEF757F908B9012000E0002004464FF48071E5
:20C580000C48FEF74DF908B9012000E0002044EA4000C4B280210748FEF742F908B9012044
:20C5A00000E0002044EA8000C4B204F0070010BDD00700200010014007E0044803F0C1FE62
:20C5C000002005F0EFFCFAF777FCF6E70001002070B50446204609F0D0FEA1890122A06808
:20C5E000FEF72AF90120FAF70CFCA1882068FEF717F90546A1890022A068FEF71DF9012088
:20C60000FAF7FFFB012D01D1012070BD0020FCE71FB50446A06809F02DFE206809F02AFEEB
:20C62000A089009001200390112001906946A068FDF768FFA088009001200390112001908B
:20C6400069462068FDF75EFF1FBD2DE9F04704460F464FF000084FF08009204609F08DFE91
:20C6600000251CE0A1890122A068FEF7E5F83220FAF7C7FBA1882068FEF7D2F80646012E82
:20C6800003D149FA05F040EA0808A1890022A068FEF7D2F83220FAF7B4FB681CC5B2082D1F
:20C6A000E0DB87F800800120FAF7ABFBBDE8F08710B50446204609F068FEA1880122206844
:20C6C000FEF7BAF80120FAF79CFBA1890122A068FEF7B2F83220FAF794FBA1890022A068F0
:20C6E000FEF7AAF8A18800222068FEF7A5F80120FAF787FB10BD10B50446204609F045FE2C
:20C70000A1890122A068FEF797F8A18801222068FEF792F83220FAF774FBA1880022206868
:20C72000FEF78AF83220FAF76CFBA1890022A068FEF782F810BD10B50446204609F025FEB7
:20C74000A18800222068FEF777F8A1890122A068FEF772F83220FAF754FBA1880122206888
:20C76000FEF76AF83220FAF74CFBA18800222068FEF762F8A1890022A068FEF75DF810BD4B
:20C780002DE9F04104460D46A8468026204609F0FCFD002736E006EA0800C0B1A1880122D7
:20C7A0002068FEF749F83220FAF72BFBA1890122A068FEF741F83220FAF723FBA189002222
:20C7C000A068FEF739F83120FAF71BFB17E0A18800222068FEF730F83220FAF712FBA18972
:20C7E0000122A068FEF728F83220FAF70AFBA1890022A068FEF720F83120FAF702FB76108B
:20C80000781CC7B2082FC6DBA18801222068FEF713F80120FAF7F5FABDE8F08101480249B4
:20C82000086070470030000808ED00E0012029490978052910D12749103109789B290BD1D7
:20C84000244914310978522906D1224918310978052901D103203BE01E49097804291BD1DF
:20C860001C4910310978C32916D11A4914310978B42911D11749183109780B290CD116493C
:20C880000988802901D1022022E013490988B1F5807F1DD105201BE00E49097881B90D4960
:20C8A0001031097810290BD10A4914310978042906D10849183109780A2901D1012007E05C
:20C8C00006490968064A914201D1042000E0002070470000D0FF0FE0E0F7FF1F002004E011
:20C8E0001004031300B585B000BF2B48806940F01000294988610846806900F010000090A7
:20C9000000BF00BF254826490860401488800846808801900020029001200390086801A992
:20C92000FDF7F0FD00201E4988714872C860C87108721A481B4908604FF48040888008467A
:20C94000808801900020029001200390086801A9FDF7D8FD0020134988714872C860C87165
:20C9600008720E48104908604FF4004088800846808801900020029001200390086801A934
:20C98000FDF7C0FD0020084988714872C860C871087205B000BD00000010024000100140D2
:20C9A000FC1B0020101C0020241C00202DE9F04104460F4616469846069DB8F1000F04D144
:20C9C0000121204609F0BAFC03E00221204609F0B5FCE07900F0010020B101206072FDF708
:20C9E00031FFE060607A01281BD1207A50B9FDF729FFE060FDF726FF20610020607201202C
:20CA000028700EE0FDF71EFFE168401AB84208D9FDF718FFE060002060722870FDF712FF27
:20CA20002061287868B966B1FDF70CFF2169401AB04206D9FDF706FF20610020607201205C
:20CA40002870BDE8F0812DE9F04105460E4617469846B8F1F10F13D100240EE0BC4201D198
:20CA6000012300E000231A4605EBC403998855F83400FDF7E1FE601CC4B2B442EEDB0DE065
:20CA8000002409E005EBC402918855F834000022FDF7D2FE601CC4B2B442F3DBBDE8F08187
:20CAA00010B586B000BF2A48806940F00400284988610846806900F00400019000BF00BF99
:20CAC00000BF0846806940F0080088610846806900F00800019000BF00BF002433E01D4A63
:20CAE00002EBC40291881B4A52F834000022FDF7A3FE184800EBC400808802900120039073
:20CB000002200590134951F8340002A9FDF7FAFC114A02EBC40291880F4A52F834000022D0
:20CB2000FDF78AFE0C4800EBC400808802900120039002200590084951F8340002A9FDF704
:20CB4000E1FC601CC4B2032CC9DB06B010BD00000010024048040020600400202DE9F04721
:20CB60000746894692461C46DDF82080FDF76AFEB0F5FA6F0DD2F0232A4603219848FFF724
:20CB800062FFF023324603219648FFF75CFFBDE8F087B9F1060F06D0B9F10C0F05D0B9F161
:20CBA000FF0F06D103E0002505E0012503E0022501E0002500BF00BFBAF1060F06D0BAF1AE
:20CBC0000C0F05D0BAF1FF0F06D103E0002605E0012603E0022601E0022600BF00BF07F037
:20CBE000F000102802D0202807D107E0F1232A4603217B48FFF727FF07E000BF43462A460E
:20CC000003217748FFF71FFF00BF00BF07F00F00072843D2DFE800F04204436F7AA6AD00D9
:20CC20004CB9F123324603216E48FFF70CFF00206D49088031E0B8F1F10F22D16B48408901
:20CC400069490988884206DDF123324603216548FFF7F9FE0FE065488089634909888842EE
:20CC600006DDF023324603215E48FFF7ECFE02E000205D4908805C480088401C5A490880B9
:20CC80000BE0B8F1F00F08D1F023324603215548FFF7D9FE0020544908809DE000BF04BBCF
:20CCA00051480088B0F5167F06DAF123324603214C48FFF7C8FE0EE04B480088B0F5966F86
:20CCC00006DAF023324603214648FFF7BCFE02E000204549088044480088401C42490880EC
:20CCE00008E04346324603213E48FFF7ACFE00203D49088070E00CB9F12000E0F020034674
:20CD0000324603213748FFF79EFE65E004BB36480088B0F5167F06DAF12332460321314819
:20CD2000FFF791FE0EE030480088B0F5966F06DAF023324603212B48FFF785FE02E0002059
:20CD40002949088028480088401C2749088008E0F023324603212348FFF775FE0020224997
:20CD6000088039E0F123324603211E48FFF76BFE32E01F4800881D490989884222DB1B487A
:20CD8000408919490988884206DDF123324603211448FFF758FE0FE0144880891249098892
:20CDA000884206DDF023324603210E48FFF74BFE02E000200C4908800B480088401C0A4919
:20CDC000088008E0002008490880F023324603210448FFF738FE00BF00BF00BFD7E60000C9
:20CDE000480400206004002078040020D00A0020F40300207CB504460D46094903C9CDE9F4
:20CE00000001084803F090FA01208DF8060003208DF8000000982060019860607CBD000046
:20CE2000E0720108000100202DE9FF4F85B0804691461D464FF0000AFE4903C9CDE90301C7
:20CE4000FD48008800B2FD490880FD48B0F9020064286DDD0846B0F90000002868DDF8481B
:20CE6000B0F9020064214843F449B1F90010B0FBF1F000B2F34908800846B0F90040F2488D
:20CE80000068C0EB0420F049096801EBA010EE49086008460068001200B2EC490880E74810
:20CEA000B0F90000EA49B1F90010401A052811DDE348B0F90200E749B1F90010401A002825
:20CEC00004DDE048B0F90000E3490880DC484088E0490880D948B0F90000DD490880DF48B0
:20CEE000007820BBDE48B0F90400192829DDDD480088401CDB49088008460088282820DBEF
:20CF000000200880D1480088D749D84A128821F81200D6480088401CD44908800846008844
:20CF200032280EDB002008800120CC49087008E0C248B0F90000C6490880C1484088C54947
:20CF40000880CB48408800B2CA490880A9F16404B4F5006F02DD4FF4006000E020460446F5
:20CF600004FB04F0C11700EB5151CC12C24800780521B1EBD00F17DBB14AD17BBF4A12798B
:20CF8000012383EAD21003F0A1F9BC490979BC4A92F910201144B84A127801EBD2010A316E
:20CFA0004843C0F3872A16E0A54AD17BB34A1279012383EAD21003F089F9B0490979B04A6C
:20CFC00092F910201144AC4A127801EBD20115394843C0F3872A0AF1010060433221484348
:20CFE000A849C98990FBF1F000B2A74908800AEB8A00162101EB40009049B1F90010884219
:20D0000002DA0020A04908809B480078C0F3800038B18A48B0F900003C2802DC00209A496C
:20D0200008809948B0F90000002803DD9648B0F9000000E00020944908800846B0F90000F3
:20D040008C49B1F90010884203DA8F48B0F9000002E08848B0F900008B4908809DF81800B6
:20D06000C0F34000B0B305F00F00012806D002280FD0032818D004282DD120E04FF4FA6272
:20D0800001217C48B0F9000007F076FA7F4908602CE040F2DC5201217648B0F9000007F07E
:20D0A0006BFA7A49086021E04FF47A7201217148B0F9000007F060FA7449086016E04FF47D
:20D0C000FA7201216B48B0F9000007F055FA6F4908600BE00BE04FF47A7201216548B0F983
:20D0E000000007F049FA6949086000BF09E04FF4FA7201215F48B0F9000007F03DFA634939
:20D1000008604FF47A7201215A48B0F9000007F033FA5F4908605248807968B94848B0F9EA
:20D120000200642808DD464840885A490880084600880004584908609DF81800C0F3400078
:20D14000F0B305F00F00012806D0022814D0032824D0042842D134E04B49B1F9001001EB6F
:20D16000C10108114C4B4A490A684849096809F029F9484908803EE04349B1F9001001EBB2
:20D18000410202EBC1010811434B41490A683F49096809F017F93F4908802CE03A49B1F9AF
:20D1A000001001EB810202EBC10108113A4B38490A683649096809F005F9364908801AE0C8
:20D1C0001AE0354B32480268304801682E48B0F9000009F0F7F82F4908800CE02E4B2C4830
:20D1E00002682A4801682848B0F9000009F0EAF82849088000BF0BE0274B2548026823489F
:20D2000001682148B0F9000009F0DCF8214908806FF0C7002149086140F634004861204860
:20D22000C08901B21D4A1B48B0F9000004F074FD1C4939E0C8720108F40300202E010020F3
:20D24000DC08002034010020100100203601002032010020300100201401002018010020DB
:20D26000DE0000201A0100201408002016010020F00A002038010020C1010020B00A0020D3
:20D28000D00A00200C0200203A0100203C010020400100204401002028010020DC0600209D
:20D2A000D00700204E01002008806FF063005849086140F21A404861564AD17B564A127A67
:20D2C000012383EAD21002F0D3FF5349097A4FF47A7251434843401400904E480089C111D5
:20D2E0004E4A009804F018FD4D4908804D4A117B484AD0884C4A128801F05EFC07464A4870
:20D30000078001231A4649480188384601F0ACFD46490880404A517A3E4A907D01F03AFCA8
:20D3200083463D4A527A0F3A91B23A4A507D01F031FC019001980BFB00F0810A02910299FD
:20D3400088B201231A463A49098801F08DFD384908803848B0F9000034490988484386121D
:20D36000334800887043861233480078B0B933480068301A022805DD30480068801C2F49D6
:20D38000086018E02D480068301A10F1030F12DA2A480068C01E294908600CE027480068B2
:20D3A000132805DD2548006810382449086002E00020214908702148006810F1C80F03DAF4
:20D3C0006FF0C7001D4908601D48008818B91D4802F0B7FF02E01B4802F0A6FF17480068EB
:20D3E0000F49B1F900100844401000B2ADF8100001208DF8120004208DF80C000398C8F850
:20D4000000000498C8F8040009B0BDE8F08F0000DC060020DC080020B00A0020B806002011
:20D4200050010020F00A00205201002054010020560100204E0100204C01002048010020BD
:20D4400044010020000100202DE9FF4F87B0824616461F46FE4903C9CDE90501002004909F
:20D460000390BE4203DA07FB07F0C01202E006FB06F0C012F749488008464088B0F5006F94
:20D4800002DD4FF4006001E0F2484088F14948809DF82000C0F3400000287CD01498032832
:20D4A0007AD004DC012807D0022876D149E0042874D03328F9D1D7E0E748007A002801DCAE
:20D4C000012001E0E448007A0490E348407A0390E0484088E049C9884843C00A04B2DE48FD
:20D4E000C088A04202DADC48C08800E0204604B2D9484089D949097A48434FF47A714843EB
:20D50000401400EBC00101EB00104FF6FF7101EA800501230522D2480188284601F0A4FCFD
:20D52000CF490880CC48C0884042CE49086100204861C948C0888002404288610020C86195
:20D54000DFE0C548007D002801DC012001E0C248007D0490C048407D0390BE484088BE4933
:20D56000498A4843C00A04B2BB48408AA04202DAB948408A00E0204604B2B748C08AB74932
:20D58000097A48434FF47A714843401400EBC00101EB001003E0B5E01DE0ADE063E04FF63E
:20D5A000FF7101EA800501230522AD480188284601F05AFCAA490880A748408A4042A94965
:20D5C000086100204861A448408A8002404288610020C86195E0A04890F82000002801DC23
:20D5E000012002E09C4890F8200004909A4890F821000390974840889749C98B4843C00ABA
:20D6000004B29548C08BA04202DA9348C08B00E0204604B29048408C9049097A48434FF47E
:20D620007A714843401400EBC00101EB00104FF6FF7101EA80050123052289480188284640
:20D6400001F012FC864908808348C08B404285490861002048618048C08B800240428861DC
:20D660000020C8614DE000BF7B4890F82C00002801DC012002E0784890F82C000490764830
:20D6800090F82D000390734840887349498D4843C00A04B27048408DA04202DA6E48408D5C
:20D6A00000E0204604B26C48C08D6C49097A48434FF47A714843401400EBC00101EB0010F5
:20D6C0004FF6FF7101EA80050123052264480188284601F0C9FB624908805F48408D404259
:20D6E00060490861002048615B48408D8002404288610020C86104E000200490039000245A
:20D7000000BF4DE09DF82000C0F34000F0BB524890F83800002801DC012002E04E4890F84A
:20D72000380004904C4890F82D000390494840884949498D4843C00A04B24748408DA04237
:20D7400002DA4548408D00E0204604B24248C08D4249097A48434FF47A714843401400EB2F
:20D76000C00101EB00104FF6FF7101EA8005012305223B480188284601F076FB3849088097
:20D780003548408D40423749086100E008E0002048613148408D8002404288610020C861C7
:20D7A000314890F90E00322805DC2F4890F90E0010F1320F02DA00202B4988732A4890F968
:20D7C0000F00322805DC284890F90F0010F1320F02DA00202449C873244800780521B1EB6B
:20D7E000D00F63DB224AD17B1C4A1279012383EAD21002F06BFD194909791B4A92F9102092
:20D8000011449DF8202001EBD201083101EB8101154A92F90E2002EB41014843C0F38F2044
:20D8200014490880124AD17B0C4A1279012383EAD21002F04BFD094909790B4A92F91020E9
:20D8400011449DF8202001EBD2010A3114E00000D0720108F0000020E40B0020B00A00206C
:20D860005A01002000070020D00A0020C1010020DC0800205E01002001EB8101BA4A92F9AA
:20D880000F2002EB410116314843C0F38F20B749088008460088B6490988401AC01E4FF48D
:20D8A000806191FBF0F0B34908804CE0B24AD17BB24A1279012383EAD21002F007FDAF493B
:20D8C0000979A94A92F9102011449DF8202001EBD201173901EB8101A34A92F90E2002EBDE
:20D8E00041014843C0F38F20A1490880A24AD17BA24A1279012383EAD21002F0E7FC9F49A8
:20D900000979994A92F9102011449DF8202001EBD201153901EB8101934A92F90F2002EBBE
:20D92000410116314843C0F38F2090490880084600888F490988401AC01E4FF4806191FBE9
:20D94000F0F08C4908808E480078C0F3800078B98C48008800908748008803B2844802888A
:20D9600000210846FAF75CF86043800A04B20EE08448008800907F48008803B27C480288EC
:20D98000FF213C20FAF74CF86043800A04B27E488480B0F90400002802DC00207A4988808B
:20D9A0007848008872490988884220DD7648B0F904007549B1F90610401A022806DD724802
:20D9C000C088401C00B27049C88033E06E48B0F904006D49B1F90610401AB0F1FF3F29DAC8
:20D9E0006948C088401E00B26749C88022E000BF6548B0F904006449B1F90610401A02281A
:20DA000007DD6148C1880498084400B25E49C88010E05D48B0F904005B49B1F90610401AA7
:20DA2000B0F1FF3F06DA5848C1880398081A00B25549C8805448B0F90600062801DA06206F
:20DA400002E05148B0F906004F49C8804D48008846490988884208DD01204B490870002083
:20DA6000C8804A4802F06DFC02E0484802F05CFC474A117B404AD088464A128801F09CF807
:20DA800081464448A0F8009001231A4642480188484601F0E9F940490880384A517A364A35
:20DAA000907D01F077F80290344A527A0F3A91B2314A507D01F06EF80190DDE901104843FF
:20DAC0004FEA902B1FFA8BF001231A463349098801F0CAF931490880274AD17B274A127ABD
:20DAE000012383EAD21002F0C3FB2D4909884843642190FBF1F0801200B200901E480089BD
:20DB0000C111284A009804F007F9274908801E48B0F906002049098848434FEAA0281F483B
:20DB2000008808FB00F04FEAA0281F48B0F9000040444FEA6008B8F1000F01DA002000E0A1
:20DB4000404600B2ADF8160001208DF81A0004208DF814000598CAF800000698CAF8040092
:20DB60000BB0BDE8F08F0000D00A0020600100205E01002062010020DC080020B00A00206B
:20DB8000C1010020F4030020F000002000010020F00A0020640100206601002068010020AC
:20DBA0005A01002000070020580100202DE9FF4F8BB081468A46FE4903C9CDE909014FF002
:20DBC000000B0020089005900490FA48A0F802A0F9480088C82801DA642002E0F64800881D
:20DBE00080100690F34841880698814204DBFCF729FEF249086020E0F148B0F90200C8282A
:20DC000007DDEF48B0F90200EE4991FBF0F086B201E04FF49666B6F5FA7F02DA4FF4FA7096
:20DC200000E030460646FCF70DFEE4490968401AB04202D90120DF490870E14800883C28A9
:20DC400012DDDD480088C82801DA96200AE0DA480088B0F52F7F02DD40F20D2002E0D64882
:20DC600000884010079010E0D3480088C82801DA962009E0D0480088B0F52F7F02DD40F234
:20DC80000D2001E0CC4800880790CA4841880798814202DB0020C7490870CB48407801288D
:20DCA00002D0C948807810B90120C2490870C148007801283ED1BF48B0F90610C3484079D9
:20DCC000002801DA032007E0C0484079052801DD032001E0BD484079401EBD4A105C814215
:20DCE0000CDC0020B349C880BA4802F02AFB0120B94908700020B9490880EEE3AD48B0F90B
:20DD00000610B2484079002801DA032007E0AF484079052801DD032001E0AC484079401E63
:20DD2000AB4A105C081A00B2A249C880A94802F0FBFAD2E39F490E984880A148B0F9020004
:20DD4000B0F5FA7F23DDA04800780F281FDB08464088C8281BDD9A48B0F902006421484379
:20DD60009949097890FBF1F09D4908609D4800680968C0EB01309B49096801EBA020994909
:20DD8000086008460068C0F30F30974908800D9804286ED006DC012809D0022863D0032890
:20DDA00068D1C0E005287DD03328F9D1F9E18F48007A002801DC012001E08C48007A8346A2
:20DDC0008A48407A0890DFF8ECC1BCF80230DFF81CC2BCF80220BCF80010BCF800C04FEAB9
:20DDE0006C00F7F7FDFB734949884843800A04B27E488088A04202DD7C48808800E02046D8
:20DE000004B27A48C088A04202DA7848C08800E0204604B2754840896C49097A48434FF4F4
:20DE20007A714843401400EBC00101EB00104FF6FF7101EA8005012305226D480188284654
:20DE400001F012F86A4908806848C088404269490861002048616548C0888002404288614C
:20DE60000020C8610CE26148007D002803DC012003E0DAE0FEE15D48007D83465B48407D56
:20DE80000890DFF830C1BCF80230DFF860C1BCF80E20BCF80C10BCF80CC04FEA6C00F7F77F
:20DEA0009FFB00E01CE1434949884843800A04B24E48008AA04202DD4C48008A00E020467E
:20DEC00004B24A48408AA04202DA4848408A00E0204604B24548C08A3C49097A48434FF46F
:20DEE0007A714843401400EBC00101EB00104FF6FF7101EA8005012305223D4801882846C4
:20DF000000F0B2FF3A4908803848408A404239490861002048613548408A800240428861A1
:20DF20000020C861ACE1314890F82000002801DC012002E02D4890F8200083462B4890F801
:20DF400021000890DFF86CC0BCF80230DFF89CC0BCF81A20BCF81810BCF818C04FEA6C00F1
:20DF6000F7F73EFB134949884843800A04B21F48808BA04202DD1D48808B00E0204604B2E3
:20DF80001A48C08BA04202DA1848C08B00E0204604B21648408C0D49097A48434FF47A71B3
:20DFA0004843401414490978484385B2012325E0E8720108F0000020C201002070010020D2
:20DFC000DC08002020550300C4030020B00A00200101002000010020790100207A0100208C
:20DFE000840100208801002006020020E40B00207601002000070020EE0000200522F94868
:20E000000188284600F030FFF6490880F648C08B4042F649086100204861F348C08B80029F
:20E02000404288610020C8612AE1EF4890F82C00002801DC012002E0EB4890F82C0083467E
:20E04000E94890F82D000890DFF8A4C3BCF80230DFF894C3BCF82620BCF82410BCF824C076
:20E060004FEA6C00F7F7BCFAE14949884843800A04B2DD48008DA04202DDDB48008D00E08E
:20E08000204604B2D848408DA04202DAD648408D00E0204604B2D448C08DD649097A48433C
:20E0A0004FF47A7148434014D3490978484385B201230522CB480188284600F0D5FEC949CA
:20E0C0000880C948408D4042C849086100204861C548408D8002404288610020C861CFE056
:20E0E000C14890F84400002801DC012002E0BE4890F844008346BC4890F845000890DFF868
:20E10000F0C2BCF80230DFF8E0C2BCF83E20BCF83C10BCF83CC04FEA6C00F7F761FAB44941
:20E1200049884843800A04B2AF48B0F84000A04203DDAD48B0F8400000E0204604B2AA48D7
:20E14000B0F84200A04203DAA748B0F8420000E0204604B2A448B0F84600A649097A48436A
:20E160004FF47A7148434014A3490978484385B2012305229B480188284600F075FE9949F9
:20E1800008809948B0F84200404298490861002048619548408D8002404288610020C861B7
:20E1A0006EE0914890F83800002801DC012002E08D4890F8380083468B4890F839000890E6
:20E1C0008B484088B0F5FF7F15DADFF824C2BCF80230DFF814C2BCF80E20BCF80C10BCF8DC
:20E1E0000CC04FEA6C00F7F7FBF9814949884843800A04B207E07E48408840437A49498ED4
:20E20000B0FBF1F004B27848808EA04202DD7648808E00E0204604B27348C08EA04202DA9E
:20E220007148C08E00E0204604B26F48408F7149097A48434FF47A71484340146E49097848
:20E24000484385B20123052266480188284600F00BFE644908806448C08E4042634908614D
:20E26000002048616048C08E8002404288610020C86105E04FF0000B00200890002400BFDF
:20E2800000BF5E4890F90E00322805DC5B4890F90E0010F1320F02DA002058498873574894
:20E2A00090F90F00322805DC544890F90F0010F1320F02DA00205149C873514AD17B4D4AC6
:20E2C0001279012383EAD21002F000F8494909794A4A92F91020114401EB8101474A92F914
:20E2E0000E2002EB41014843C0F38F2045490880434AD17B3F4A1279012383EAD21001F06D
:20E30000E5FF3C4909793D4A92F91020114401EB81013A4A92F90F2002EB410116314843CE
:20E32000C0F38F20384908800846008835490988401AC01E4FF4806191FBF0F033490880C1
:20E340003348008800900846008803B22D48028800210088F9F764FB6043800A04B2244859
:20E360008480B0F90400002802DC002020498880274800882349098801EB8101B0EB410F08
:20E3800020DD1B48B0F904001949B1F90610401A022806DD1648C088401C00B21449C8808E
:20E3A000ADE01348B0F904001149B1F90610401AB0F1FF3F05DA0E48C088401E00B20C4993
:20E3C000C8809CE000BF13480078012875D109484078032822D100200F4908800D49087083
:20E3E0008DE0000076010020E40B002000070020F0000020B00A0020EE000020D00A0020F1
:20E40000DC0800208C0100208E01002090010020F4030020790100207A010020824840781D
:20E42000012805D14FF4967005901E20049003E0642005900A2004907C480088401C7B4907
:20E44000088008460188059881422FDC7848B0F904007749B1F90610401A022814DD7348D5
:20E460000188049891FBF0F0C0F10A006F49098891FBF0F200FB121070BB6D48C0885844B8
:20E4800000B26B49C8803AE06948B0F904006849B1F90610401AB0F1FF3F30DA6448C188AD
:20E4A0000898081A00B26249C88028E000205F4908806049087022E0FFE75D48B0F9040042
:20E4C0005B49B1F90610401A022807DD5848C088584400B25649C88011E02EE05448B0F90F
:20E4E00004005349B1F90610401AB0F1FF3F06DA4F48C1880898081A00B24D49C8804C48DD
:20E50000B0F90600062801DA062002E04848B0F906004749C8804848008848490988884220
:20E5200008DD0120424908700020C880444801F008FF02E0424801F0F7FE424A117B424AF0
:20E54000D088424A128800F037FB80463F48A0F8008001231A463E480188404600F084FC2D
:20E560003B490880304A517A374A907D00F012FB02902D4A527A0F3A91B2334A507D00F024
:20E5800009FB0190DDE901104843810A0391039988B201231A462F49098800F065FC2D493B
:20E5A0000880294AD17B204A127A012383EAD21001F05EFE284909884843642190FBF1F0E0
:20E5C000801200B2009020480089C111234A009803F0A2FB224908801548B0F906001C49AB
:20E5E0000988484387121B480088784387121C48B0F9000038444710002F01DA002000E03D
:20E60000384600B2ADF8260001208DF82A0002208DF824000998C9F800000A98C9F804009B
:20E620000FB0BDE8F08F0000B00A00207A010020F000002079010020F40300208E01002012
:20E6400000010020F00A0020DC0800207C0100207E010020800100207601002000070020E0
:20E66000740100202DE9FF5F82460E468C4903C9CDE90201002700BF0025002E40D1A946E2
:20E680008848C07F08B9872001E08648C07F8146854840680A21C1EB4911884205D282483D
:20E6A0004068401C8049486010E07F4840680A2101EB4911884205D97B484068401E7A49E1
:20E6C000486003E04FEA491077494860774AD17B744A127A012383EAD21001F0C9FD71497A
:20E6E000097A4FF4FA7251434843401400906F480089C1116E4A009803F00EFB044655E008
:20E700006C484088400141F2883190FBF1F0C5B2012D01DA012000E0284605466548408835
:20E720004001654909784843642190FBF1F00A385D494968884205D95B48406828445A4952
:20E74000486026E05B48408840015B4909784843642190FBF1F00A305349496888420DD28E
:20E7600051484068A84205D94F484068401B4E4948600EE000204C4948600AE04D48408825
:20E7800040014D4909784843642190FBF1F046494860464A1289D111424A127A4FF47A7319
:20E7A0005A43D011424A03F0B7FA04463F4AB2F902103D4A5268520910B2404A03F0ACFA9A
:20E7C0000746381907B236BB4FF000093548807F08B93C2001E03348807F814633480088EB
:20E7E000A9F105018AB2009088B280230021F9F717F97843800A07B22C480088484506DD45
:20E800000020294948602E4801F09BFD02E02C4801F08AFD02E02A4801F086FD254A117B2E
:20E82000224AD088274A128800F0C6F980462548A0F8008001231A4623480188404600F021
:20E8400013FB21490880174A517A184A907D00F0A1F9019001231A461C480188019800F008
:20E8600003FB1A4908801848008878434FEAA02B084600880BFB00F04FEAA02B0FFA8BF0B4
:20E88000ADF80C0001208DF80E008DF808000298CAF800000398CAF80400BDE8FF9F000086
:20E8A000D8720108B00A0020F8000020DC080020B8060020F00A0020DB010020DC06002019
:20E8C000000100206A0100206C0100206E01002070B504460D461646FBF7B4FF3C490968B7
:20E8E000401A642870D3FBF7ADFF394908603948006828443749086037480078401C364958
:20E9000008700846007808280ADB32480068C0F3CF003249088000202F4908702D4908604F
:20E92000462C0BDA2D48008841F27071884205DD2B480088401C2A49088002E000202849FE
:20E940000880462C05DC2548008841F28831884207DA962E05DA23480088401C214908806C
:20E9600002E000201F4908801D480088B0F5967F05DD00201A49088001201B4908701948B3
:20E980000088642804DD0020164908801649087015480078012814D1462C0EDA04F11E0054
:20E9A0001249087008460078642801DD642001E00E4800780D49087006E064200B4908701D
:20E9C00002E06420094908700848007870BD0000A4000020A8000020AC000020AE000020EC
:20E9E000B0000020B2000020B4000020B50000202DE9FF4385B0074615469846DDE910944F
:20EA000008EA090000F00103BDF81A10554800782A46049001F0E6FB06462078B04223D074
:20EA20005148007800BB052601204F4908702078042819D14D480068142806DD042600209A
:20EA4000087001204A4908700EE000204949086049490860494908804449086044490870FC
:20EA60000526012040490870062E68D2DFE806F06733574B03683B48007800F0010078B95A
:20EA800005F00F03BDF81A20364800780146029003A8FEF7C9F9039820600498606016E0E2
:20EAA0003048007800F0010088B105F00F000090BDF81830BDF81A202A48007801460290F9
:20EAC00003A8FEF7C1FC039820600498606000202549087041E02A480078012807D12948DF
:20EAE000B0F9020040012649486000200870394603A8FFF7B7FD0398206004986060002010
:20EB00001949087029E0294603A8FEF773F903982060049860600020134908701DE01A48CD
:20EB20000389BDF818102A4603A8FFF73FF8039820600498606000200B4908700DE000BF15
:20EB4000124801F0FEFB1248F6F794FF052020700020A0716080A08000BF00BF09B0BDE8D5
:20EB6000F0830000C101002092010020480100204C010020100100202801002044010020D8
:20EB8000F8000020DC080020C4030020000100209401002010B502464FF480608A4208DDBB
:20EBA00001FB01F4A302B3FBF2F4B4FBF2F4A0B201E04FF4806010BDF0B503460E461546D6
:20EBC000002100244FF48060182E04D0242E12D0302E34D121E0E721FC2401EBC10707EB4D
:20EBE0000117B3EB870F02DD4FF4806701E0B3FBF1F73A4625E04FF4A5714FF4B47401EB14
:20EC0000C10707EB0117B3EB870F02DD4FF4806701E0B3FBF1F73A4613E040F2AD114FF4C8
:20EC2000EA7401EBC10707EB0117B3EB870F02DD4FF4806701E0B3FBF1F73A4601E064221D
:20EC400000BF00BF02FB02F74FF0640CB7FBFCF75743B7FBFCF75743BF0242F2107CB7FBE0
:20EC6000FCF2B2F54D7F02D24FF44D7700E017463A46AA4201D290B200E0284604EBC40792
:20EC800007EB0417B3EB870F01DD4FF48060F0BD2DE9F04105460E4617461C46002F7DD163
:20ECA000552D66D14748007820BBFBF7CBFD45494968401AB0F57A7F15D9012041490870B7
:20ECC0000020207040480078C043404908703E484078C04348703E48007820F00200801CDB
:20ECE0003B49087018E03A48007820F002003849087011E00020207033480078C043334908
:20ED0000087031484078C04348703148007820F00200801C2E490870AA2E06D12C48007866
:20ED200020F004002A49087023E02A480078C8B9FBF788FD27494968401AB0F57A7F0AD9F3
:20ED40000120244908702248007820F00400001D1F4908700DE01E48007820F004001C4976
:20ED6000087006E01A48007820F00400001D1849087019480078E0B9FBF764FD164949687C
:20ED8000401A41F2883188420CD90120124908700F48007820F00100401C00E010E00C4929
:20EDA00008700DE00A48007820F001000849087006E00748007820F00100401C044908706B
:20EDC000BDE8F081E4010020DA000020DC000020B8010020EC010020F401002001201349AA
:20EDE000087000204860012011490870002048808880C8800F4908600F4908600F49086068
:20EE00000F4908600F4908600F4908600F4908600F4908620F4908620F4908620F490862EA
:20EE20000F4908620F49086270470000F8000020F000002004000020080000200C000020F7
:20EE40001000002014000020180000201C000020700600204C0600209406002000070020F1
:20EE6000DC060020B806002070B504461546661A32B2002A06DDAA4202DB4E19B0B20CE0F9
:20EE800020460AE0002A07DA56429E4202DBCE1AB0B202E0204600E0204670BD10B5FBF706
:20EEA000D1FC2E490968401A642855D3FBF7CAFC2A4908602A4800782A4908702A4800783D
:20EEC000487000208870C8702848008800B288802748008800B2C88026484088088125485B
:20EEE0000088488124480088888123484088C88122480089088222480068801200B24882EB
:20EF000020480068801200B2888215480078022803D113484088C8821EE01148007801289B
:20EF200004D10F4880880F49C88215E00C48007804280ED11448007800F0010020B9084841
:20EF400080880849C88207E0054840880549C88202E000200349C88210BD00008400002071
:20EF6000DE000020FC0800203000002004000020080000202C0000202A050020C403002051
:20EF8000100000200C000020C101002070B505460E46144608216748FBF742FC66490870E6
:20EFA0004FF400416548FBF73BFC6549087062480078644909784840634908705E480078B7
:20EFC000604908705E480078604909784840604908705B4800785D4908705748007858492E
:20EFE000097848405B490870FBF72CFCB0F57A7F0CD2FBF727FC58490860FBF723FC574987
:20F000000860FBF71FFC5649086070BD2088C0F38030002878D1B5F5966F7CDD462E7ADDF8
:20F020004948007800BBFBF70DFC4B490968401A42F2107188421BD9206820F4804000F5EE
:20F04000804020600120474948800846F8F75EFA00204549087045484088401C4349488037
:20F06000022043490870D0E7FBF7ECFB3A4908603748007800BBFBF7E5FB38490968401A1F
:20F0800041F2883188421BD9206820F4804000F5804020600220334948800846F8F736FA62
:20F0A00000203149087031484088401C2F49488002202F490870A8E7FBF7C4FB2749086037
:20F0C0002448007810BBFBF7BDFB25490968401A41F2883188422AD9206820F4804000F594
:20F0E0008040206003201F4948800846F8F70EFA00201D4908701D484088401C1B49488085
:20F1000002201B49087080E711E004E0FBF79AFB134908600BE0FBF795FB0F490860FBF74B
:20F1200091FB0E490860FBF78DFB0D49086000BF6BE70000000C0140DC02002000080140A7
:20F14000DD020020C5020020C4020020CD020020CC020020D4020020C8020020D002002034
:20F16000D802002090070020A5030020300B0020C60100201FB53848007890B93748807E42
:20F1800055280ED1364A374800783749498889B2CDE9010200913549887835490EC900F003
:20F1A000A5FE2F492F480078CDE9010130488068304A00901178304A10892D4A0CCA00F04A
:20F1C0002DFF274801902D488088ADF80000264B5B889AB2244B1989224B9879274B1C68BC
:20F1E00002949B88ADF80C30234600F09FFD1E4A917D507D1A4A00F01BFD1F4988891849F7
:20F2000000F074FA1D48016802918088ADF80C00134ADDE9020100F0D1FB114800F03CF817
:20F220000F48134A009011780F4A528890B2144A12680392134A1388039A00F093FC0848BB
:20F24000114900904A8911490878114B1149098800F00EFB1FBD0000D8000020B00A002029
:20F2600094010020DE000020DC080020F4030020C4030020DA0000205C1D00203A050020E7
:20F280002A050020060200206E1D0020DC010020DB070020D801002010B50446FBF7D2FA87
:20F2A00041F2883188420CD2FBF7CCFAEE490860FBF7C8FAED490860FBF7C4FAEC490860C4
:20F2C00010BD2068C0F3804000286FD14FF40041E848FBF7A5FA00BBFBF7B4FAE3490968C1
:20F2E000401A41F2883188421BD9206820F4802000F5802020600120DF4948800846F8F76B
:20F3000005F90020DD490870DD484089401CDC4948810220DB49087003E0FBF793FAD349BD
:20F320000860D9480088002847D1D8480078012843D1D748007805283FD0D5488079012895
:20F340003BD1D348B0F90400C82804DCD048B0F90200C82831DDCF48807A40BBCE4800899D
:20F36000C82825DAFBF76EFAC1490968401A41F28831884225D9206820F4802000F58020EA
:20F3800020600220BC494880BF48008888800846F8F7BCF80020B9490870B9484089401CB6
:20F3A000B74948810220B74908700AE08DE0FFE7FBF748FAAE49086003E0FBF743FAAC4913
:20F3C0000860FBF73FFAA8490968401A14287CD3FBF738FAA4490860B048C088B049096830
:20F3E0000844AF490860AF480088AF4909680844AD490860AB484088AC4909680844AB496E
:20F400000860A8488088AA4909680844A8490860A8480078401CA749087008460078202849
:20F420007EDB002008709E4800684FF4FA71B1EB501F2FD89A480068C900B1EB501F29D3B3
:20F440009948006841F28831B1EB501F22D8964800684EF66021B1EB501F1BD3934800682B
:20F4600041F28831B1EB501F14D8904800684EF66021B1EB501F0DD38D48006841F2883190
:20F48000B1EB501F06D88A4800684EF66021B1EB501F16D2206820F4802000F58020206040
:20F4A0000320754948800846F8F730F800207349087073484089401C7149488102207149AB
:20F4C00008707D480068C82100E0C2E0B1EBA02F36DA7A48008872490968C0EB51101928DE
:20F4E0002AD277480078401C75490870084600780A2828DD206820F4802000F580202060F9
:20F5000004205D49488066480068C0F34F1088800846F7F7FBFF002058490870584800E03A
:20F520001AE04089401C5649488102205549087000206349087006E000206149087002E0BE
:20F5400000205F4908700020554908605649086056490860564908604F48407B00287AD16B
:20F560004D484088002876D1FBF76CF955490968401A41F28831884274D94848C088524989
:20F58000524A127821F812004648008850494F4A127821F81200434841884E484B4A127814
:20F5A00020F812103F4881884B48484A127820F8121046480078401C44490870084600786B
:20F5C00032284FDB0020087032213F48F8F746FF4249086032213E48F8F740FF4049086016
:20F5E00032213C48F8F73AFF3E49086032213A48F8F734FF3C49086038480068B0F5FA7F33
:20F600000DD83748006842F6E061884207D835480068884203D834480068884222D9206841
:20F6200020F4802000F5802020600520124948802A48008888800846F7F768FF00200F499C
:20F6400008700F484089401C0D49488102200D49087007E0FFE700201C490870FBF7F2F801
:20F660001849086000BF2BE6680200206C020020700200200010014090070020A503002077
:20F68000300B0020C6010020D001002030000020DE000020D0070020DC0800206E1D002043
:20F6A00078020020220500207C0200208002002084020020740200200C000020400500205C
:20F6C000750200209C020020D212002088020020361300209A130020FE1300208C02002012
:20F6E0009002002094020020980200207047000013B50C465448007860B9FBF7A3F85349C1
:20F7000008609DF8012006215148F4F7DAF901204D4908702078C0F3C01000287ED19DF8F7
:20F72000000018B19DF80000072821D1FBF78AF846490968401AB0F57A7F1DD9206820F050
:20F740008000803020600120424948809DF8000088800846F7F7DAFE00203F4908703F482D
:20F76000C08A401C3D49C88201203D4908701CBDFBF768F8354908609DF800009DF80110A8
:20F7800088425FD09DF80010364802780078401C344B18702E48815418460078062851DB7D
:20F7A00000201946087006212948F5F7E3FE28B92D480068401C2C49086006E000202A497D
:20F7C0000860FBF73FF82949086027480068322838D9FBF737F82549096801F5FA71884251
:20F7E00030D9206820F08000803020600220194948801748007800021549497800EB011078
:20F80000134989780844134988801148C07800020F49097900EB01100D4900E012E0497988
:20F8200008440C49C8800846F7F770FE00200A4908700A48C08A401C0849C8820120084945
:20F84000087094E700BF92E7AE020020B0020020B802002090070020A5030020000B002057
:20F86000C6010020BE020020C0020020B40200202DE9F04105460E4614469846069FFAF755
:20F88000E1FFB0F57A6F01D2BDE8F081FAF7DAFF42F21071884220D23868C0F3804000289B
:20F8A0007CD1FAF7CFFF3E490968401A142875D3FAF7C8FF3A49086098F80000A8BB0DB112
:20F8C000C82E0BDD40F2C270844207DD40F63E00844203DA0020334908705FE031480078E1
:20F8E000401C3049087008460078FA2856DB00200870386820F4802000F580203860082061
:20F900002949488005EB860088800846C480F7F7FDFD00202549087025484089401C2449B0
:20F92000488102202349087038E0FFE70DB1C82E03DD002088F8000030E040F68B608442CF
:20F9400002DCB4F5BA7F26DA1B480078401C1A49087008460078FA2820DB002008703868BA
:20F9600020F4802000F58020386009200E49488005EB860088800846C480F7F7C7FD00207C
:20F980000A4908700A484089401C0949488102200849087002E000200749087000BF73E73C
:20F9A000A8020020AC02002090070020A5030020300B0020C6010020AD02002037B51446D9
:20F9C0006048007801280CD0FAF73CFF5E490860FAF738FF5D490860FAF734FF5C49086060
:20F9E0003EBD2068C0F30040002875D1BDF90000002801DB014600E0414244F62062914230
:20FA000028DDFAF71FFF50490968401AB0F57A7F24D9206820F4803000F580302060012041
:20FA20004C494880BDF90000002801DB014600E04142484A91801046F7F768FD002046490A
:20FA400008704648C088401C4449C880022044490870C5E7FAF7F6FE3B490860BDF90200CB
:20FA6000002801DB014600E0414244F62062914228DDFAF7E7FE35490968401AB0F57A7F87
:20FA800024D9206820F4803000F580302060022030494880BDF90200002801DB014600E0B2
:20FAA00041422C4A91801046F7F730FD00202A4908702A48C088401C2849C880022028495E
:20FAC00008708DE7FAF7BEFE20490860BDF90400002802DB014601E031E0414244F6206285
:20FAE000914228DDFAF7AEFE19490968401AB0F57A7F24D9206820F4803000F58030206058
:20FB0000032014494880BDF90400002801DB014600E041420F4A91801046F7F7F7FC002074
:20FB20000D4908700D48C088401C0C49C88002200B49087054E7FAF785FE0549086000BF4F
:20FB40004EE700003000002050020020540200205802002090070020A5030020300B0020E4
:20FB6000C60100202DE9FF4105460E461F460A9C2068C0F3805000284BD1FAF763FE26498E
:20FB80000968401A142844D3FAF75CFE22490860B5F5FA7F3ADD0F2E38DBBDF80800C828F2
:20FBA00034DDBDF80A00322830DA40F2DC50874228DD1A480088401C1849088008460088E0
:20FBC000FA2826DB00200880206820F4800000F580002060002012494880BDF80800888041
:20FBE000BDF80A00C8800846F7F790FC00200D4908700D480089401C0B49088102200B49BB
:20FC0000087006E000200549088002E0002003490880BDE8FF810000A0020020A40200200D
:20FC200090070020A5030020300B0020C601002070B504460E461546FAF704FE41F2883106
:20FC4000884201D35A2C08DDFAF7FCFD31490860FAF7F8FD2F49086070BD2888C0F3402019
:20FC6000002855D1052C01DBBE2C22DDFAF7EAFD28490968401A41F2883188421DD92868F0
:20FC800020F4007000F50070286001202249488008468480C680F7F739FC00201F490870E4
:20FCA0001F48408B401C1E49488301201D490870D2E7FAF7C7FD17490860052E01DBBE2E54
:20FCC00022DDFAF7BFFD18490968401A41F2883188421DD9286820F4007000F5007028609F
:20FCE00002200D49488008468480C680F7F70EFC00200A4908700A48408B401C08494883B4
:20FD0000012008490870A7E7FAF79CFD0649086000BFA1E74802002090070020A5030020FA
:20FD2000000B0020C60100204C0200200FB42DE9F04105460E4617460B9C2088C0F300201B
:20FD4000002877D1012D76D141F28830864272DDB7F5FA7FFBDDBDF92400002801DB01469A
:20FD600000E04142B1F5967F2CDAFAF76BFD58490968401A41F28831884227D9206820F448
:20FD8000807000F580702060012052494880BDF92400002801DB014600E041424D4A91805A
:20FDA0001046F7F7B3FB00204B4908704B48008B401C4A490883012049490870BDE8F001CC
:20FDC0005DF814FBFAF73EFD41490860BDF92600002801DB014600E04142B1F5967F2BDA57
:20FDE000FAF730FD3F490968401A41F28831884226D9206820F4807000F5807020600220CA
:20FE000034494880BDF92600002801DB014600E04142304A91801046F7F778FB00202E493A
:20FE200008702E48008B401C2C49088301202C490870C3E73CE03CE0FAF704FD2949086031
:20FE4000BDF92800002801DB014600E04142B1F5967F29DAFAF7F6FC23490968401A41F20B
:20FE60008831884231D9206820F4807000F580702060032017494880BDF92800002801DBD7
:20FE8000014600E04142134A91801046F7F73EFB0020114908701148008B401C0F490883B8
:20FEA00001200F49087089E7FAF7CCFC0E4908600BE0FAF7C7FC06490860FAF7C3FC094911
:20FEC0000860FAF7BFFC0849086000BF76E700003C02002090070020A5030020000B002031
:20FEE000C601002040020020440200202DE9FF410646DDE90A870C9C00252078C0F34010F2
:20FF0000002878D1052F08D1FAF79CFC3B490860FAF798FC3A4908606DE0012F01D0042FFD
:20FF200032D1B8F1320F2ADD4EBB364890FBF8F085B242F21070854200DA00E028460546AE
:20FF4000FAF780FC2D490968401AA84253D9206820F020002030206001202B4948800846AA
:20FF6000F7F7D4FA0020294908702948408A401C27494882012027490870BDE8FF81FAF7CB
:20FF800061FC1E49086036E09DF8040005282EDB9DF8050058BB56BB9DF804001E4991FB06
:20FFA000F0F085B242F21070854200DA00E028460546FAF747FC12490968401AA8421AD905
:20FFC000206820F020002030206002200E4948800846F7F79BFA00200C4908700C48408A7C
:20FFE000401C0B49488201200A490870C5E7FAF729FC0349086000BFBFE70000240200207A
:020000040801F1
:200000002802002048F13E0090070020A5030020000B0020C6010020D8B805000FB42DE920
:20002000F04104460F46DDE90B85FAF70BFC41F28831884207D350480078012803D04E4870
:200040000078022807D1FAF7FDFB4C490860FAF7F9FB4B490860FAF7F5FB4A490968401A20
:2000600014287DD3FAF7EEFB46490860002607E04549701C31F8100021F81600701C86B2D0
:20008000182EF5D3404804862878C0F3801000286FD119213C48F8F7E1F93C490860222F30
:2000A00037D007F00F0098B39DF820001E2830DD9DF8210060BBB8F1020F2AD108460068A4
:2000C0000A2826D2FAF7BEFB2C490968401A43F69821884221D9286820F04000403028607E
:2000E00001202B4948802948008888800846F7F70DFA0020274908702748808A401C264913
:200100008882012025490870BDE8F0015DF814FBFFE7FAF797FB19490860322C03DB40F62F
:20012000D270844221DDFAF78DFB15490968401AB0F57A7F1DD9286820F0400040302860AB
:2001400002201349488008468480F7F7DFF90020104908701048808A401C0F49888200E050
:2001600007E001200D490870CEE7FAF76BFB0449086000BFC8E70000D80000202C02002034
:200180003002002038020020A01200203402002090070020A5030020000B0020C6010020FA
:2001A00010B50C49487B01F0D1FC0A49487B05F0C9FA094803F060FC0748F5F75BFC074855
:2001C0000189074804F0D4FD01F0C0FE012001F0E9FE10BDB00A0020940100205C1D0020E4
:2001E0006E1500202DE9FF410E4615461F461D48006850BB25B3012F22D1FAF723FB40F6DA
:20020000B83188421CD9C82E0BDD9DF80000552807D09DF80000F82801D1012411E00424AA
:200220000FE0642E0DDA222D01D1012409E005F0F00018B1332D01D0032402E0022400E039
:200240000524012001F0AEFE08E0052400200649087008460078C04304490870204604B017
:20026000BDE8F08194010020DA000020DC00002010B502464FF480630AB9184610BD022971
:2002800002DC4FF480731FE0062906DC881E4FF4807404EB801083B216E0162908DC881FE9
:2002A00000EB40004FF4007404EBC00083B20BE01E2907DCA1F116004FF4607404EB0010A5
:2002C00083B201E04FF480631846D7E710B502464FF480630AB9184610BD022902DC4FF459
:2002E00000731FE0062906DC881E4FF4007404EB401083B216E0162908DC881F00EB80007F
:200300004FF4207404EB800083B20BE01E2907DCA1F116004FF4707404EBC00083B201E0B9
:200320004FF480631846D7E710B50446207838B9F7F78AF8FBF7EAFFF7F71EFA01202070E1
:2003400010BD10B5044601F021FFF7F703FAFEF745FD0020207010BD2DE9F04107460D462A
:20036000144605EB4500C0F34F06207800F0010050BBB74203DAFAF765FA1C490860FAF76E
:2003800061FA1A490968401A41F2883188422AD9206820F00100401C20600220144948805F
:2003A00008468680F7F7B2F800201249087012480089401C10490881012010490870FAF75A
:2003C00041FA0F4908600EE0FAF73CFA0C490968401A41F28831884205D90A48006820F08F
:2003E000010008490860BDE8F08100001003002090070020A5030020000B0020C601002069
:2004000014030020940100201CB52C492C48808BC0F30B0010B940F6B83001E02848808B2A
:20042000284CCDE90001237B274C247814B9274C248801E0264CE4882246254CE17B224C96
:20044000207800F0FFF92248008941F2883188420DDA1C4A117B2246127812B91B4A1288DE
:2004600001E01B4AD2881046144A00F0FFF8194A917A174A1089114A00F060F90F48104C82
:200480000090A37A124CA27D617DE07D00F04EF822461189D088094A00F0ACFA084A127AA0
:2004A00002EB4203C3EBC2124FF6FF7303EAC20122461089014AFFF74FFF1CBD9401002003
:2004C000B00A0020F00A0020F40100207C090020DC080020D007002070B504460D46207819
:2004E00068B900200F4908700F480078C0B90E480078401C0C490870F6F78CFF10E0002024
:200500000949087007480078012802DB0020207001E0F6F7D1FC03480078401C0149087018
:2005200070BD000018030020190300202DE9F04180460E4617461C46069DFAF783F940F6B1
:20054000B831884207D2FAF77DF940490860FAF779F93F4908602878C0F3001000283DD1CB
:200560003C48C07A58B9A4F11900B04215DD2330874212DAFAF766F9344908600DE0A4F15B
:200580001900B04209DD2330874206DA1E38404503DDFAF757F92D490860FAF753F92B49E3
:2005A0000968401A41F2883188424CD9FAF74AF927490860286820F01000103028602648A3
:2005C000F6F7A4FF0020254908702548008A401C2349088201202349087034E01D48C07A84
:2005E000B8B9A4F12300B0422DDD0F30B8422ADDFAF728F916490968401A1B49884222D931
:20060000286820F010002860FAF71CF90F49086019E0A4F12D00B04215DD1930B84212DD0B
:200620000A3840450FDDFAF70DF909490968401A0D49884207D9286820F010002860FAF7CA
:2006400001F902490860BDE8F08100000003002004030020D007002090070020A503002017
:20066000000B0020C6010020E09304002DE9F04105460E4614460027182E04D0242E05D049
:20068000302E09D105E047F60C3707E04AF6C87704E04EF2844701E02F4600BF00BF2078FC
:2006A000C0F3800030BBBD4203DCFAF7CBF81D490860FAF7C7F81B490968401A41F28831F1
:2006C000884212D9206820F00400001D20601648F6F71CFF00201549087015488089401C0E
:2006E00013498881012013490870FAF7ABF81249086014E0A7F5FA70A84203DAFAF7A2F8FD
:200700000D490860FAF79EF80B490968401A41F28831884203D9206820F004002060BDE822
:20072000F0810000EC02002090070020A5030020000B0020C6010020F002002070B5054627
:200740000E4614462078C0F3C000002849D1012E08D1FAF777F831490860FAF773F830497F
:20076000086014E040F6C410854208DAFAF76AF82A490860FAF766F82949086007E041F6F5
:200780004C50854203DAFAF75DF825490860FAF759F822490968401A41F28831884208D8EF
:2007A000FAF750F81E490968401A40F6B831884232D9206820F00800083020601948F6F734
:2007C000A5FE0020184908701848C089401C1749C881012016490870FAF734F815490860F4
:2007E0001AE0FAF72FF813490968401A41F28831884211D91048007870B9104800880A2815
:200800000ADA0E4840880A2806DA0D48807818B9206820F00800206070BD0000F402002043
:20082000F802002090070020A5030020000B0020C6010020FC020020DA0000202A050020A6
:20084000C40300202DE9F0478046894615469A46DDE9086400270120B0EBE63F4ED12078A3
:20086000C0F34000A0BBB9F1010F03DBF9F7EAFF5A490860F9F7E6FF58490968401AC6F3B4
:20088000023101EB8101052202EB410101EB4102C2EBC111B0EBC10F15D9206820F00200C0
:2008A000801C20604E484580A0F80480F6F72EFE00204C4908704C484089401C4A4948814A
:2008C00001204A490870F9F7BDFF4949086082E0FFE7B9F1050F03DAF9F7B4FF44490860CB
:2008E000F9F7B0FF42490968401A41F28831884271D9206820F0020020606CE0BAF1180FCB
:2009000006D0BAF1240F08D0BAF1300F12D10AE0C6F30B00C0EBC0070EE0C6F30B0000EBC1
:200920008000470008E0C6F30B0000EB800101EBC00701E02F4600BF00BF2078C0F34000C6
:2009400098BBBD4203DBF9F77DFF24490860F9F779FF22490968401AC6F3023101EB81012E
:20096000052202EB410101EB4102C2EBC111B0EBC10F15D9206820F00200801C2060184804
:200980004580A0F80480F6F7C1FD00201549087015484089401C1449488101201349087038
:2009A000F9F750FF1249086015E0FFE707F57A70854203DAF9F746FF0D490860F9F742FFAC
:2009C0000B490968401A41F28831884203D9206820F002002060BDE8F0870000E40200202A
:2009E00090070020A5030020000B0020C6010020E80200202DE9F04107468846144600267A
:200A0000F9F720FF2B490968401A642850D3002507E02949681C31F8100021F81500681CEC
:200A200085B2092DF5D3244847820A21F7F716FD06462068C0F3404090BBB8F1320F2BDADF
:200A4000B6F57A7F28D91D480078322830DD206820F4003000F500302060C6F30F201849F3
:200A600048800A211448F7F76DFC154988800A211148F7F778FC1249C8800846F6F746FD63
:200A800000201049087010480089401C0E49088102200E4908700BE000200849087007E09C
:200AA000FFE7B6F57A7F03D8206820F400302060BDE8F08108030020480700200C030020A6
:200AC00090070020A5030020300B0020C601002010B5F9F7B7FEA2490968401AC8287DD3F5
:200AE000F9F7B0FE9E4908609E480088C01268B99D480089FA2148439C49097A4FF47A72FD
:200B00005143B0FBF1F09849888016E095480088C0F30A0093490988012202EBE1214843AA
:200B200040119149098948439049097A4FF47A725143B0FBF1F08C4988808B4880881428CE
:200B400001DA002001E08848808887498880884840780873874800881C2190FBF1F082493B
:200B6000C8728548007848738348407888738348007800F0010040B17A48037B0846C27BCD
:200B80007F498048F3F752FE01E07F48407A7649C8737A48007800F0010010B14EF6EE60B1
:200BA00001E07A48C08A704908827048807EEE2815D177488078012823D1754880684FF497
:200BC0004821B1FBF0F07349096808447149086008460068000B6E49C86012E0BFE06348A9
:200BE000807EAA280DD1624840686049897948435E49C979B0FBF1F03221B0FBF1F06449BE
:200C0000C8605A48007B594991F91B10084442F2107191FBF0F15E48C0685F4A1268801A3F
:200C2000814206D801205D4908705948C0685A4908605A48007801283ED100205749087076
:200C400057480068401C564908605648406A401C5449486252488068401C51498860084691
:200C600080685149884203D900204D498860C8603D48008B401C3C490883494800680A21E6
:200C8000B0FBF1F03849488248480078401C47490870084600781E280EDB424B30224C21D0
:200CA000434803F07CF83E4B1022D621404803F076F800203D4908702B4800881E281ADB53
:200CC0003C480078401C3B49087008460078052814DB0020087038480088401C36490880DB
:200CE0002148408B401C2049488334480078401C3249087002E000202E4908702F4800780D
:200D00003C2811DB00202D49087025484068401C234948602348C06A401C2249C862204802
:200D2000C068401C1E49C86023480088B0F5167F0EDB0020204908801A4B30224C211C48F1
:200D400003F02DF8164B1022D621194803F027F80E48808A0A2190FBF1F00349087510BDF1
:200D60006C000020F00A0020DC080020B00A0020C40300202A050020DA000020B8010020E6
:200D8000B40900203C0300207C0900201C030020F40300207C00002070000020740000205C
:200DA0002C0C0020000B00209F8601008000002034040020750000207800002076000020CF
:200DC00010B50446F9F73EFD10490968401A4EF66021884218D3F9F735FD0C4908602068D4
:200DE000401C20600A480078401C09490870084600780A2808DB074B30224C21064802F0FB
:200E0000CEFF00200249087010BD0000C0000020C4000020000B00203404002010B50446FF
:200E2000022C1BD1F9F70EFD0F490968401AC82818D30E4B4FF481520C214FF4E26003F08B
:200E40004DF80B4B4BF620220C2140F2157003F045F8F9F7F7FC0449086003E0F9F7F2FC07
:200E60000149086010BD000090000020DC080020FC08002001B511480078022800D108BDD4
:200E80000098A0B1F9F7DEFC0D490968401AB0F5FA7F10D9F9F7D6FC094908606B4641F217
:200EA00004120C214FF4E26003F018F803E0F9F7C9FC0349086000BFE1E700005D00002017
:200EC0008800002010B50446012C13D1F9F7BAFC0B490968401AC82810D30A4B4FF4815247
:200EE0000C214FF4E26002F0F9FFF9F7ABFC0449086003E0F9F7A6FC0149086010BD000016
:200F00008C000020DC08002010B5FBF711FAFBF7FDF9F4F76BF903F06DF9FBF7E3FC0548B1
:200F20000189054803F06CFF024881890348F6F785FE10BD5C1D00206E1500207C040020C4
:200F40001CB50446F9F77EFC40490968401AB0F5FA7F7AD33E480088401C3D490880084687
:200F60000088142837DB3B48007800F0010010B900203949487437480088C0F3002010B9E5
:200F800000203549087433480078C0F3801010B90020314908812F480078C0F3C01010B9DA
:200FA00000202D4948812B480078C0F3001010B900202949888127480078C0F3401010B90D
:200FC00000202549C8814FF480512448F9F730FC00201F4908802248007868B900204FF428
:200FE00008430C2240F2FF7100901E4802F0C2FF01201B49087024E019480078012820D139
:2010000000200190184801780078401C164A107005290CDC01A841F20133162240F2FF7192
:201020000090104802F0A6FF0A20F9F725F941F214030C2240F2FF710A48009402F09AFF6E
:2010400000BFF9F7FFFB014908601CBD9C000020A0000020D0010020D00B002000100140A3
:201060005D000020F8050020A200002070B504464D48007880BB08214C48F9F7D1FB4C494F
:2010800008704FF400414B48F9F7CAFB4A49087080214A48F9F7C4FB494908704FF48071E1
:2010A0004648F9F7BDFB474908704FF400514348F9F7B6FB4449087004214448F9F7B0FBE1
:2010C00043490870002020816081A081E081207460740120344908703E48C08860803D4837
:2010E0008088A0804FF40060E0803A480089208008212E48F9F794FB05462D480078A842DA
:2011000002D02089401C2081294805704FF400412848F9F785FB054627480078A84202D01F
:201120006089401C60812448057080212348F9F777FB054622480078A84202D0A089401CCC
:20114000A0811F4805704FF480711C48F9F768FB05461C480078A84202D0E089401CE0819E
:20116000184805704FF400511448F9F759FB054615480078A84202D0207C401C20741248A4
:20118000057004211148F9F74BFB054610480078A84202D0607C401C60740D4805704FF436
:2011A0007A70608270BD00009A000020000C0140940000200008014095000020001001402C
:2011C00096000020970000209800002000140140990000206E1D002010B5F9F733FB42F21A
:2011E0001071884204D2F9F72DFB4149086010BDF9F728FB3E490968401A41F288318842DC
:2012000074D3F9F71FFB3A4908603A48407D3A4991F82310884207DA3648407D364981F836
:2012200023000020354908703248407D324991F82210884207DD2F48407D2F4981F8220013
:2012400000202E4908702B48807D2B4991F82910884207DA2748807D274981F82900002090
:20126000264908702348807D234991F82810884207DD2048807D204981F8280000201F494D
:2012800008701C48C07D1C4991F82B10884207DA1848C07D184981F82B00002017490870C7
:2012A0001448C07D144991F82A10884207DD1148C07D114981F82A000020104908701048EB
:2012C0000088401C0E490880084600880C280DDD0A48007850B900200880012007490870F3
:2012E000054B30224C21074802F059FD00BF7EE7C8000020DC080020000B0020CE0000201F
:20130000CC0000203404002010B50748007850B9F9F798FA04494968401AB0F5FA6F02D931
:2013200001200149087010BDDC01002000B587B0012003900320049003A90E48F9F7E2F8DD
:201340000D480068806820F001000B4909688860002000900820019007200290694606480B
:20136000F7F732FB20B140F29D2104A004F046FF07B000BD00080140801D00202E2E5C433F
:201380006F72655C5372635C6164632E630000000EB550485049086081154F4881600021E3
:2013A000C16041614FF46021C16100204A494860092149480161F7F71DFE18B1592147A0D9
:2013C00004F01CFF0A200090012001900720029069464148F7F7F8FA18B163213FA004F0A1
:2013E0000DFF0B200090022001900720029069463948F7F7E9FA18B16D2138A004F0FEFE9A
:201400000C200090032001900720029069463248F7F7DAFA18B1772130A004F0EFFE0D2079
:201420000090042001900120029069462A48F7F7CBFA18B1812129A004F0E0FE0520009025
:2014400001900120029069462348F7F7BDFA18B18B2122A004F0D2FE072000900620019020
:201460000720029069461C48F7F7AEFA18B195211AA004F0C3FE0E20009007200190012085
:20148000029069461448F7F79FFA18B19F2113A004F0B4FE10200090082001900220029019
:2014A00069460D48F7F790FA18B1A9210BA004F0A5FE1120009009200190072002906946F8
:2014C0000548F7F781FA18B1B32104A004F096FE0EBD000000240140801D00202E2E5C43A5
:2014E0006F72655C5372635C6164632E6300000000B589B0234824490860811522488160FE
:201500000021C1604161C16100201F49486001211D480161F7F76EFD18B1C7211BA004F0F3
:201520006DFE01200190029003200590002003904FF480500890002007900690049001A95B
:201540001148F7F737F818B1D62110A004F056FE02200190029001A90B48F7F72BF818B141
:20156000DF210AA004F04AFE03200190029001A90548F7F71FF818B1E82104A004F03EFE9D
:2015800009B000BD00280140B01D00202E2E5C436F72655C5372635C6164632E63000000A5
:2015A00010B50F480F4908601220486000210D488160C1604FF4A0210161002141618161F2
:2015C0000121C1610021016241628162C162F8F757F918B15C2104A004F010FE10BD0000A2
:2015E00000640040B42200202E2E5C436F72655C5372635C63616E2E6300000008B500BFF1
:201600000A48406940F00100084948610846406900F00100009000BF00BF022211460B2008
:20162000F9F7DFF90B20F9F7CFF908BD0010024000B585B000BF3A48806940F01000384913
:2016400088610846806900F01000009000BF00BF00BF0846806940F02000886108468069F6
:2016600000F02000009000BF00BF00BF0846806940F0040088610846806900F0040000907E
:2016800000BF00BF00BF0846806940F0080088610846806900F00800009000BF00BF002256
:2016A00089142048F9F7C8F84EF2203001900320029001A91B48F8F725FF40F61870019030
:2016C0000320029001A91848F8F71CFF4EF6024001900320029001A91448F8F713FF4FF42B
:2016E00080500190124802900020039001A90F48F8F708FF4FF4805001900120029002207A
:20170000049001A90748F8F7FDFE002211462820F9F767F92820F9F757F905B000BD000047
:20172000001002400010014000080140000C01400000211010B508480849086003204860A6
:2017400040F2E24105488160F9F782F818B13A2103A004F053FD10BD003000400408002028
:201760002E2E5C436F72655C5372635C697764672E63000000B595B0314832490860002096
:20178000486020212F4881604FF41661C1600021016101214161F9F7FFFF4FF48050119044
:2017A00011A92848FAF7A0F82648FAF7D1FA70200F90802010900FA92248F9F776FF4FF413
:2017C000006008904010099000200A9039200B9000200C900D900E9008A91A48F9F726FF5B
:2017E0006FF08000174909680861602001904FF496600290002003900490059006900790EB
:20180000002201A90F48FAF71FFA042201A90D48FAF71AFA082201A90A48FAF715FA6020CB
:20182000019040F65F10029000200390082004900C2201A90348FAF707FA15B000BD0000DA
:20184000002C01409C1C002000B587B000200390049005900690019002904FF08040194961
:201860000860002048600021164881604FF6FF71C1600021016141618161F9F78DFF18B1B6
:201880007E2111A004F0BAFC4FF400500390002004900590069003A90A48FAF725F818B174
:2018A000862109A004F0AAFC00200190029001A90448F9F7FAFE18B18C2103A004F09EFC76
:2018C00007B000BDDC1C00202E2E5C557365725C5372635C74696D2E6300000000B589B07C
:2018E0001C481D4908600020486000211A4881604721C1600021016180218161FAF728FAE8
:2019000020B14FF48F7115A004F078FC00200790089007A91048F9F7C8FE20B140F2251150
:201920000EA004F06BFC6020009024200190002002900490002269460748FAF785F920B113
:201940004FF4977105A004F059FC0348FAF732F909B000BD000400401C1D00202E2E5C55C7
:201960007365725C5372635C74696D2E6300000010B50C480C4908604FF41650486000211A
:2019800009488160C16001610C21416100218161C161FAF71BFC18B1462104A004F02EFCA4
:2019A00010BD000000480040F82400202E2E5C436F72655C5372635C75736172742E6300B5
:2019C00000BFFEE730B504460A460021002329480078401C274D2870284600780F2841DB16
:2019E0000020287024480089244D2D88411B002907DA214800894FF6FF7528441F4D2D8876
:201A0000411B44F62060814200DD00211A4800891A4D28804FF47A70414319480068081A59
:201A2000174D2D6805EB2020154D2860284600680314C3EB031040F35C0000B2114D28809E
:201A40000D488089104D2D68C5EB80200E4D2D6805EB60100C4D286028460068C0F38F207D
:201A6000054DE88112B90020064D28800548B0F9000030BDB2030020D0070020B40300203F
:201A8000B8030020C0030020BC0300202DE9F04107460C46154629462046F6F7C9FB80461C
:201AA000002606E0701C34F8100024F81600701C86B2681EB042F5DC24F810704046BDE84C
:201AC000F081704702480068C0F30220704700000CED00E010B5002807DA0A07140E054A77
:201AE00000F00F031B1FD45403E00A07130E024A135410BD18ED00E000E400E010B5F8F790
:201B0000A1FE40F6B831884216D90C480078012812D10020094908700948C07AAA280BD153
:201B200033200849087008460078C0430649087004484078C043487010BD0000CF0000207E
:201B4000B00A0020DA000020DC00002010B50446012C06D0022C23D0032C40D0042C7DD1C5
:201B60005CE024224E494F48F1F799FF24224E494E48F1F794FF24224D494E48F1F78FFF5F
:201B800024224D494D48F1F78AFF24224C494D48F1F785FF24224C494C48F1F780FF7CE055
:201BA00024224B493F48F1F77AFF242249493F48F1F775FF242248493E48F1F770FF2422AE
:201BC00046493E48F1F76BFF242245493D48F1F766FF242243493D48F1F761FF5DE02422D6
:201BE00041493048F1F75BFF242240492F48F1F756FF24223E492F48F1F751FF24223D49D6
:201C00002E48F1F74CFF24223B492E48F1F747FF24223A492D48F1F742FF3EE02422384961
:201C20002048F1F73CFF242236492048F1F737FF242235491F48F1F732FF242233491F4861
:201C4000F1F72DFF242232491E48F1F728FF242230491E48F1F723FF1FE0FFE72422104987
:201C60001048F1F71CFF24220F491048F1F717FF24220F490F48F1F712FF24220E490F4833
:201C8000F1F70DFF24220E490E48F1F708FF24220D490E48F1F703FF00BF00BF10BD000047
:201CA000D86C01084C060020FC6C010870060020206D010894060020446D0108B806002076
:201CC000686D0108DC0600208C6D010800070020B06D0108D46D0108F86D01081C6E01088A
:201CE000406E0108646E0108886E0108AC6E0108D06E0108F46E0108186F01083C6F01083A
:201D0000606F0108846F0108A86F0108CC6F0108F06F0108147001082DE9F04304460D46B0
:201D2000601B06B2B2F9000000FB06FC908810B90020106212E0B2F9040000FB06F7106A42
:201D4000C319D069984202DAD069106206E09069984202DD9069106200E0136250889CFB46
:201D6000F0F0B2F80690D2F8208098FBF9F800EB0801002906DA1069884203DD108A00B2E9
:201D8000BDE8F083002905DD5069884202DC908A00B2F5E708B2F3E72DE9F34F83B00C46A6
:201DA000204603F069F800901D4800990160BDF90C001B49B1F9001000FB01F7FF13BDF9DF
:201DC0000E001749B1F9021000FB01F84FEAE8380FFA87FB0FFA88F001900198ABEB0000C0
:201DE00000B2ADF80800BDF90C000D49B1F9021000FB01F5ED13BDF90E000949B1F90010EF
:201E000000FB01F6F6130FFA85F90FFA86FA09EB0A0000B2ADF80A00029805B0BDE8F08FE5
:201E20004C0000207047000030B50246B2F900303F4CB4F90040A34202DD13883C4C238075
:201E4000B2F902303B4CB4F90040A34202DD5388384C2380B2F90430374CB4F90040A34237
:201E600002DD9388344C2380344B1B885B1C1BB2324C23802346B3F90030B3F5FA7F56DB27
:201E80002B4BB3F900000023294C2380031E01DB1C4600E05C42B5256C43294D2D68C5EBC4
:201EA0008404274D2D6805EB6414254D2C602B461B689B121BB20B801E4BB3F900000023FA
:201EC0001C4C2380031E01DB1C4600E05C42B5256C431C4D2D68C5EB84041A4D2D6805EB6F
:201EE0006414184D2C602B461B689B121BB24B80114BB3F9000000230F4C2380031E01DB1A
:201F00001C4600E05C42B5256C430F4D2D68C5EB84040D4D2D6805EB64140B4D2C602B4683
:201F20001B689B121BB28B800023044C238030BD7405002076050020780500207A05002026
:201F40007C050020800500208405002000B585B000BF1148806940F004000F4988610846E4
:201F6000806900F00400009000BF00BF002289140A48F8F761FC4FF48050019001200290C2
:201F80000220049001A90548F8F7BCFA00200449087005B000BD00000010024000080140FD
:201FA0007A04002010B50446012C0BD10C480078A8B9012211030B48F8F73EFC0120084919
:201FC00008700CE05CB906480078012807D1002201030448F8F730FC00200149087010BD85
:201FE0007A0400200008014010B5044619480078012816D1B4F5D16F0FDB17480088401CEC
:2020000080B21549088047F23051884220DD0020114908800F4908701AE000200E4908805C
:2020200016E0B4F5BC6F10DA0C480088401C80B20A4908803C280BDDF4F73EFF01200549C4
:20204000087000200649087002E000200349088010BD00008C050020880500208A05002071
:202060000B02002038B50446002034490870F020487008460078C043314908702F48407835
:20208000C04348702D4840782E4B0090DA79997958792D4B1B78FAF761FD2C48007810BB08
:2020A0002B4800682B4908602948406848602848806888602648C068C8602748406808612A
:2020C0002548406A48612448C06A88612822234801F002FE042222A12048083801F0FCFDA0
:2020E00001201A49087020A341F205320C214FF4E26001F0F3FE04B938BDF8F7A3FB1C497F
:20210000086000201B49087012E0F8F79BFB18490968401A64280BD9F8F794FB1449086005
:2021200014480078401C134908701348F8F7B8FB104800780A28E8DB00BFDDE7DA0000205C
:20214000DC000020D00A002044040020B60000202C0C0020900B0020000B002008E8010814
:20216000464C4147000000005245414459000000B8000020BC0000200408002010B50248E1
:20218000F9F7A3FB10BD00009C1C002010B500210B48F9F731FE04210948F9F72DFE0821FA
:2021A0000748F9F729FE00210548F9F7C5FA04210348F9F7C1FA08210148F9F7BDFA10BD9B
:2021C0009C1C002008B508490968C9084FF47A72B1FBF2F14143009100BF00BF00994A1E85
:2021E00000920029F9D108BD000000202DE9F04705460E4617469846F8F724FB8449096802
:20220000401A052801D2BDE8F087F8F71BFB804908600FFA88F07F4948807F480088281A70
:20222000C8810846007801287ED1F8F70BFB7949C969401AB0F5FA6F06D9F8F703FB75493C
:20224000C8610120887601E0744886607148407E01281BD100206F494876002405E0002068
:202260006F4921F81400601CC4B2192CF7DB00206C4908806C4908606C4908706548408A52
:2022800020B16448408A0002694908606148C0890A2849DB604805605E48807E00286FD17A
:2022A0005E4886600774C068002869D05B4880895A490989401A00B25E4908800846B0F97B
:2022C0000000002803DD0846B0F9000000E00020584908800846B0F900001E2803DA08466E
:2022E000B0F9000000E01E20524908800846008818B94A48007C642842D0494849490988ED
:2023000030F8110048490968081A47490860084600684849B1F9001008444349086045489A
:20232000008881B23F4800E06FE002880088401C3C4B18803A4820F81210184600881928BC
:2023400007DB002019460880012038490870314908763548006840B334480078012810D1AC
:20236000314800684FF47A7148436421484329498989FA225143B0FBF1F02649088217E003
:202380003FE02848008800EB80004100214880894143254800684FF47A72504364225043D4
:2023A000B0FBF1F01B49088202E00020194908821C480088A0B91748B0F810901C480068FD
:2023C000C0EB09201E2190FBF1F01949096808441749086008460068C0F30F200D494882DF
:2023E0000C48408A002808DD0C4880680949898AB0FBF1F00749C88203E04FF6FF70054906
:20240000C882064880680549C86000BFFBE60000800300201C030020840300203C0300203E
:202420005C0700207003002074030020780300207C0300207A0300202DE9F04104460D4634
:2024400017469846069E00201349086088601348008848600020C8600DB9084686600020E4
:202460000F49087048800520888000208860084684810020C881088248824FF6FF70C88281
:2024800000200876487601208876F8F7DBF90449C861BDE8F08100003C030020B409002036
:2024A0001C0300202DE9F04106460F4606F00F0000287DD0052FFCD001206F4908700846DC
:2024C000007E012864D1002008760846408A6B49098888425CD06848408A002854D06648BB
:2024E000408A67490988401A642100FB01F56448008895FBF0F004B214F11E0F44DBB4F5AD
:20250000E47F41DA04F164005D4909884843642190FBF1F0584988825A48058804F16400FE
:202520006843642190FBF1F0574908805548458804F164006843642190FBF1F05249488015
:202540005048858804F164006843642190FBF1F04D4988804B48C58804F1640068436421DA
:2025600090FBF1F04849C8804648058904F164006843642190FBF1F0434908810B4610226D
:20258000A221424801F00BFC3B48408A3B4908803F480078864203D13E480078874265D006
:2025A000032E1DD005DC012E08D0022E33D10EE054E0042E1DD0332E2DD123E0324800883C
:2025C0002D4948822F4800882D49088029E02E484088294948822B4840882949088020E006
:2025E0002948808824494882264880882449088017E02548C088204948822248C0882049C6
:2026000008800EE0204800891B4948821D4800891B49088005E00020174948821849088033
:2026200000BF00BF1448408A144908801248408A114988820846408A002807DD164880681F
:20264000898AB0FBF1F00C49C88203E04FF6FF700949C88201200849487607E00020064983
:202660000870488288824FF6FF70C8820848067008480770BDE8F0811C0300208A03002081
:202680008C030020687401083C0C00203404002088030020890300203C0300202DE9F047E3
:2026A000074689461546AD10002414E057F82460300E144A02F82400C6F30741A000401C44
:2026C0001154C6F30721A000801C1154A000C01C1654601CC4B2AC42E8DB57F825A0A100D5
:2026E0000848F2F767FD8046BAEB080007D1AA0004494846F1F7D3F90020BDE8F0874FF03E
:20270000FF30FAE7FC15002010B5B0F900205243B0F9023003FB03210C4A914214D9091623
:202720003939CBB20A4C34F81320B0F9003003FB02F1CB131BB20380B0F9023003FB02F131
:20274000CB131BB2438000BF10BD0000400AC139387001082DE9F14181B0BDF90400DFF880
:202760006880B8F9008000FB08F1C913BDF90600DFF85480B8F9028000FB08F2D2130EB23C
:2027800017B2F01900B2ADF80000BDF90400DFF83880B8F9028000FB08F3DB13BDF90600F4
:2027A000DFF82480B8F9008000FB08F4E4130FFA83FC25B2CCF10000284400B2ADF802009E
:2027C0000098BDE8FC8100004C00002010B504462078012808D10B4B30224C210A4801F0D2
:2027E000DEFA002020700AE02078022807D1074B1022EC21044801F0D2FA00202070002063
:2028000010BD0000000B002034040020300B00204FF055301F4A106040001F4A10601D48F2
:202820000168B1F1553F01D0002070471A480168B1F1AA3F01D00020F7E74FF0AA30154AB4
:2028400010604008144A106012480168B1F1AA3F01D00020E9E710480168B1F1553F01D01B
:202860000020E2E74FF055300A4A106040000A4A106008480168B1F1553F01D00020D4E748
:2028800005480168B1F1AA3F01D00020CDE70120CBE70000000800201008002001200C49A9
:2028A0000968B1F1EE3F00D0002009494968B1F1CC3F00D0002006498968B1F1BB3F00D09C
:2028C00000200349C968B1F1DD3F00D0002070478029002010B5214800780D282FD2DFE88A
:2028E00000F0070A0D101316191C1F2225282B00F0F764FC24E0F0F795FC21E0F0F7D1FC2B
:202900001EE0F0F713FD1BE0F0F756FD18E0F0F79AFD15E0F0F7DEFD12E0F0F722FE0FE078
:20292000F0F767FE0CE0F0F7ADFE09E0F0F7EEFE06E0F0F72FFF03E0F0F770FF00E000BF3E
:2029400000BF06480078401C04490870084600780C2801DD0020087010BD00000806002066
:2029600010B5F0F72BFCF0F75DFCF0F79AFCF0F7DDFCF0F721FDF0F766FDF0F7ABFDF0F742
:20298000F0FDF0F736FEF0F77DFEF0F7BFFEF0F701FFF0F743FF10BD10B53B480068B0F1FB
:2029A000AA3F70D138480068384909684840401C002866D136490860C04336490860344883
:2029C0000068801C32490860FFF784FF31480068801E304908602E4800680D302C4908603F
:2029E000FFF75CFF08B9F4F7E7FF2A4800680D3828490860264800680B302549086000F025
:202A0000C5FC044634B1012C0AD0032C04D0042C05D100E007E006E0F4F7CEFF03E000BFAF
:202A2000F4F7CAFF00BF00BF1A4800680B381949086017480068C01C1549086000F044F8F8
:202A400008B9F4F7B9FF13480068C01E114908600F480068401D0E490860FFF7D9FE08B946
:202A6000F4F7AAFF0B480068401F0A490860222003F064FD08B9F4F79FFF0020024908603A
:202A800001E0F4F799FF10BD482500206C250020382500205C25002010B500F047FC00F0C1
:202AA00055FC00F001F810BD4FF0EE30054908604FF0CC3048604FF0BB3088604010C8608F
:202AC0007047000080290020F0B55527552F01D00020F0BDAA27AA2F01D00020F9E74FF079
:202AE0005531B1F1553F01D00020F2E74FF0AA31B1F1AA3F01D00020EBE74FF47A714A0070
:202B00008C1840F6B830844201D00020E1E74FF0FF3102228C18012C01D00020D9E74FF41C
:202B20007A73F94D5E1916F57A7F01D00020D0E76FF0004301255E19B6F1004F01D0002019
:202B4000C7E76FF0004302255E19981C864201D00020BEE76FF0004303255E19D81C864278
:202B600001D00020B5E74FF4FA614A108C1AB4F57A7F01D00020ACE74FF4FA614A1C8C1A5A
:202B8000601C08B10020A4E7002101228C1A601C08B100209DE74FF47A735D005E1B16F581
:202BA0007A7F01D0002094E7002301255E1B701C08B100208DE74FF0004301255E1B581E7E
:202BC000864201D0002084E74FF47A71491C0846814201D000207CE74FF0FF31491C09B14B
:202BE000002076E70021491C012901D0002070E74FF47A735B1C1846834201D0002068E756
:202C000000235B1C012B01D0002062E76FF000435B1CB3F1004F01D000205AE74FF00043F4
:202C20005B1C1846834201D0002052E74FF47A71491E0846814201D000204AE70021491E80
:202C4000481C00B145E74FF0FF31491E881C00B13FE74FF47A735B1E1846834201D0002025
:202C600037E74FF000435B1E1846834201D000202FE76FF000435B1E1846834201D00020E2
:202C800027E700235B1E581C00B122E764210A2201FB02F4B4F57A7F01D0002019E76FF0C7
:202CA0007041112201FB02F49848844201D000200FE74FF0FF31012201FB02F4601C08B1F8
:202CC000002006E76421002201FB02F40CB10020FFE64FF47A710A22B1FBF2F4642C01D03F
:202CE0000020F6E601210A22B1FBF2F40CB10020EFE600210A22B1FBF2F40CB10020E8E6BC
:202D00004FF47A710022B1FBF2F40CB10020E0E64FF0FF310122B1FBF2F4601C08B10020B5
:202D2000D7E602214C00042C01D00020D1E602210C02B4F5007F01D00020CAE60221CC079F
:202D40000CB10020C5E64FF6FF714C084810844201D00020BDE64FF6FF710C0AFF2C01D069
:202D60000020B6E64FF6FF71CC0F0CB10020B0E6012109B90020ACE6002109B10020A8E675
:202D8000FF2109B90020A4E664210A22914201D800209EE664216422914201D9002098E650
:202DA0000A216422914201D9002092E64FF0FF310022914201D800208BE66FF00043DD07C9
:202DC000AB4201DC002084E60A216422914201D300207EE664216422914201D2002078E694
:202DE00064210A22914201D2002072E600214A1E914201D300206CE64FF000435D1EAB4278
:202E000001DB002065E664210A22914201D200205FE664216422914201D2002059E60A2174
:202E20006422914201D3002053E64FF0FF310022914201D200204CE66FF00043DD07AB4210
:202E400001DA002045E60A216422914201D900203FE664216422914201D9002039E664212D
:202E60000A22914201D8002033E600214A1E914201D900202DE64FF000435D1EAB4201DD10
:202E8000002026E664216422914201D0002020E64FF0FF310A46914201D0002019E600218E
:202EA0000022914201D0002013E64FF000431D46AB4201D000200CE600230025AB4201D078
:202EC000002006E66FF000431D46AB4201D00020FFE564216422914201D00020F9E54FF033
:202EE000FF310A46914201D00020F2E500210022914201D00020ECE54FF000431D46AB420D
:202F000006D00020E5E5000030F8FFFFEFFFFF0F00230025AB4201D00020DAE56FF0004348
:202F20001D46AB4201D00020D3E50121002221B9022904D0032906D103E0921C04E0121DD4
:202F400002E0083200E000BF00BF022A01D00020BFE502210022012904D0022904D00329C8
:202F600006D103E0921C04E0121D02E0083200E000BF00BF042A01D00020AAE50321002268
:202F8000012904D0022904D0032906D103E0921C04E0121D02E0083200E000BF00BF082AE1
:202FA00001D0002095E504210022012904D0022904D0032906D103E0921C04E0121D02E0D9
:202FC000083200E000BF00BF0AB1002081E50021002211B10AB100207BE501B90AB1002043
:202FE00077E50021012211B10AB1002071E511B90AB900206DE50121012201B10AB9002065
:2030000067E511B90AB9002063E50121FF2201B10AB900205DE511B90AB9002059E5002149
:20302000FF2211B10AB1002053E511B90AB900204FE54FF055310A4681EA02040CB1002056
:2030400047E54FF055314A0081EA0204601C08B100203EE50021002281EA02040CB10020BB
:2030600037E54FF0FF310A4681EA02040CB100202FE500214A1E81EA0204601C08B10020C4
:2030800027E54FF05531CC43B4F1AA3F01D000201FE5E443B4F1553F01D0002019E500215D
:2030A000CC43601C08B1002013E5E4430CB100200FE501200DE5000008B500BF714880698B
:2030C00040F004006F4988610846806900F00400009000BF00BF00BF0846806940F00800B4
:2030E00088610846806900F00800009000BF00BF00BF0846806940F0100088610846806954
:2031000000F01000009000BF00BF00BF0846806940F0200088610846806900F0200000909B
:2031200000BF00BF5848F4F79BFC08B9002008BD5648F4F795FC08B90020F8E75448F4F7E8
:203140008FFC08B90020F2E75248F4F789FC08B90020ECE74B48806920F004004949886161
:203160000846806920F0080088610846806920F0100088610846806920F0200088614648F9
:20318000F1F7C2FA00BF3F48C06940F000703D49C8610846C06900F00070009000BF00BFE8
:2031A0003E48F1F7C1FF08B90020C0E73548C06920F000703349C86100BF0846406940F0A8
:2031C000010048610846406900F00100009000BF00BF3348F2F7DEFC08B90020A7E7294831
:2031E000406920F001002749486100BF0846806940F4007088610846806900F4007000904E
:2032000000BF00BF00BF0846806940F4806088610846806900F48060009000BF00BF2148BB
:20322000F1F78AF908B9002081E71F48F1F784F908B900207BE71348806920F400701149A9
:2032400088610846806920F48060886100BF0846806940F4006088610846806900F4006073
:20326000009000BF00BF114801F089FB08B900205DE70448806920F400600249886101204F
:2032800055E700000010024000080140000C0140001001400014014000000140006400407F
:2032A000080002400024014000280140002C014010B5002419480068194909684840401C20
:2032C00048BB164800681749884210D316490846F0F7DCFA012801D1042400E0032411482B
:2032E0004B380E490860C0430D49086014E00E490A480068F0F7CAFA01280AD10748006860
:2033000010300649086008460068C0430449086002E0032400E00124204610BD3C060020A5
:20332000400600207B0000201C06002004480549086008460068C043034908607047000024
:20334000300000203C0600204006002010B50A480A490860C0430A4908600A480A490860B8
:203360000846F6F7B4FD08480068806840F0010005490968886010BD00300008542500204B
:2033800078250020003002401006002010B502241F4800681F4909684840401C002834D124
:2033A0001B4800681C49884223D2002006E01849096851F82010194A1160401C18498908AB
:2033C000174A9209B1FBF2F18142F0D814498908134A9209B1FBF2F10D4A126802EB810122
:2033E0000B4A116011460968C9430A4A116000240CE00A48006808490968884201D104241E
:2034000000E00324FFF7A2FF00E00124204610BD54250020782500208089010800300240FC
:203420008059010070B50A2050490870F7F74CFA00F0E2FF00204E490860C0434D4908602D
:203440004B480068801C4A490860FFF789FA49480068801E47490860EFF764FE0C204349D2
:203460000870434800680B304149086042484349086008460068806840F00100096888600E
:203480003E48F6F724FD002405E03D4951F8240039490860641C3B48B4EB900FF5D336482B
:2034A000056839480068854201D0F4F785FA314800680B382F4908600E202C4908702C4821
:2034C0000068C01C2A490860FFF7FEFA08B9F4F773FA28480068C01E26490860102023499D
:2034E000087023480068401D21490860FFF790F908B9F4F761FA1F480068401F1D490860D0
:2035000012201A4908701A480068C01D18490860FFF7D2FD08B9F4F74FFA1420134908706C
:20352000FFF7CAFD08B9F4F747FA12480068C01F1049086016200D4908701C2002F0FEFF50
:2035400008B9F4F739FA1820084908704FF400510804F0F714FA08B9F4F72EFA00F0B6FF7D
:20356000AA2005490871EFF7C1FD70BD0C060020382500205C2500200030024010060020F1
:2035800000300008805901008089010810B5124800780A281EDB00200F4908704FF0AA303C
:2035A0000E49086040080E49086072B6FFF780FE044662B634B1012C08D0032C05D0042C29
:2035C00002D100E005E004E000BF00BFF4F7F4F900BF00BF10BD00005900002048250020C8
:2035E0006C250020002107E041F64C5100BF0A00A1F1010399B2FAD10200A0F1010398B2E8
:20360000F2D17047002106E0072100BF0A00A1F1010399B2FAD10200A0F1010398B2F3D1E7
:20362000704770472DE9F143BDF9000044F2F30100FB01F9BDF902004FF416514843C0F15F
:203640000008444608EB09004710A8EB09004610002F0FDA002E03DA0520F749088018E08B
:20366000002C03DC0420F449088012E00320F24908800EE0002E03DB0220EF49088008E0BA
:20368000002C03DC0620EC49088002E00120EA4908800020E9490870E748008807287BD281
:2036A000DFE800F07A044D97E0FCFB0004F51650801B4FF4966101EBA040E149088008461A
:2036C000008800EB6640488008464088A0EB6440888008460088C0F5166080B2E22803DD9F
:2036E00040F65F10C88029E0D5480088D4494988401A85B2B5F58B7F05DBD1480088333810
:20370000CF49C8801AE0CE480088C0F5166080B28A2813DDCA480088E230C949C88008465E
:20372000C088B0F5166F09DB0120C4490870C448C088C0F59650401EC149C88074E107F59D
:203740001650801B4FF4966101EBA040BC4908800846008800EB6640488008460088A0EB45
:203760006740888008464088C0F5166080B2E22803DD40F65F10C8802AE0B1484088B0498C
:203780000988401A85B2B5F58B7F06DBAC4840883338AB49C8801BE045E1A9484088C0F580
:2037A000166080B28A2813DDA5484088E230A449C8800846C088B0F5166F09DB01209F4916
:2037C00008709F48C088C0F59650401E9C49C8802AE1C4F5165038444FF4966101EBA04070
:2037E0009749088008460088A0EB674088800846808800EB6440488008464088C0F5166063
:2038000080B2E22803DD40F65F10C88029E08C4840888B498988401A85B2B5F58B7F05DBF0
:203820008748408833388649C8801AE084484088C0F5166080B28A2813DD81484088E2303F
:203840007F49C8800846C088B0F5166F09DB01207A4908707A48C088C0F59650401E784994
:20386000C880E1E004F51650801B4FF4966101EBA040734908800846008800EB66404880CC
:2038800008464088A0EB6440888008468088C0F5166080B2E22806DD01E078E02EE040F6BE
:2038A0005F10C88029E06648808865494988401A85B2B5F58B7F05DB614880883338604929
:2038C000C8801AE05E488088C0F5166080B28A2813DD5B488088E2305949C8800846C088BC
:2038E000B0F5166F09DB0120544908705448C088C0F59650401E5249C88095E007F51650ED
:20390000801B4FF4966101EBA0404D4908800846008800EB6640488008460088A0EB6740B1
:20392000888008468088C0F5166080B2E22803DD40F65F10C88029E0414880884049098841
:20394000401A85B2B5F58B7F05DB3D48808833383B49C8801AE03A488088C0F5166080B29D
:203960008A2813DD36488088E2303549C8800846C088B0F5166F09DB012030490870304819
:20398000C088C0F59650401E2D49C8804CE0C4F5165038444FF4966101EBA0402849088062
:2039A00008460088A0EB674088800846808800EB6440488040F65F10C88008460088C0F5D2
:2039C000166080B2E22803DD40F65F10C88029E01B4800881A498988401A85B2B5F58B7FBB
:2039E00005DB1748008833381549C8801AE014480088C0F5166080B28A2813DD1048008832
:203A0000E2300F49C8800846C088B0F5166F09DB01200A4908700A48C088C0F59650401ED1
:203A20000749C88000E000BF00BF0448007848B9002000F003FB08E034000020360000202B
:203A400038000020022000F0F9FA40F64C100949C880088800F0DAFA0649488800F0DCFAA4
:203A60000449888800F0DEFA0249C88800F0E0FABDE8F883380000202DE9F041044600258E
:203A800000260027F3F758FAA84618E000BF334800780128FBD100203049087030480088FF
:203AA00005442F48408806442D48808807440C212C48F8F781F908F101001FFA80F8B8F12E
:203AC0000A0FE3DB0A20B5FBF0F0274908800A20B6FBF0F048800A20B7FBF0F088800846C8
:203AE000008846F2A81188421DDB1F48008849F64041884217DC1C48408846F2A811884238
:203B000011DB1948408849F6404188420BDC1648808846F2A811884205DB1348808849F67C
:203B20004041884216DD206820F4802000F58020206006200D4948800846F3F7E7FC002077
:203B40000B4908700B484089401C0A494881022009490870F3F7F0F9BDE8F08128050020E3
:203B60001C0500209C1C00202E05002090070020A5030020300B0020C601002008B500203B
:203B8000009053480088072870D2DFE800F0933362630405320000BF4E480088404201B272
:203BA00011F5004F04DA4FF40040ADF8000009E0B1F5004F04DB47F6FF70ADF8000001E0BB
:203BC000ADF8001043484088404201B211F5004F04DA4FF40040ADF8020009E0B1F5004F6D
:203BE00004DB47F6FF70ADF8020001E0ADF8021061E000BF37484088404201B211F5004F2A
:203C000004DA4FF40040ADF8020009E0B1F5004F04DB47F6FF70ADF8020001E0ADF80210F4
:203C20002C488088BDF80220801A01B2B1F5004F04DB47F6FF70ADF8000009E011F5004F81
:203C400004DA4FF40040ADF8000001E0ADF8001031E000BF1F480088404201B2B1F5004FDF
:203C600005DB47F6FF70ADF800000AE022E011F5004F04DA4FF40040ADF8000001E0ADF846
:203C8000001014488088BDF80020801A01B211F5004F04DA4FF40040ADF8020009E0B1F5A2
:203CA000004F04DB47F6FF70ADF8020001E0ADF8021000E000BF00BFBDF900000011ADF821
:203CC0000000BDF902000011ADF80200009808BD34000020340500202DE9F04781460D4603
:203CE00016463046F11706EB9171C1F38707002415E015F824000106A000401C285C01EBF8
:203D00000041A000801C285C01EB0021A000C01C285C08440A4941F82400601CC4B2BC42A9
:203D2000E7DB31462846F1F745FA8046044840F827807A1C01464846F3F7E6FCBDE8F08771
:203D4000FC1600202DE9F04190B080460D4616463046F11706EB9171C1F38707002414E06A
:203D6000A000C01C285C0106A000801C285C01EB0041A000401C285C01EB002015F8241082
:203D800008444DF82400601CC4B2BC42E8DB3A4669464046F3F7B8FC10B0BDE8F0812DE97C
:203DA000F84381460D4616461F46002000908046002420E02819C1B26A464846F3F7F2F98C
:203DC000401C18B94FF0FF30BDE8F883385D9DF8001088420DD0385D00902819C1B29DF8D9
:203DE00000204846F3F734FA401C10B94FF0FF30EAE7601CC4B2B442DCDB31463846F1F71D
:203E0000C1F980464FEA28200090A819C1B29DF800204846F3F71CFA401C10B94FF0FF3007
:203E2000D2E708F0FF000090A819401CC1B29DF800204846F3F70CFA401C10B94FF0FF30EC
:203E4000C2E70020C0E7000070B505460C46002C33D11E4800691E4948600B4630224C2112
:203E60002846FFF79CFF401C28B9194B30224C212846FFF794FF1548006816490860134805
:203E8000406848601148806888601048C068C8600E4840690E4948620C488069C8620D4B42
:203EA0001022D6212846FFF77AFF401C28B9094B1022D6212846FFF772FF064800680A218C
:203EC000B0FBF1F004494882002070BD900B0020000B00202C0C0020DC0800202DE9F04763
:203EE00006468846174699460025FCB255201F490870AA204870084680F80280A01CC87086
:203F0000380A08710846447122464946801DEFF7C6FD552016490870AA204870301288709E
:203F2000CE70221D1149891C1148001DEFF7B7FD04F108010E48F1F73DF90546280EA11D44
:203F40000A4A5054C5F30741E01D1154C5F30721401C1154401C1554F021401C1154421C71
:203F600002493046F1F742F8BDE8F0874A0E0020490F00202DE9F04781460E4690461F46AF
:203F8000DDF820A00025FCB255201E490870AA204870300A8870CE70084680F80480A01C6D
:203FA0004871380A88710846C471224651460830EFF775FD04F1080212491348EFF76FFDF4
:203FC00004F108011048F1F7F5F80546280E04F108010C4A5054C5F3074104F109001154DA
:203FE000C5F30721401C1154401C1554F021401C1154401CC2B20349484601F008F9BDE848
:20400000F087000048100020DE10002001490968486370479C1C0020014909688863704751
:204020009C1C002001490968C86370479C1C002001490968086470479C1C002008490968BB
:20404000096A21F40051064A1268116204490968096A41EA0031024A1268116270470000CD
:204060009C1C002010B51048007801281BD10F4A32210F4800F048F90446EFF70FFF0D49F6
:20408000086008460068EFF72CFF0B490860002005490870084800681E2804DA03480088A0
:2040A00000B20649088010BD1801002024010020140800201C01002020010020140100203D
:2040C0002DE9F04705460C4616461F46DDE90889F6F7B8FB19490968401A32282BD3F6F7CC
:2040E000B1FB1649086005FB06F090FBF7F000FB08F000EBC000000142F2107190FBF1F025
:20410000208020880E49096808440D4908600D480078401C0B4908700846007808280ADBB5
:204120000020087006480068C0F3CF00A9F80000002003490860BDE8F08700000C040020EE
:20414000140400201004002070B504460D461646F6F778FB24490968401A322841D3E07877
:2041600028B9F6F76FFB214908600120E070F6F769FB1E490968401AB0F57A6F04D90020B6
:20418000A0704FF6FF70A060208980B24FF6FF71884202D10020A07001E00120A070A078D4
:2041A000012812D1A06810B94FF0FF30A0604FF4B4707043A168B0FBF1F0208020880A2291
:2041C0000B49FDF763FC288007E00020208028800A210748F0F71FFB70BDF6F733FB024933
:2041E000086000BFF8E70000180400201C0400205A15002000B585B000BF1048806940F094
:2042000020000E4988610846806900F02000009000BF00BF0420019009480290012003909D
:2042200001A90848F6F76EF9002202210820F6F7D8FB0820F6F7C8FB05B000BD0010024067
:2042400000001110001401402DE9F04104460D4617461E46F6F7F6FA28490968401A3228D0
:204260004AD3E07828B9F6F7EDFA254908600120E070F6F7E7FA22490968401A4FF47A61AB
:2042800091FBF6F1884201D90020A070A078012822D1A06810B94FF0FF30A0604FF4B470FD
:2042A0007843B0FBF6F0A168B0FBF1F0208020880A221449FDF7EAFB2880F6F7C3FA616858
:2042C000411AA068B1EB400F12D940F20E41A0684843800AA0600BE00020208028800A2189
:2042E0000848F0F798FA4FF0FF30A060BDE8F081F6F7A8FA0149086000BFF7E7040400206B
:2043000008040020461500202DE9F74F88B0044689464FF0000BDA460020069000210F46B3
:2043200088460D460E4600BF0FE034F81B00EFF7CBFD3A464346CDE90401EFF799FC0746D9
:2043400088460BF1010000F0FF0BCB45EDDB4846EFF7BAFD02460B46CDE90201384641463E
:20436000EFF72DFDCDE90401EFF733FE06900698EFF7D0FD81B20A9801804FF0000A23E0D2
:2043800034F81A00EFF78AFD00900699EFF738FC029034F81A00EFF781FD00900699EFF7D0
:2043A0002FFC01900299EFF731FC0390EFF7FEFD2A463346CDE90401EFF75AFC05460E46A0
:2043C0000AF1010000F0FF0ACA45D9DB2846314602F0AAFBCDE90201EFF7CFFD80B2059077
:2043E000EFF772FD05460E4628463146EFF7C5FD80B20BB0BDE8F08F10B594B009200A905F
:204400004FF480300B9000200C9001200E90109002201190C10312914FF4E01113910AA83F
:20442000F6F7BEFD18B1CD211AA001F0E7FE0F20059002200690002007904FF4806008909F
:2044400000200990022105A8F6F768FC18B1DB2110A001F0D3FE022001908003039001A8D9
:20446000F6F7C4FB18B1E2210AA001F0C7FEF6F727FD4FF47A71B0FBF1F42046F7F7B6F893
:204480000420F6F7ADFF00221146501EF6F7A9FA14B010BD2E2E5C53656C66546573745520
:2044A0007365725C7372635F6D6964646C6577617265735C73746D33326678785F53545558
:2044C000737461727475702E6300000010B590B00220069001200A9010200B9000200D9038
:2044E00006A8F6F75DFD20B140F2031114A001F085FE0F2001900020029003904FF4806060
:20450000049000200590002101A8F6F707FC20B140F211110AA001F071FEF6F7D1FC4FF46C
:204520007A71B0FBF1F42046F7F760F80420F6F757FF00221146501EF6F753FA10B010BD3F
:204540002E2E5C53656C6654657374557365725C7372635F6D6964646C6577617265735CEA
:2045600073746D33326678785F535455737461727475702E63000000034618044843B0FB92
:20458000F2F0704710B5F6F793F9F7F749F803480078401C0149087010BD000059000020EE
:2045A00010B594B009200A904FF480300B9000200C9001200E90109002201190C10312915C
:2045C0004FF4E01113910AA8F6F7EAFC20B14FF4DA711CA001F012FE0F20059002200690E6
:2045E000002007904FF48060089000200990022105A8F6F793FB20B14FF4E17111A001F03D
:20460000FDFD022001908003039001A8F6F7EEFA20B140F2C9110BA001F0F0FDF6F750FCBA
:204620004FF47A71B0FBF1F42046F6F7DFFF0420F6F7D6FE00221146501EF6F7D2F914B043
:2046400010BD00002E2E2F436F72652F5372632F6D61696E2E6300001148006840F00100CB
:204660000F490860084640680E4908400C494860084600680C490840094908600846006825
:2046800020F4802008600846406820F4FE0048604FF41F008860C8030449086070470000CD
:2046A000001002400000FFF8FFFFF6FE08ED00E010B50248F7F7B2F910BD00009C1C00209D
:2046C00000220268184B984208D0B0F1804F05D0164B984202D0164B984203D122F0700254
:2046E0004B681A43104B984208D0B0F1804F05D00E4B984202D00E4B984203D122F4407284
:20470000CB681A4322F080024B691A4302608B68C3620B688362044B984201D10B690363BD
:204720000123436170470000002C0140000400400008004030B50023012404FA01F3046A74
:204740009C430462046A02FA01F52C43046230BD30B50023042404FA01F3046A9C4304621D
:20476000046A02FA01F52C43046230BD30B50C460021816821F47F4142EA032525432943D9
:20478000816030BD0A460021816821F0700142F0070319438160704730B5002400220023F1
:2047A000056A25F001050562026A4368846924F0700424F003040D682C4322F002028D6872
:2047C0002A430D4DA84206D100BF22F00802CD682A4322F00402084DA84207D123F480739B
:2047E00023F400734D692B438D692B43436084614D684563026230BD002C014030B50024FB
:2048000000220023056A25F010050562026A4368846924F4E04424F440740D6844EA05247B
:2048200022F020028D6842EA05120F4DA84207D100BF22F08002CD6842EA051222F04002CF
:20484000094DA84209D123F4806323F400634D6943EA85038D6943EA8503436084614D6877
:204860008563026230BD0000002C014030B5002400220023056A25F480750562026A436849
:20488000C46924F0700424F003040D682C4322F400728D6842EA05220E4DA84207D100BFB8
:2048A00022F40062CD6842EA052222F48062094DA84209D123F4805323F400534D6943EAAF
:2048C00005138D6943EA05134360C4614D68C563026230BD002C014030B5002200230024D4
:2048E000056A25F480550562036A4468C26922F4E04222F440720D6842EA052223F400537E
:204900008D6843EA0533074DA84204D124F480444D6944EA85144460C2614D680564036287
:2049200030BD0000002C014030B50B46144600210022026A056A25F001050562816921F0F2
:20494000F00141EA041122F00A021A438161026230BD30B50B46144600210022056A25F021
:20496000100505628169026A21F4704141EA043122F0A00242EA03128161026230BD0146D0
:20498000002240F205100860086882B240F20510824201D00020704740F28A20086008683B
:2049A00082B240F28A20824201D00020F3E70020086045F255504860486882B245F255508C
:2049C000824201D00020E6E742F6A8204860486882B242F6A820824201D00020DBE7002032
:2049E000486045F255508860886882B245F25550824201D00020CEE74AF6A2208860886807
:204A000082B24AF6A220824201D00020C3E70020886045F25550C860C86882B245F25550B5
:204A2000824201D00020B6E742F6AA20C860C86882B242F6AA20824201D00020ABE700202D
:204A4000C86045F255508861886982B245F25550824201D000209EE74AF6AA20886188694A
:204A600082B24AF6AA20824201D0002093E70020886145F25550C861C86982B245F255507A
:204A8000824201D0002086E74AF6AA20C861C86982B24AF6AA20824201D000207BE700201B
:204AA000C86141F255500862086A82B241F25550824201D000206EE742F6AA200862086A25
:204AC00082B242F6AA20824201D0002063E70020086245F255504862486A82B245F25550CF
:204AE000824201D0002056E74AF6AA204862486A82B24AF6AA20824201D000204BE7002019
:204B0000486245F255508862886A82B245F25550824201D000203EE74AF6AA208862886A63
:204B200082B24AF6AA20824201D0002033E70020886245F25550C862C86A82B245F2555016
:204B4000824201D0002026E74AF6AA20C862C86A82B24AF6AA20824201D000201BE7002018
:204B6000C86255200863086B82B2552A01D0002011E7AA200863086B82B2AA2A01D000207B
:204B800009E70020086345F255504863486B82B245F25550824201D00020FCE64AF6AA20AF
:204BA0004863486B82B24AF6AA20824201D00020F1E60020486345F255508863886B82B214
:204BC00045F25550824201D00020E4E64AF6AA208863886B82B24AF6AA20824201D000209F
:204BE000D9E60020886345F25550C863C86B82B245F25550824201D00020CCE64AF6AA2030
:204C0000C863C86B82B24AF6AA20824201D00020C1E60020C86345F255500864086C82B261
:204C200045F25550824201D00020B4E64AF6AA200864086C82B24AF6AA20824201D000206C
:204C4000A9E60020086441F215508864886C82B241F21550824201D000209CE640F60A205E
:204C60008864886C82B240F60A20824201D0002091E600208864086101208CE62DE9F04145
:204C800004460E4690461F4630480078012812D12F4801780078401C2D4A10702D4820F8F7
:204CA00011601046007832281CDB0020274908701146087016E0322226493046FCF7E6FE87
:204CC00005462088A84209DDF5F7BCFD22490968401AB0F57A7F05D9258003E0F5F7B2FD97
:204CE0001D49086040F6340008FB00F0642190FBF1F0C0F580502188884203DBF5F7A2FD37
:204D000016490860F5F79EFD14490968401A42F21071884217D9386820F0400040303860B6
:204D200003200F494880208888800846F2F7EEFB00200C4908700C48808A401C0A4988825C
:204D400001200A490870BDE8F0810000210400202204002086150020280400202404002077
:204D600090070020A5030020000B0020C60100202DE9F04704460F46E7824FF00908414676
:204D80002046F3F755FAC01B0FFA80F919F1780F2ADDB9F1780F27DA002606E0701C34F889
:204DA000100024F81600701CC6B2A8F10100B042F4DC24F8107041462046F3F7C3FA05B26A
:204DC000608AA84200DA658241462046F3F7CBFA05B2A08AA84200DDA582064B18227E21A9
:204DE0000548FEF7DCFF02E0002004490870BDE8F08700006E150020340400202004002074
:204E000003B50246002006E002EB4001BDF804300B80411CC8B20C28F6D30CBDF0B504465E
:204E20000D46671B39B2178892F802C007FB0CF74FF0640C97FBFCF7BBB29778C7EBC70792
:204E400007EB4706002901DA002014E0994206DA4FF4B6774F4397FBF3F7B8B20BE0CF1A84
:204E60004FF4D96C07FB0CF7A6EB030C97FBFCF707F5B677B8B2F0BD08B5024602F5004004
:204E800081B20846CB1701EB936399114FF6FE70014001F4407038B3B0F5807F36D0B0F550
:204EA000007F03D0B0F5407F40D10DE0C8B2214B33F81000ADF80200C8B2C0F1FF0033F821
:204EC0001000ADF8000032E0C8B2C0F1FF00194B33F81000ADF80200C8B233F81000404264
:204EE00000B2ADF8000022E0C8B2124B33F81000404200B2ADF80200C8B2C0F1FF0033F817
:204F00001000404200B2ADF8000010E0C8B2C0F1FF00084B33F81000404200B2ADF8020025
:204F2000C8B233F81000ADF8000000E000BF00BF009808BDC670010870B505466C6A0020B7
:204F4000E085E0842046F7F79AF870BD2DE9F04106460D461446002025490870F5F772FCD5
:204F60002349486005F0FF08A5F50040083830B1A0F6FA70B8B1B0F5545F2DD108E04246F7
:204F800021461C48EEF78BFD00201B4908702BE023462A46314640F21560FEF79FFF012027
:204FA0001649087020E02178627801EB02218FB2002007E0124931F81010B94200DD03E0F1
:204FC000411CC8B20B28F5D300BF00F14901CAB20C4981F8252007E023462A46314640F20D
:204FE0001560FEF77BFF00BF00BFBDE8F0810000DC010020D0010020DA0100205D000020D3
:20500000907401081C09002010B50A46C37893421EDBC3681B68DB6823F02003C468246841
:20502000E360C3789B1AC370C3681B68DB6843F02003C4682468E360114683780B4499B2DC
:2050400003788B4202DC0378CB1A99B281701BE0C3681B68DB6823F02003C4682468E36071
:20506000C1780023C370C3681B68DB6843F02003C4682468E3608378194403788B4202DCE1
:205080000378CB1A99B2817010BD0168C96821F490710268D1600168496921F001010268C4
:2050A0005161202180F83A10704710B504462068C06820F040002168C860202084F83900CF
:2050C0002046F7F722F9002010BD00BFC27803789A42FBD0C2681268D26822F08002C368BC
:2050E0001B68DA60C2788AB9C26812681268C2F3C0125AB1C26812685160C2681268D26893
:2051000042F08002C3681B68DA60704743788268D1544278521CD2B2427003789A4201D1EB
:2051200000224270C278521CC270C2681268D26842F08002C3681B68DA6000BFE5E710B5F7
:2051400002460B461946D4789C4209DB94780C44A1B214788C4204DC14780C1BA1B200E07A
:2051600000219468605C10BD70B5044694F83A0022284AD1A068B0F5805F13D1A56A2069E7
:2051800040B920684068C0F308002880A06A801CA06219E020684068C0B22880A06A401C32
:2051A000A06211E0206938B920684068C1B2A26A501CA062117007E02068406800F07F015D
:2051C000A26A501CA0621170E08D401E80B2E085C8B92068C06820F020002168C8602068D8
:2051E000C06820F480702168C8602068406920F0010021684861202084F83A002046F7F714
:2052000083F8002070BD0020FCE70220FAE7F0B507460D461646002405E0295D3846FFF71C
:2052200054FF601CC4B2B442F7DBF0BD2DE9F041044600252068006920F44050E1680843D5
:20524000216808612169A06808436169084305432068C06841F20C61884328432168C860EB
:205260002068406920F44070A1690843216848615F49206888425CD1F5F738FE00EBC001BD
:2052800001EB001061688900B0FBF1F6F5F72EFE00EBC00101EB001061688900B0FBF1F090
:2052A0006421B0FBF1F000EBC00101EB0010A6EB8000322101EB00106421B0FBF1F000F0D4
:2052C000F006F5F713FE00EBC00101EB001061688900B0FBF1F06421B0FBF1F006EB00163D
:2052E000F5F704FE00EBC00101EB001061688900B0FBF1F7F5F7FAFD00EBC00101EB0010A8
:2053000061688900B0FBF1F06421B0FBF1F000EBC00101EB0010A7EB8000322101EB001095
:205320006421B0FBF1F000F00F003044216888605BE0F5F7CBFD00EBC00101EB0010616818
:205340008900B0FBF1F6F5F7C1FD00EBC00101EB001061688900B0FBF1F06421B0FBF1F0F1
:2053600000EBC00101EB0010A6EB8000322101EB00106421B0FBF1F000F0F006F5F7A6FD9F
:2053800000EBC00101EB001061688900B0FBF1F06421B0FBF1F006EB0016F5F797FD00EB04
:2053A000C00101EB001061688900B0FBF1F7F5F78DFD00EBC00101EB001061688900B0FB30
:2053C000F1F06421B0FBF1F000EBC00101EB0010A7EB8000322101EB00106421B0FBF1F0C1
:2053E00000F00F00304421688860BDE8F081000000380140014691F8390021282CD18868FB
:20540000B0F5805F0FD10A6A1088C0F308000B685860086918B9086A801C086209E0086A21
:20542000401C086205E00B6A581C086218780B685860C88C401E80B2C88458B90868C068DA
:2054400020F080000B68D8600868C06840F040000B68D860002070470220FCE710B5054870
:2054600000F00EF8044800F040F80448F6F708FE10BD0000E8050020F8050020F824002050
:2054800008B5C26812681268C2F3401262B3C26812685268D1B2C268126812680022B2B989
:2054A00043788268D1544278521CD2B2427003789A4201DB00224270C278521CD2B2C2705F
:2054C00003789A4203DD0278C2700122027100BF00220092C268126812680092C26812688C
:2054E0005268009200BF00BF08BDC16809680968C1F3C01139B3C1680968C96801F0800164
:2055000009B36FF08001C26812681160C17891B1C178491EC17082788168895CC268126822
:2055200051608178491CC9B28170027891420ADB0021817007E0C1680968C96821F0800168
:20554000C2681268D160704710B50248F4F76EF810BD0000B422002010B54FF4FA710248DF
:2055600000F004F810BD0000E80500202DE9F34F83B00398C0780D2873DB00210398FFF7D2
:20558000DEFD01906B490198087001210398FFF7D6FD8146674981F80190019855287DD16F
:2055A000B9F1AA0FFBD102210398FFF7C8FD6149887003210398FFF7C2FD5E49C870042129
:2055C0000398FFF7BCFD06465A490E71112E03D0162E01D00C2E7DD105210398FFF7AFFD01
:2055E00007465448477107210398FFF7A8FD834606210398FFF7A3FD0BEB00201FFA80F8E4
:205600004FEA18204B49887181F8078007210398FFF795FD0446381B02287AD10398C1785B
:2056200007F10B0081421DDA43480078012806D1F5F708F94149086000203F490870F5F7BF
:2056400001F93E490968411A0498814206D9F5F7F9F83A49086001203749087005B0BDE884
:20566000F08F64E001203449087000250FE005F10800C1B20398FFF762FD31494855084677
:20568000415D05F108002B4A1154681C85B2A542EDDB04F10800C1B2039800E043E0FFF726
:2056A0004EFD4FEA006B04F10900C1B20398FFF746FD0BEB004B04F10A00C1B20398FFF772
:2056C0003EFD0BEB002B04F10B00C1B20398FFF736FD00E022E05844029004F108011548CC
:2056E000EFF768FD82460298B0EB0A000CD1144A41463046FFF72AFC07F10B00C1B20398F3
:20570000FFF782FCAAE704E001210398FFF77CFC0DE001210398FFF777FC08E001210398BD
:20572000FFF772FC03E001210398FFF76DFC00BF94E700000A120020200200201C02002010
:2057400074110020012806D0022854D003287DD004287CD1C8E0FE49FE4A13680B6053688E
:205760004B6092688A600A46FB490B68D3604B68136189685161F9490B6893614B68D36106
:20578000896811621146F64A13684B6253688B629268CA62F34A13680B6353684B6392688F
:2057A0008A63F14A1368CB6353680B6492684A64EE49C978AA291DD140F27321E44A118088
:2057C00040F2FD31918140F2226111834FF40C72DF494A8340F63411DD4A91844FF40C72E0
:2057E000DB49CA8440F60B31D94A91874FF40C72D749CA87A0E0D64ADD490B6813604B68F9
:205800005360896891601146DA4A1368CB6053680B6192684A61D84A13688B615368CB6196
:2058200092680A62D54A13684B6253688B629268CA62D34A13680B6353684B6392688A6397
:20584000D04A1368CB6353680B6401E025E072E092684A64C549C978AA291DD140F2CA214E
:20586000BB4A118040F27641918140F2747111834FF40C72B6494A8340F62E31B44A9184B7
:205880004FF40C72B249CA8440F66A51B04A91874FF40C72AE49CA874EE0AD49BA4A13684F
:2058A0000B6053684B6092688A60B84A1368CB6053680B6192684A610A46B5490B6893610A
:2058C0004B68D36189681162B2490B6853624B6893628968D1621146AF4A13680B6353689A
:2058E0004B6392688A6327E09949AC4A13680B6053684B6092688A60A94A1368CB605368B0
:205900000B6192684A610A46A6490B6893614B68D361896811621146A34A13684B6253685E
:205920008B629268CA62A14A13680B6353684B6392688A6300E000BF00BF9D49897B782947
:205940000DDC9B49897B502909DB81490988984A927B5143642291FBF2F17D4A1180944911
:20596000097C78290DDC9249097C502909DB784989898F4A127C5143642291FBF2F1744ADA
:2059800091818B49897C78290DDC8949897C502909DB6F49098B864A927C5143642291FB8E
:2059A000F2F16B4A11838249097D78290DDC8049097D502909DB6649898C7D4A127D514386
:2059C000642291FBF2F1624A91847949897D78290EDC7749897D50290ADB5D49498E744A5F
:2059E000927D5143642291FBF2F18AB258494A866F49C97B5A2905DC5549097A491E544ADC
:205A0000117208E06A49C97B6E2904DB5049097A491C4F4A11726649497C5A2906DC4C49A3
:205A2000097D491ECAB24A490A7509E06049497C6E2905DB4649097D491CCAB244490A751B
:205A40005B49C97C5A2908DC414991F82010491ECAB23F4981F820200BE05549C97C6E292A
:205A600007DB3B4991F82010491CCAB2384981F820204F49497D5A2908DC354991F82C10E4
:205A8000491ECAB2324981F82C200BE04849497D6E2907DB2E4991F82C10491CCAB22C4996
:205AA00081F82C204249C97D5A2908DC284991F83810491ECAB2264981F838200BE03C4914
:205AC000C97D6E2907DB224991F83810491CCAB21F4981F838203749C97C78290DDC3549E4
:205AE000C97C502909DB1A49C988324AD27C5143642291FBF2F1164AD1802E49497D78296E
:205B00000EDC2C49497D50290ADB1149498A294A527D5143642291FBF2F18AB20C494A82AD
:205B20002449C97D78290EDC2249C97D50290ADB0749C98B1F4AD27D5143642291FBF2F133
:205B40008AB20349CA831B49497E782943DC33E0E40B0020A6740108B2740108BE740108D6
:205B6000CA740108D6740108E2740108C2010020EE740108FA740108067501081275010853
:205B80001E7501082A75010836750108427501084E7501085A7501086675010872750108D5
:205BA0007E7501088A75010896750108A2750108B00A0020D00A00204049497E50290ADB2B
:205BC0003F49498D3D4A527E5143642291FBF2F18AB23B494A853949C97E78290EDC374924
:205BE000C97E50290ADB3649C98E344AD27E5143642291FBF2F18AB23149CA862F49897C50
:205C000078290DDC2D49897C502909DB2C4949892A4A927C5143642291FBF2F1284A51818C
:205C20002649097D78290EDC2449097D50290ADB2349C98A214A127D5143642291FBF2F151
:205C40008AB21F49CA821D49897D78290EDC1B49897D50290ADB1A49498C184A927D514358
:205C6000642291FBF2F18AB215494A841349097E78290EDC1149097E50290ADB1049C98D6B
:205C80000E4A127E5143642291FBF2F18AB20C49CA850A49897E78290EDC0849897E5029FD
:205CA0000ADB0749498F054A927E5143642291FBF2F18AB202494A8770470000D00A0020E6
:205CC000E40B002000BFFEE700B587B00020C7490860C74908800720C64908701821C64800
:205CE000EDF7F6FE1821C548EDF7F2FE1821C448EDF7EEFE1022C349C348EDF7D0FEC34897
:205D0000C3490A680260496841601022C1A1C648EDF7E9FE1022C5A1C3481030EDF7E3FE3C
:205D20002E21C148203880F83F102022C4A1CD48EDF7D9FE00BFCCA2D2E900109268CDE9CD
:205D400005020491CBA207CA01AB07C39DF81A0030389DF81910303901EB810100EB41001B
:205D6000C04988760322C6A104A8EDF7DEFE18B90120BC49C87670E00322C2A104A8EDF787
:205D8000D4FE18B90220B749C87666E00322BEA104A8EDF7CAFE18B90320B249C8765CE075
:205DA0000322BAA104A8EDF7C0FE18B90420AD49C87652E00322B6A104A8EDF7B6FE18B929
:205DC0000520A849C87648E00322B2A104A8EDF7ACFE18B90620A349C8763EE00322AEA1E2
:205DE00004A8EDF7A2FE18B907209E49C87634E00322AAA104A8EDF798FE18B908209949D1
:205E0000C8762AE00322A6A104A8EDF78EFE18B909209449C87620E00322A2A104A8EDF7A5
:205E200084FE18B90A208F49C87616E003229EA104A8EDF77AFE18B90B208A49C8760CE074
:205E400003229AA104A8EDF770FE18B90C208549C87602E000208349C8769DF815103039AC
:205E60009DF81400202801D1002002E09DF81400303800EB800001EB40007A4908779DF8DE
:205E8000051030399DF80400202801D1002002E09DF80400303800EB800001EB400071497D
:205EA00048779DF8081030399DF80700202801D1002002E09DF80700303800EB800001EBFA
:205EC0004000684988779DF80B1030399DF80A00202801D1002002E09DF80A00303800EB0C
:205EE000800001EB40005F49C87700BF7048007828B930214C48203880F82A1036E06C4886
:205F00000078012805D131214748203880F82A102CE067480078022805D1322142482038B7
:205F200080F82A1022E062480078052805D132213D48203880F82A1018E05D480078032866
:205F400005D133213848203880F82A100EE058480078042805D134213348203880F82A10AB
:205F600004E030213048203880F82A10102251A12D482038EDF7B7FD102253A12A48103801
:205F8000EDF7B1FD082255A15748EDF7ACFD082256A155480830EDF7A6FD082256A15248EB
:205FA0001030EDF7A0FD5748574B0ECB0EC000F0D7F800F0AFF85548007B544991F91B1078
:205FC0000844524989794843C0EB001001034F48C07941F2C6125043B1FBF0F04C498881F6
:205FE00008468089C88107B000BD000094010020D0010020B80100208C090020980A002097
:20600000800A0020F0720108A4090020B9010020CC730108202020202020202034382020D0
:2060200020202020000000003C0900205636723272325F3230323431313038430000000073
:2060400054433031313030302D4D53303030302D563072322E202020202020202020202015
:20606000000000005C0900204E6F7620203820323032340032323A35363A3237000000005C
:206080004A616E00466562004D617200417072004D6179004A756E004A756C0041756700FB
:2060A000536570004F6374004E6F76004465630004020020564C363530302026205653377A
:2060C0003530302E0000000030303030303030303030303030303030000000004D4F5449C4
:2060E0004E4F564100000000400B0020575548414E2E202000000000323032313039303181
:2061000000000000B80B0020E8F7FF1FB00A00200C02002010B5302209490A48EDF7BFFC3D
:20612000102209490948EDF7BAFC0948094C1ECC1EC0102208490948EDF7B1FC10BD000050
:2061400028740108000B002058740108300B00202C0C002078740108687401083C0C0020A5
:2061600010B50C2213A11748EDF7BDFC164817490A6802604968416015481649096801600A
:20618000202215491548EDF78AFC1448007814490870202213491448EDF781FC1022134906
:2061A0001348EDF77CFCCC2212491348EDF777FC10BD000030303030303030303030303020
:2061C00000000000C40B0020C701002088740108C201002014740108D4730108B00A002045
:2061E000C1010020F4730108D00A002018740108F00A002000730108B409002088B00446C9
:206200000D4631E01948FAF79CF80020FBF7CAFEF0F752FE20216846EDF75AFC2046EDF7B0
:206220006EFC0646324621466846EDF738FC2046EDF765FC694608440DA10A88028089789A
:2062400081702046EDF75BFC69460844C0F803506B464FF620720C214FF4E260FDF73EFE3C
:20626000C820F4F709F800BFCCE7000000010020202C200008B52B4988420DD100BF2A4940
:20628000896941F00401284A91611146896901F00401009100BF43E0244988420DD100BFEC
:2062A0002149896941F008011F4A91611146896901F00801009100BF32E01D4988420DD13A
:2062C00000BF1949896941F01001174A91611146896901F01001009100BF21E01549884252
:2062E0000DD100BF1049896941F020010E4A91611146896901F02001009100BF10E00E4928
:2063000088420DD100BF0849896941F04001064A91611146896901F04001009100BF00BF95
:2063200008BD00000008014000100240000C014000100140001401400018014070B5044642
:206340000E46A1882068F4F76BFA28B9A07908B9012506E0002504E0A07908B9002500E039
:206360000125012E04D1207A68402840E07102E0207A6840E071257270BD10B50446A18887
:2063800001222068F4F758FA10BD00BF704702E008C8121F08C1002AFAD1704770470020A3
:2063A00001E001C1121F002AFBD1704700F0010181F313887047000001490860704700003B
:2063C00018060020F0B504460E4619681F683D14A54206DA31440814A04212DD204601044F
:2063E0000FE0A5420CDD02EB04473DB2A94202DA2046010405E0891A081410B9002100E017
:2064000020461960F0BD000010B50A46437993421EDB1E4B1B685B6923F002031B4C246896
:20642000636143799B1A4371184B1B685B6943F00203164C24686361114603790B4499B272
:2064400083788B4202DC8378CB1A99B201711BE00E4B1B685B6923F002030C4C246863619E
:20646000417900234371094B1B685B6943F00203064C246863610379194483788B4202DC97
:206480008378CB1A99B2017110BD0000B422002010B502460B46194654799C4209DB1479C3
:2064A0000C44A1B294788C4204DC94780C1BA1B200E000219468605C10BD00007FB50646F3
:2064C000002404E0305D18490855601CC4B2082CF8DB3823154A02A9304600F0BFFB0024C7
:2064E0001EE0002504E002A800F0E0FA681CC5B20F48005DA842F6DC40230E4A694602A8A2
:2065000000F0ACFB002507E01DF805000A4901EBC4014855681CC5B2082DF5DB601CC4B22B
:20652000102CDEDB7FBD00009D030020707C0108487F0108A87C010862140020014601207A
:20654000064A12688A4206D1044A1268044B1B685A40521C02B10020704700003825002025
:206560005C2500202DE9F04F87B082460F469046994600250AE0785D3A49495D884203D072
:206580003846FFF79BFF0725681CC5B2082DF2DB4023354A05A9504600F060FB012536E017
:2065A000002405E005A8005D03A90855601CC4B2082CF7DBB8F1000F04D1681E2B4901EB54
:2065C000C00B04E0C5F11000284901EBC00B002406E003A9201D085C05A90855601CC4B2CA
:2065E000042CF6DB01AA05A9584600F043F8002409E003A8005D01A9095D484005AA211DDE
:206600005054601CC4B2042CF3DB681CC5B2112DC6DB9DF814609DF818008DF814008DF838
:2066200018609DF815609DF819008DF815008DF819609DF816609DF81A008DF816008DF8B8
:206640001A609DF817609DF81B008DF817008DF81B604023064A494605A800F0FFFA07B0D9
:20666000BDE8F08F9D030020B07B010862140020F07B0108F0B587B005460E4617464023BD
:20668000104A05A9304600F0E9FA002410E005A8005D295D484000F03F0003A908550A48F3
:2066A00000EB8410095D405C01A90855601CC4B2082CECDB2023054A394601A800F0CEFAF3
:2066C00007B0F0BDE87C0108487D0108287D01081CB5F6F7A3F8F6F7A9F8CD490870F4F70D
:2066E000F3F8FDF75DFFF6F7DBF9FAF7A1FFFBF741F8FBF7A9F8FBF7F1F8FAF77FFFFAF714
:2067000047FEFAF7F5FEFAF74BFFFBF731F9FCF7C3F9EDF7DDFE1420F3F7AEFDBD48F5F7D1
:20672000C5F8FFF7D1FAFBF705F8FAF7EDFBBA48F0F76AFCF0F7ECFDB748F0F71DFCF0F70E
:2067400033FEB649087008460178B348FDF77CFBB349B448F0F706FEF9F722FDF1F7F6FA9A
:206760000020B149087051E1B0480078401CAF49087008460078C82801DD00200870AC48F9
:206780000088F1F765FDFBF7B9F9EEF797FEFEF7E3FEA84A5178A84AD07AA84BA84A1278CD
:2067A000F8F776FAFAF7B0FDF0F750FBA248807EAA2841D1A348007BC0B1A248B0F9020072
:2067C0000B2190FBF1F084B29E499B48007B9A4A92F91B20104480B2CDE900019648C379A5
:2067E000827999492046FDF76BFC46E09548B0F902000B2190FBF1F09249897A884206DD2A
:206800009048B0F902000B2190FBF1F001E08D48807A84B28B498848007B874A92F91B20C1
:20682000104480B2CDE900018348C379827986492046FDF745FC20E07F48807EEE280AD1F9
:206840007D48007B7C49C97E0844C2B27D497E48FDF77AFC11E07848007B7749C97E0844B7
:20686000C2B27548007E08B9012001E07248007E034674497448FDF7E7FC7448F1F7CAFC6B
:206880007348EEF735F900BF7248007818BB7248007828B1F3F7D6FF42F21071884229D91B
:2068A0006848C0880A2190FBF1F084B26B488088614A0090127B604D95F91B502A4490B23A
:2068C000674A137B644A11782246FBF7B5FD0120604908700EE05B4C2389604C627AA18802
:2068E000594CE068FBF782FC5E4A1178534A1078FBF7D8FD00BFFAF7EBF8F8F7CFFA5A4831
:20690000FAF75EFAFAF768FC4E4B9A7D1989987AF7F7DEFF554908705248807910B954489C
:20692000F0F716FD4F48807930B952495248F0F7B1FD5248FBF74AFF51480078E8B95148FA
:206940000068514908604F48406848604D48806888604C48C068C8604348001F40680861E2
:20696000282230480830FDF7B7F9042247A12D48FDF7B2F9012042490870F8F7FBFBF9F75E
:2069800043FD44480068FAF775FA2D480078FAF799FA2B480078FAF741FA3F48FAF7D0FA99
:2069A000FDF760FBF1F732FA00BF3C48007820B1012803D002281FD111E01EE0F3F742FFB8
:2069C00037490968401A42F6E061884206D9022032490870F3F736FF324908600DE0F3F75C
:2069E00031FF30490968401A47F23051884202D900202A49087000E000BF00BF00BFFCF7A9
:206A0000C5FDFBF7C9FF2848F3F74AFFACE6000004020020DC1C0020340400202C040020DF
:206A2000FFEF010800E801085C0000205A00002008020020B9010020B00A0020DA000020A0
:206A4000D8000020DC080020F403002045040020440400205B000020F40100207C0900201D
:206A6000F00A0020DE000020040B0020EE0000202D040020A503002090070020C60100200A
:206A80000B0200202C0C0020900B0020464C41470000000094010020D00B002006010020C5
:206AA000080100200C010020040800200CB5002104E0425C0DF801204A1CD1B20829F8DBDD
:206AC000002112E0425C5206120E425406290ADA4A1C1DF8022002F08002802A03D1425CB7
:206AE00042F0010242544A1CD1B20729EADB9DF8002002F0800222B1C27842F01002C27041
:206B000003E0C27822F01002C2709DF8032002F0080222B1827942F00102827103E082797A
:206B200022F0010282710CBD2DE9F04106460F46EDF726FB04000D4618BF0120284320F0CD
:206B40000040C0F17F6000F1E040C00F0ED0301C18BF0120384320F00040C0F17F6000F117
:206B6000E040C00F04BF0120FFF726FC20462946BDE8F08130B502460023002952D0334829
:206B8000007890B13248334C247830F81400324C2468201A304C2060204600681044206089
:206BA0002B482C4C247820F814202A480078401C284C2070204600781E280FDB00202070FA
:206BC0002248007818B90120204C207006E01F480078012802D102201C4C20701B4800782F
:206BE000022806D11C4800681E24B0FBF4F083B211E01648007801280CD11648007808B95E
:206C0000134608E014480068124C2478B0FBF4F083B200E01346052093FBF0F0904212DD24
:206C2000134610E0002005E00024094D25F81040441CE0B21E28F7DB0020064C2070064CC1
:206C40002060024C2070184630BD0000F0030020F6140020E8030020EC0300202DE9F041ED
:206C600004461D46154E002000BF4FF000080746401C01F807800828F7DB002000BF12F8CA
:206C8000013B04EBE3073F7803F0070C16F80CC007EA0C0767B101EBE0073F7800F0070C9F
:206CA00016F80CC047EA0C0701EBE00C8CF80070471C3846AF42E2DBBDE8F081587F010865
:206CC000000000000000000001020304060708090000000001020304204E00040300000409
:206CE00000000004000000009CFFFFFFFF7F0000000000FE00FCFF0100000000204E00040D
:206D00000300000400000004000000000080FFFFFF7F0000000000FE00FCFF010000000072
:206D2000400000040300000400000004000000000000FCFF00000000000000F00000000019
:206D400000000000307500012C0100040000000400000000CCF7FFFF000000000030DFFF89
:206D60000000000000000000001000040100000400000004000000009CFFFFFF1A0400003F
:206D80000070FEFF0068100000000000307500042C0100040000000400000000E6FBFFFF51
:206DA000000000000098EFFF0000000000000000204E0004030000040000000400000000D0
:206DC0009CFFFFFFFF7F0000000000FE00FCFF0100000000204E0004030000040000000425
:206DE000000000000080FFFFFF7F0000000000FE00FCFF0100000000400000040300000452
:206E000000000004000000000000FCFF00000000000000F0000000000000000030750001DD
:206E20002C0100040000000400000000CCF7FFFF000000000030DFFF00000000000000004E
:206E4000001000040100000400000004000000009CFFFFFF1A0400000070FEFF0068100079
:206E600000000000307500042C0100040000000400000000E6FBFFFF000000000098EFFFCF
:206E80000000000000000000204E00040300000400000004000000009CFFFFFFFF7F00005E
:206EA000000000FE00FCFF0100000000204E00040300000400000004000000000080FFFFDD
:206EC000FF7F0000000000FE00FCFF010000000040000004030000040000000400000000EB
:206EE0000000FCFF00000000000000F00000000000000000307500012C01000400000004CC
:206F000000000000CCF7FFFF000000000030DFFF0000000000000000001000040100000489
:206F200000000004000000009CFFFFFF1A0400000070FEFF00681000000000003075000408
:206F40002C0100040000000400000000E6FBFFFF000000000098EFFF000000000000000097
:206F6000204E00040300000400000004000000009CFFFFFFFF7F0000000000FE00FCFF0183
:206F800000000000204E00040300000400000004000000000080FFFFFF7F0000000000FE7A
:206FA00000FCFF0100000000400000040300000400000004000000000000FCFF000000008B
:206FC000000000F00000000000000000307500012C0100040000000400000000CCF7FFFF25
:206FE000000000000030DFFF00000000000000000010000401000004000000040000000066
:207000009CFFFFFF1A0400000070FEFF0068100000000000307500042C01000400000004F6
:2070200000000000E6FBFFFF000000000098EFFF0000000000000000657F367E107D807CCA
:20704000657B527A467940784177C476CE75DF74F47310739F72C271EA701770486F7D6ED4
:207060001A6E566D966CDA6B216B6D6A136A6469B8680F68696718677666D8653D65A46428
:207080000E64C4633263A26215628A614561BE603960B55F345FB55E765EFA5D805D085DD8
:2070A000915C1C5CE25B705BFF5A905A235AED5981591859AF584858E357B1574D57EB5644
:2070C0008A562B56CC550000C90092015B022403ED03B6047F0548061107D907A2086A09BD
:2070E000330AFB0AC40B8C0C540D1C0EE30EAB0F72103A110112C8128F1355141C15E215C4
:20710000A8166E173318F918BE19821A471B0B1CCF1C931D571E1A1FDD1F9F206121232209
:20712000E522A62367242825E825A82667272628E528A329612A1F2BDC2B992C552D112EB5
:20714000CC2E872F4130FB30B5316E322633DF3396344D350436BA366F372438D9388C39A4
:20716000403AF23AA53B563C073DB83D683E173FC53F73402141CE417A422543D0437A44A5
:207180002445CD4575461C47C34769480F49B449584AFB4A9D4B3F4CE04C814D204EBF4E77
:2071A0005D4FFB4F97503351CE51685202539B533254C9546055F5558A561D57B0574258BB
:2071C000D3586459F359825A0F5B9C5B285CB35C3E5DC75D4F5ED75E5D5FE35F6860EB60F9
:2071E0006E61F0617162F1627063EE636C64E8646365DD655666CF664667BC673268A66896
:2072000019698B69FD696D6ADC6A4A6BB76B236C8E6CF86C616DC96D306E966EFB6E5E6FD5
:20722000C16F22708370E27040719D71F9715472AE7207735E73B5730A745F74B2740475D5
:207240005575A575F37541768D76D87622776B77B377FA773F788478C77809794A7989798B
:20726000C879057A417A7C7AB67AEE7A267B5C7B917BC57BF87B297C597C887CB67CE37CBF
:207280000E7D397D627D897DB07DD57DFA7D1D7E3E7E5F7E7E7E9C7EB97ED57EEF7E097F09
:2072A000217F377F4D7F617F747F867F977FA67FB47FC17FCD7FD87FE17FE97FF07FF57FD8
:2072C000F97FFD7FFE7F00000500000000000000050000000000000005000000000000002E
:2072E00005000000000000000500000000000000A028240000000000000000000000000098
:20730000983A38100810F90FEE0FE60FE00FDB0FD70FD30FCF0FCB0FC70FC20FBC0FB50FB2
:20732000AD0FA40F9B0F900F850F7A0F6F0F640F5A0F4F0F460F3D0F340F2B0F230F1B0F46
:20734000120F0A0F030FFA0EF20EE90EE10ED70ECE0EC40EB90EAF0EA40E990E8F0E840E54
:207360007A0E700E670E5D0E550E4C0E440E3D0E350E2E0E270E210E1B0E150E0F0E090E6A
:20738000030EFE0DF80DF40DEE0DE90DE40DDF0DDA0DD40DCE0DC80DC30DBC0DB60DAF0D6D
:2073A000A70D9F0D970D8E0D850D7B0D700D640D570D490D3B0D2E0D250D1C0D120D080D5A
:2073C000FD0CF10CE00CC70C930C1C0C045500000000000055026400190310100F87A55541
:2073E000DB026464646464646464646401025500B80B3C870000000055020C0C96004B009A
:20740000960000000000646464646464646464640000000090016400FA004006C8000A00E7
:207420000A0080BB30080000010000000000000000000000000000000000000000000000CE
:207440000000000000000000000041410000000041414141000000000000000000000000A6
:2074600000000000000000006400A000BE000E01B400000000000000000000000000000087
:20748000000000000000000041564F4E49544F4D7401E8025C04D1054507B9082D0AA20BF9
:2074A000160D8A0EFF0F880100006400200302010002120300006400E8030201AE021D05B5
:2074C000BC026400140503016603AC07480364003408050100040000CC01640034080401EA
:2074E000000434094803640060090701CC04C40100006400480302010002BA0300006400C1
:20750000B0040201AE02E005BC026400360603016603320948036400340805010004000024
:20752000CC016400340804010004080B4803640060090701CC04DC0130020000A903020114
:2075400052017604BC020000E2040302E9016F0748030000B3050402AE02290BD403000091
:207560003408050300040000B00400003408040200040B023002640067030101EB00AE041D
:20758000BC0264001F0402014B01B00648036400B805030100022D0BD40364003408050279
:2075A000000400003A076400340804010004000000002110422063308440A550C660E77081
:2075C000088129914AA16BB18CC1ADD1CEE1EFF13112100273325222B5529442F772D6621B
:2075E000399318837BB35AA3BDD39CC3FFF3DEE36224433420040114E664C774A4448554DB
:207600006AA54BB528850995EEE5CFF5ACC58DD55336722611163006D776F6669556B4469A
:207620005BB77AA719973887DFF7FEE79DD7BCC7C448E5588668A77840086118022823385A
:20764000CCC9EDD98EE9AFF9488969990AA92BB9F55AD44AB77A966A711A500A333A122A1A
:20766000FDDBDCCBBFFB9EEB799B588B3BBB1AABA66C877CE44CC55C222C033C600C411CDA
:20768000AEED8FFDECCDCDDD2AAD0BBD688D499D977EB66ED55EF44E133E322E511E700E9A
:2076A0009FFFBEEFDDDFFCCF1BBF3AAF599F788F8891A981CAB1EBA10CD12DC14EF16FE192
:2076C0008010A100C230E3200450254046706760B9839893FBA3DAB33DC31CD37FE35EF31A
:2076E000B1029012F322D2323542145277625672EAB5CBA5A89589856EF54FE52CD50DC5DA
:20770000E234C324A01481046674476424540544DBA7FAB79987B8975FE77EF71DC73CD799
:20772000D326F2369106B01657667676154634564CD96DC90EF92FE9C899E9898AB9ABA959
:207740004458654806782768C018E1088238A3287DCB5CDB3FEB1EFBF98BD89BBBAB9ABB19
:20776000754A545A376A167AF10AD01AB32A923A2EFD0FED6CDD4DCDAABD8BADE89DC98DD9
:20778000267C076C645C454CA23C832CE01CC10C1FEF3EFF5DCF7CDF9BAFBABFD98FF89F99
:2077A000176E367E554E745E932EB23ED10EF01E00000000B71DC1046E3B8209D926430D61
:2077C000DC7604136B6BC517B24D861A0550471EB8ED08260FF0C922D6D68A2F61CB4B2B71
:2077E000649B0C35D386CD310AA08E3CBDBD4F3870DB114CC7C6D0481EE09345A9FD524121
:20780000ACAD155F1BB0D45BC2969756758B5652C836196A7F2BD86EA60D9B6311105A67B0
:2078200014401D79A35DDC7D7A7B9F70CD665E74E0B6239857ABE29C8E8DA1913990609520
:207840003CC0278B8BDDE68F52FBA582E5E66486585B2BBEEF46EABA3660A9B7817D68B3F0
:20786000842D2FAD3330EEA9EA16ADA45D0B6CA0906D32D42770F3D0FE56B0DD494B71D9A0
:207880004C1B36C7FB06F7C32220B4CE953D75CA28803AF29F9DFBF646BBB8FBF1A679FF30
:2078A000F4F63EE143EBFFE59ACDBCE82DD07DEC77708634C06D4730194B043DAE56C53950
:2078C000AB0682271C1B4323C53D002E7220C12ACF9D8E1278804F16A1A60C1B16BBCD1F70
